:020000040800F2
:10000000000002203D3301088333010885330108D5
:1000100087330108893301088B3301080000000091
:100020000000000000000000000000008D33010807
:100030008F330108000000009133010839C6000821
:1000400097330108993301089B3301089D33010858
:100050009F330108A1330108A3330108A533010828
:10006000A7330108A9330108AB33010849E00008B0
:10007000AF330108B1330108B3330108B5330108C8
:10008000B7330108A1E00008BB330108BD33010804
:10009000BF330108C1330108C333010861170108E8
:1000A000C7330108C9330108CB330108CD33010838
:1000B000CDF90008D1330108D3330108D5E0000899
:1000C000D7330108D9330108DB330108DD330108D8
:1000D000DF330108E13301084DC60008E5330108AC
:1000E000E7330108E9330108EB330108ED33010878
:1000F000EF330108F1330108F3330108F533010848
:10010000F733010889F30008FB330108FD330108C8
:10011000FF330108013401080334010805340108E4
:1001200007340108093401080B34010869F3000899
:100130000F34010811340108133401081534010883
:1001400017340108193401081B340108F5F60008BA
:100150001F34010821340108233401082534010823
:1001600027340108293401082B3401082D340108F3
:100170002F340108313401083334010835340108C3
:10018000373401083934010810B5054C237833B9E8
:10019000044B13B10448AFF300800123237010BD5A
:1001A0003801002000000000D07C0108084B10B589
:1001B0001BB108490848AFF300800848036803B939
:1001C00010BD074B002BFBD0BDE81040184700BF07
:1001D000000000003C010020D07C01083801002014
:1001E00000000000154B002B08BF134B9D46A3F5E4
:1001F000803A00218B460F461348144A121A13F016
:10020000CAFD0F4B002B00D098470E4B002B00D09F
:1002100098470020002104000D000D48002802D05E
:100220000C48AFF3008013F0D5FC2000290000F04B
:1002300013F813F011F900BF0000080000000220BD
:1002400000000000000000003801002048C4012028
:1002500000000000000000002DE98048D9B00EF039
:10026000AFFFBD4B9A6802F00C02042A09F0FD8131
:10027000082A09F0DF81B94BB94A1A60B64EB94F66
:10028000B168B94CB94ADFF818C3B948B94DC1F3E0
:1002900003114FF0C808795C1F68CCF8008027FA7A
:1002A00001F18F09A4FB0774A409196004F1FF3E52
:1002B0000721F02400270523C2F804E085F8234035
:1002C0009760116003608DF86A70336C4FF0804462
:1002D00043F001033364238823F45C731B044FF061
:1002E00001081B0CD1222380E1622285A4F814802E
:1002F000A3899BB243EA0803A3811C220F2316A8FB
:100300008DF858208DF859308DF85A308DF85B8073
:100310000CF012FB2288984B92B242EA080222802B
:100320001A68B2F5E13F09F078814FF4E1321A60C2
:10033000336B924D43EA08033363336B43EA08039C
:100340003363336C04F5003443F400333364236ABD
:1003500023F470632362236A43F4E0632362236A15
:1003600023F470432362236A022143F4E0432362AF
:100370000322204604238DF85C1016A98DF85D2019
:1003800016938DF85E708DF85F800CF081FA204630
:10039000082316A916930CF07BFAAB896FEA434346
:1003A0006FEA53439BB2AB812B8A23F440531B0467
:1003B0001B0C2B82AB899BB223F4B05323F00C03AC
:1003C00043F00C03AB81AB8A23F440731B041B0C7A
:1003D000AB8218A80CF010FAAA891A9B674812F48D
:1003E000004F03EB8303664A03EB8303A2FB032363
:1003F00014BF5A0C9A0C634BA3FB02418489480931
:10040000642100FB11210201200409F1FC80090193
:100410003231A3FB0113C3F3431343EA0201574BE9
:10042000594A89B21981998989B241F40051998157
:10043000136843F02003136000242623012518A825
:100440008DF860308DF861408DF862408DF8635012
:100450000CF072FA474B4D4ADA6031238DF8635045
:100460008DF861408DF862408DF8603018A80CF06E
:1004700063FA9DF863303B2101228DF860108DF8FE
:100480006120002B49F0AC81414B4FF00062C3F872
:100490008420314D3F4C2B6B3F4F43F00C032B63BB
:1004A000636A23F00F036362636A43F00C036362C1
:1004B000636A23F0F0036362636A43F0C00363621C
:1004C000636A23F470636362636A43F44063636244
:1004D000636A23F470436362636A43F44043636274
:1004E000636A23F470236362636A43F440236362A4
:1004F0003B6A23F470633B623B6A43F440633B62B4
:100500004FF4706202232046002618A94FF001081C
:1005100018928DF865308DF864308DF866608DF82E
:1005200067800CF0B5F93846042318A918930CF02D
:10053000AFF920464FF4805318A918938DF86760DF
:100540000CF0A6F96B6C154843F400636B642B6BDD
:1005500043F480032B6325E0003802407000002044
:100560000024F40060000020632D3E0510E000E050
:100570001000002000ED00E00407002000440040CF
:10058000C5B3A2911F85EB510C4400400006FA054B
:1005900000E100E000080240000C0240F45C0108A9
:1005A000780000200CF006F9434B444918689F88F6
:1005B00012901A4653F8080F149052F8100F9C88A6
:1005C0009388ADF85C300A683D4BADF84C709A42A8
:1005D000ADF85440169049F075805523F022022161
:1005E00018A88DF861308DF8602012F019FC0346D0
:1005F000002809F0FA80334B0D931B68002B08F09C
:10060000FC87314E11AD3368022B0CBF2F483048A8
:100610000CF0D0F82F4F3B68002B40F00F83DFF831
:10062000C480DFF8C4B0DFF8C4901C469A4618A80E
:10063000C5F80080CDF848B0CDF860800BF0B4FA72
:10064000031E4FF0000212A9284651DB59F823601F
:100650000EB186F800A0129E0EB186F800A0129E80
:1006600049F823600CF090F90328064608F07A87D1
:10067000002808F0B887184B0A931B68174AD868F7
:10068000174914F089FC731E122B08F2A287DFE8C9
:1006900013F08C47824778475F4747033E03350393
:1006A0002C03FF02F6023700ED0223031A031103A5
:1006B0000803E402DB029647BC5B0108F403002058
:1006C000801A060018B8012044B801202C5D0108EA
:1006D000445D01086803002028010020B45D010882
:1006E000BC5D0108745D01082C2000207C220020E4
:1006F000BC4B0A931B68BC4ABC49D86814F04CFC3C
:100700000A9BBB481B682022DB68012114F0A4FC73
:10071000DFF8F4A2B74CDAF83030B74DB74EB84F27
:10072000DFF8E88243F00103CAF83030C0234FF00D
:100730000009204618A918934FF001038DF8643082
:100740008DF865908DF866908DF867900CF0A0F8A4
:10075000402323834FF080032383DAF8303043F0C3
:100760000403CAF830304FF4005428464FF0010318
:1007700018A98DF8643018948DF865908DF86690FE
:100780008DF867900CF084F86C83DAF8303043F021
:1007900018034FF0030BCAF8303030464FF2B373F2
:1007A00018A918934FF680758DF864908DF86790AE
:1007B0008DF865B00CF06CF8384618A918950CF057
:1007C00067F8DAF8303043F07803CAF830304CF28A
:1007D00033733046189318A94FF002038DF8643034
:1007E0008DF865B08DF866908DF867900CF050F834
:1007F000336A23F00F033362336A43F00C0333622E
:10080000336A23F0F0033362336A43F0C003336288
:10081000336A23F470233362336A43F44023336230
:10082000336A23F470033362336A43F44003336260
:10083000736A23F00F037362736A43F00C037362ED
:10084000736A23F0F0037362736A43F0C003736248
:10085000736A23F470637362736A43F44063736270
:10086000736A23F070637362736A43F04063736268
:10087000736A23F070437362736A43F04043736298
:10088000384618A918950CF003F83B6A5D4D23F023
:1008900070433B623B6A43F040433B627B6A23F018
:1008A0000F037B627B6A43F00C037B627B6A23F05D
:1008B000F0037B627B6A43F0C0037B627B6A23F4B4
:1008C00070637B627B6A43F440637B627B6A23F4E0
:1008D00070437B627B6A43F440437B627B6A23F410
:1008E00070237B627B6A43F440237B627B6A23F440
:1008F00070037B627B6A43F440037B627B6A23F074
:1009000070637B627B6A43F040637B627B6A23F0A7
:1009100070437B627B6A43F040437B62304618A998
:1009200018940BF0B5FF736A23F470037362736A53
:1009300043F4400373623046802318A918930BF0E8
:10094000A7FF336A23F070433362336A43F04043B6
:100950003362DAF838304FF0204443F001000F21C1
:100960000D2241F21003CAF8380018911A92CDF8FE
:100970006490CDF86C90CDF87090CDF87490CDF86F
:1009800078902360189F1E9B199E1A981B9A1C9999
:100990003B4343EA061343EA002343EA02431D9A1A
:1009A00043EA015343EA02626FF0704362602B60D6
:1009B00023684FF0C04543F0010323604FF001036B
:1009C0002B8005200BF018FEE22223232A80A8F8B2
:1009D00000304FF00203A8F80030E02404264FF066
:1009E000010315E028010020B45D0108BC5D010889
:1009F000245F01080000024000080240000C024091
:100A000000100240040100A000380240000008600D
:100A1000A8F8006064202C80A8F800300BF0FAFDE4
:100A2000E62393222C80B021A8F800B01F202B8051
:100A3000DF27A8F80060B423A8F80020E8264FF0CC
:100A40000102A8F800404FF0080E29804FF0330C47
:100A5000A8F800901721A8F800901224A8F800B078
:100A60004FF0B60AA8F80000A8F800201820A8F84F
:100A70000070F022A8F80090AE4F2B80A8F800B0CC
:100A80002923A8F800604FF00206A8F80090A8F803
:100A900000C0A8F800E0A8F80090A8F800B0A8F8F6
:100AA0000090A5F800A0A8F80060A8F80040A8F8F9
:100AB0000090A8F80000A8F800B0A8F80090A8F8E6
:100AC00000102A80A8F800B02B803A689A4C12F0E7
:100AD000010F0CBF73464B46910748BF43F002031A
:100AE000520748BF43F001034FF0C04699B2BE22FF
:100AF000362333800025218006203280FF21012209
:100B000020802180284622802180258040F21F31CC
:100B100025803A60338025800EF0F2FB284640F2B3
:100B2000DF110EF0D9FB2C232946224633804FF4E7
:100B300048754FF4F073013B11804FF00004FAD177
:100B4000013DF6D12946FF2010F098FE7B4B93E83B
:100B500003007B4B18647A48A3F844100A0C80F811
:100B60004620774A7749784882F881500123C2F8B5
:100B7000C450147082F8C94082F8C84082F88030AE
:100B800012F0F6FE0546002800F00D816F4F2A4650
:100B90004FF4807118A812F0F3FD002800F0FE80D9
:100BA000232118A814F022FE0446002809F04F85DE
:100BB0000023037018A814F039FE0028E7D0431E64
:100BC00018A90B44C01A1A78093AD2B227FA02F1CE
:100BD000172A01F0010204D882F00101002A49F02D
:100BE00040853D2118A814F001FE03460028CED010
:100BF00000220270564918A85C1C14F0D9FD064664
:100C0000002809F04B85534918A814F0D1FD064679
:100C1000002809F03985504918A814F0C9FD0028AA
:100C200049F046854D49204614F0C2FD002849F0A0
:100C30001F85434A012382F88030A8E7484B494882
:100C40000A9314F07BFD63E50A9B47481B68222248
:100C5000DB68012114F000FA5AE50A9B43481B683F
:100C60002A22DB68012114F0F7F951E50A9B40487C
:100C70001B681822DB68012114F0EEF948E50A9B95
:100C80003C481B682222DB68012114F0E5F93FE5AE
:100C90000A9B39481B682122DB68012114F0DCF92A
:100CA00036E50A9B35481B683B22DB68012114F0BE
:100CB000D3F92DE50A9B32481B684122DB680121EC
:100CC00014F0CAF924E50A9B2E481B682422DB682D
:100CD000012114F0C1F91BE50A9B2B481B681D225A
:100CE000DB68012114F0B8F912E50A9B27481B685C
:100CF0002722DB68012114F0AFF909E50A9B24489B
:100D00001B683922DB68012114F0A6F900E50A9B73
:100D100020481B681C22DB68012114F09DF9F7E4D0
:100D20000A9B1D481B681A22DB68012114F094F904
:100D3000EEE400BF9400002000000860A8600108F5
:100D400074A50120B0600108B460010813008000A0
:100D5000C0600108C8600108CC600108D8600108C3
:100D600028010020785D0108586001082C60010806
:100D7000485F0108005F0108DC5E0108F05F0108C0
:100D8000AC5F0108845F0108645F0108B45E01087C
:100D9000785E0108585E01083C5E01080CF09EFF79
:100DA000284612F0BFFBAF4BD3F8C42012B9012282
:100DB000C3F8C4208022AC49AC4814F03FFD11F0C8
:100DC00023FE0DF035F9A74BD3F8C430DE0752D51A
:100DD000A74CA848236B43F002032363002580231C
:100DE00018A918938DF864508DF867500BF050FDDA
:100DF000616CA14AA14B41F480416164D16821F446
:100E00007041D160D16841F48051D160196821F0FE
:100E100080011960596821F080015960196841F01A
:100E200080011960996821F080019960D96821F0EA
:100E30008001D960D2F80C3443F08003C2F80C343E
:100E400016A8012317228DF859308DF85A308DF8E5
:100E50005B308DF858200BF06FFD236B854843F015
:100E60000203236318A940238DF864508DF867505E
:100E700018930BF00DFD7B4BD3F8C4309D0708F1A0
:100E80000F85784BD3F8C4305B0724D50024784B0A
:100E9000199418941A6B7A4F7A4842F01402FF267C
:100EA0001A6301253E833F2318A98DF864408DF80D
:100EB000654018938DF867500BF0EAFC384618A986
:100EC00018968DF864508DF866508DF867408DF84F
:100ED00065400BF0DDFC6C4B08936C4B02936C4B44
:100EE00009936C4B1B68002B40F0FA826A4B6A4AEC
:100EF0001B68002B40F01982684B1B78002B40F0D8
:100F00008A80674B1878002840F08580654A664BD8
:100F100011881B78654A634D1180634A002B62D0AB
:100F2000634B634C1B78002B5DD010708B0B614AB8
:100F3000207052F82320C1F30D03D35C594A762B5D
:100F400004BF4B1C2B805C4B10881B88013B9AB262
:100F5000594BB2F5804F1A800DD3B2F5B64F02D27D
:100F6000564901230B70930BC2F30D01514A52F8FD
:100F70002320030A5354504B1B88013B9AB24E4B1B
:100F8000B2F5804F1A800CD3B2F5B64F02D24B495E
:100F900001230B70930B4749C2F30D0251F8233024
:100FA0009854474B1B78012B40F22384022B1AD113
:100FB000444B454A1B7816683E4C1902481C821364
:100FC0008B0B54F8225054F82340C0F30D023E48D6
:100FD00006F11303C1F30D010360AA5C635C03EB2C
:100FE0000223304A13802F4B1A8840F262539A42F0
:100FF00008F0AF8740F2C2439A4208F07787334B3C
:101000001B7803F0FF02002B00F00384304B1B68B9
:10101000002B48F04C86234B264C19882D4B186822
:101020008B0BC1F30D0254F823309C5C002877D061
:1010300043F6FE43994202F0AB8043F6FF439942E8
:101040006ED1254B1B68002B02F09A80234B244A5B
:101050001B682249D25C0133802B0B6008BF002340
:10106000D2B23FE074A50120B4A5012054BC0120F8
:10107000003802400004024000380140003C0140BA
:1010800000080240001002400040001000BD012096
:101090004065012060220020000700204EBD012095
:1010A000ACBD0120AABD0120DCBC0120F4BC0120A4
:1010B0005C02002044A501204EBC0120A5000020B8
:1010C00050BC012019070020B0BD01207400002091
:1010D000201F0020A4BD012010070020F0030020E5
:1010E0006C03002008BF0B6072B60B4B0A491B68EB
:1010F000013B0B6062B6029B02999B79CA7143F077
:1011000001030D2A8B710BD1044B5B6803F5E1528F
:101110001C322023137003E01007002044A5012097
:10112000FF2C09F2FF85DFE814F09B4DCB4D9F4566
:10113000AE4D4F4D892B5B2BB64F9D4F614F3B4FB3
:10114000174FCD4E754E564E885068503E501B502E
:101150001051C650752C562CFC53E453A8538E5393
:10116000F3544554A854374E235205529A513B51DB
:10117000BE527552E152112BD930BB300530C42F0D
:1011800096314E31672F492F1B2FFD2ED62E9C2EC8
:10119000802EEF2D3B2DD92C89336B333133F43234
:1011A000D6328C3234321532D734AE34AE34AE341B
:1011B000AE34AE34AE341734AE34EC33EC33EC33FF
:1011C000EC33EC33EC337F34EC3346344634463482
:1011D0004634463446341E354634302B302B302BC3
:1011E000302B302B302BF53E302BD93ED93ED93E1B
:1011F000D93ED93ED93EB93CD93E8F3C8F3C8F3C3D
:101200008F3C8F3C8F3C053E8F3C9F3D9F3D9F3DDB
:101210009F3D9F3D9F3D6B369F3D42364236423655
:10122000423642364236074142365E3E5E3E5E3EC2
:101230005E3E5E3E5E3E91405E3E1B3C1B3C1B3C68
:101240001B3C1B3C1B3CD53F1B3C2D3D2D3D2D3DF0
:101250002D3D2D3D2D3D333F2D3DE12BE12BE12B50
:10126000E12BE12BE12B4F39E12BEA38EA38EA3860
:10127000EA38EA38EA38ED3AEA38A038A038A03837
:10128000A038A038A0388D3BA038053A053A053A79
:10129000053A053A053A5F3A053AD135D135D135A7
:1012A000D135D135D1350337D135CE36A236783662
:1012B0007138A9370B38B12AA7298129EE29572976
:1012C0003B0ACC0971090D09BC0896086A08400858
:1012D0002108BF076A070D07F724D124A4247A2424
:1012E0005D24FB23D8237423CD25A62575254B2506
:1012F000D526732641270406E311AD119B11711108
:10130000A5124312C712A1102A1104113823DA10B2
:10131000F1069106E5223E06B80F920F7B0F510FA2
:101320002F0FCD0EBC0E5F0ECD030024C249C34863
:10133000146012F01DFB0746002801F01C878DF891
:101340003D408DF83E408DF83F400CF071FEBC49A9
:10135000384611F0DBFABB49384611F0D7FABA49E2
:10136000384611F0D3FAB949384611F0CFFAB849E6
:10137000384611F0CBFAB749384611F0C7FAB649EA
:10138000384611F0DDFAB549384611F0D9FAB449BA
:10139000384611F0BBFA0DF13F01384611F0B6FAAC
:1013A0000DF13D01384611F0B1FA9DF83D30FF2BAB
:1013B00001F0DB8603F0200303F0FF02002B41F075
:1013C000C88615469DF83D30A64AA749C3F3420397
:1013D0003846137011F09AFAA449384611F096FA7B
:1013E000A349384611F092FAA249384611F08EFA14
:1013F000A149384611F08AFAA049384611F086FA18
:101400009F49384611F082FA9E49384611F07EFA1B
:101410009D49384611F07AFA9C49384611F076FA1F
:101420009B49384611F072FA9A49384611F06EFA23
:101430009949384611F06AFA9849384611F066FA27
:101440000DF13E01384611F061FA9DF83E30002B57
:1014500001F07B86924A012313709249384611F0BD
:1014600055FA0DF13E01384611F050FA7A4A9DF8CE
:101470003E3014888C4A03F003031370002C00F0F4
:101480000983D5B94FF4804401250DF13E0138465A
:1014900011F03CFAB4F5B64F38BF84489DF83E20B1
:1014A00038BF0570A30B8248C4F30D0150F82330F8
:1014B0000134B4F5803F5A54E7D1674B7D4A1B880D
:1014C00013807D4B00241C707C4B1C707C4B1C706B
:1014D0007C4B38461C6012F025F87B4B1C700BE5EA
:1014E0007A4B7A4A1B787A490133DBB20020102B01
:1014F0001370086000F0BD825A4B1978754B1B7849
:101500008B422AD0744B33F8114000942F2340F2C1
:101510004722102108200DF007FF40F2AF132722C9
:101520003021082000940DF0FFFE40F2AF1340F28E
:10153000472230214FF40A7000940DF0F5FE40F27E
:10154000CF1340F2472200944FF4D87108200DF0D9
:10155000EBFE444B5F4A1B7813705C4B1B780C937B
:1015600023B1524B1B78002B3FF4C0AC4FF48043A7
:101570000B930B9B9B1003F038010B9BC3F30222D0
:101580005B110A4303F0C00342EA0301CB085A018E
:101590004B0003F1300BBDF82C3004933723079335
:1015A000282302F5B04205933823069203934B4B50
:1015B000BDF814601B68002B00F0F580049B099AAD
:1015C000C3F30D0312F803A0454B09931946069B7C
:1015D000C3F30D02434B8A5C1B7843B1424B049921
:1015E0000B44A3F580431B78534500F0E6803E4B47
:1015F00004990B44A3F58043150683F800A000F17D
:10160000EA80C2F3C20802F00709540607D508F1C0
:10161000080209F108035FFA82F85FFA83F9BAF168
:10162000000F00F08380BAF1FF0F00F0DE8080250C
:101630000BF1010767E000BF14610108241F0020BF
:1016400007BD012006BD012001BD012000BD012014
:1016500005BD012004BD0120AABD01204EBC012012
:101660001907002054A5012003BD012002BD01205F
:10167000E1BC0120E0BC0120E3BC0120E2BC012070
:10168000E5BC0120E4BC0120E7BC0120E6BC012050
:101690000BBD01200ABD012009BD012008BD0120AC
:1016A000DCBC01201C1F002050BC0120A500002034
:1016B00044A50120F4BC01204DBD01204EBD0120F8
:1016C000ACBD0120B0BD01205C020020580100200B
:1016D000602200205C000020D45B010840A50120AE
:1016E00040650120180700201C070020664C34F8D4
:1016F000194000940DF018FEB31C9EB2039B9E424D
:101700004FEA55051DD01AEA050F3B4606F10102C6
:1017100059463046EAD15C4B33F818300093721CBE
:101720003B46594630460DF0FFFDE5E7564B33F892
:1017300018300093079A05980BF1010359460DF0F4
:10174000F3FD039B0499069A059810339BB203930B
:10175000079B10300131013289B292B21033B0F5DB
:101760000A7F05900491069207937FF420AF0B9BAC
:101770002033B3F5B04F0B937FF4FBAE434B444A99
:101780001968444B4448002914BF114619464FF4C8
:10179000407212F0F5FA414901220A70404A0023D2
:1017A0001370FFF7A3BB049B089AC3F30D0312F851
:1017B00003A03C4B0893194609E7374B06990B44A5
:1017C000A3F5B0431B7893427FF411AF0C9B002B21
:1017D000B7D11706B5D5344B1B78002B3FF411AFAA
:1017E000C2F3C20902F007080FE7274B33F819309C
:1017F0009FE72E4B2D491B6803F10D020A602C4A0E
:10180000382313802B4B1B7803F0FF02002B7FF44F
:10181000FDAB294B1046196810F030F80D9B1B6882
:101820000BB110F003F80027DFF88CA0DFF88C80F4
:10183000DFF88C9011E0B2F5B97F08F0F38240F246
:1018400075139A4206D12FB11B4B013F38461968D8
:1018500010F014F801200DF0BFFA10F06FF87628A0
:10186000024609F092805A2A02D0E4D8292AF1D1FE
:10187000062FEFD8DFE817F08F496E495C492249FF
:10188000A9487A489B4800BFD45B010840A50120C5
:10189000407D012000580010F803002018070020A8
:1018A000A5000020004000106C220020B0BD0120E7
:1018B000AABD012074000020EC03002074A50120C3
:1018C000C40000207F4B80491B8808887F4A013B69
:1018D00099B2431C7B48126801807C480B32B1F5F9
:1018E000804F026098B20DD3B1F5B64F02D2784A5C
:1018F000012313708B0B774AC1F30D0152F823209B
:10190000030A53546F4B1B88013B9AB26D4BB2F5DF
:10191000804F1A800CD3B2F5B64F02D26C49012326
:101920000B70930B6B49C2F30D0251F8233098549E
:10193000654A38231380684B1B7813B9674B1B78B3
:1019400053B1674B664A1B78002B52D06249002383
:101950000B70624913700B70624B5C4A1B68126813
:101960005A4913F0030F40F29F2318BF4FF4287316
:101970009A42FFF4B6AA5C4804685C48D0F8C400F8
:10198000D31A42070B6004F10A0542D4574BD3F82F
:10199000C4309B0702D500200DF01EFA0D9B1B687A
:1019A0006BB1534B196800292FD1524B514A1B6818
:1019B0000133642B136002D111600EF08FF84B4B92
:1019C000D3F8CC30C3B14C4B1D60464B46491A6826
:1019D000494B1B680B60531C424A642B1360114631
:1019E0007FF47FAA00220A60444A01231370FFF7A4
:1019F00078BA01231370AFE73F4B1B689D42E4D9CF
:101A00003D4B1B689D42F7D8DFE701200EF0C0F880
:101A1000D5E73B4B3A4C1B68F3B1012BB6D1394BA0
:101A20001B69DBB203F0200203F03F0102F0FF0369
:101A30000AB9354A1370354B1A68184661F01F030E
:101A400033498B54531C082B03602D4A04BF0023D9
:101A500003600023136099E72C4B2E481B6801217B
:101A600001FA03F3DB43DAB2FF23438302832160ED
:101A70008CE7294B10702949294A1B78097812787C
:101A8000254CB3FA83F35B098A4223707FF43AADA5
:101A90000C906BE518A9384610F052FFBDF8603085
:101AA0000949172B38460CBF0225032510F048FFC3
:101AB000BDF86030023B9BB2ADF86030002B43D1E3
:101AC0005CE000BF4EBC0120AABD0120B0BD0120DA
:101AD000A500002044A501204EBD0120ACBD012081
:101AE0004DBD0120682200207022002074A5012035
:101AF0003CB8012074220020540100205C02002028
:101B000078220020001002407400002064030020AE
:101B100034250020000802406C22002054A501203A
:101B20005C0000209DF83E30012B40F29780022D92
:101B300000F08580043B012B40F28580621CBDF8DB
:101B4000603094B2A34219D90DF13E01384610F02D
:101B5000DDFE002CE6D0022CF0D1AF4B1B68B3F5B4
:101B6000004FEBD19DF83E20FD217F200CF0F6F9CF
:101B7000621CBDF8603094B2A342E5D80023DFF8C0
:101B8000C8A28DF840308DF842304FF6FF7B18A97F
:101B9000384610F0D5FE0DF14201384610F0B6FE81
:101BA000BDF860305B4504BF4FF48043ADF8603052
:101BB000994B1B680CBF4FF000094FF00109B3F5BA
:101BC000804F9DF8423000F08180033B934A52F8E9
:101BD0002380BDF8603023B3002634460DE09DF825
:101BE0003E50ED2D5BD0731C08F806509EB2621C6F
:101BF000BDF8603094B2A34213D90DF13E013846CE
:101C000010F084FEB9F1000FE9D19DF83E3008F8DC
:101C10000630731C9EB2621CBDF8603094B2A342C1
:101C2000EBD87B68013B002B7B605BDB3A68531C85
:101C30003B6013781846394612F04AFFA7E7033B8A
:101C4000012B3FF67BAF744B1B68B3F5804F7FF4DD
:101C500075AF734B1B78E3B1724B09E06E4B1B6899
:101C6000B3F5804F3FF46AAF6D4B1B788BB16E4B71
:101C700000936E4A6A4B6E48802113F067FD00287E
:101C8000FFF63AA910F0C0FE634B18680CF05EF83E
:101C900054E780226449664813F0D0FDF2E70DF165
:101CA0003E01384610F032FE9DF83E20631CED2ABE
:101CB00099B221D008F80650731C9AB29DF83E30B4
:101CC00008F80230B31C0C469EB290E7052B01F0D9
:101CD0007C82082B01F07582042B0CBFD0464FF09C
:101CE000000876E70A9B3946186812F04BFB03465A
:101CF00001303FF4E2AB9DE710A9384610F006FE34
:101D00000DF13E01384610F001FE9DF84020E31C25
:101D10009CB2002A3FF46BAF00219DF83E3008F8DA
:101D200006309DF840200131731C91429EB2F4DBD5
:101D30005DE7404B404C1D88404B1968029BD879A9
:101D40006B1C9BB29A0B073154F82220394C23802C
:101D50003A4CC3F30D032160D35C394A1840029B0F
:101D6000D8719379002803F00D8503F0BF030706AF
:101D7000937143F10A8563F07F039371029B029E86
:101D80009979304B2E4C185C01F0FC0242F01003A4
:101D9000B371002803F0EF8442F01403A371254AC5
:101DA000AB1C1380C7E5234B234D1C88234B1968BC
:101DB000029BD879631C9BB29A0B073155F82220FD
:101DC0001C4D2B801D4DC3F30D032960D35C1C4AB1
:101DD0001843029BD8719379002800F0A98003F082
:101DE000BF030506937140F1A68063F07F039371F2
:101DF000029B029D9979134B1A5C114801F0EC0388
:101E0000AB71002A00F0908043F004038371094A0B
:101E1000A31C13808FE500BFF0BC0120E062010825
:101E200074A5012040610108A8600108386101081B
:101E300054BC0120AABD012044A50120B0BD012051
:101E400000BD0120F45B0108008000108F4B90481A
:101E50001C88029B9D79631C9BB29A0BA11C50F8B5
:101E600022008A4A1380C3F30D0289B28B0B805C77
:101E7000874A52F82320854B1980C1F30D032F06A2
:101E8000D35C824900EB03239EB237D4814B824A54
:101E90001B881068013BE11C9AB200F1110388B263
:101EA0007C490A807C49B2F5804F0B600DD3B2F5B6
:101EB000B64F02D2794901230B70930BC2F30D0187
:101EC000734A52F82320030A5354724B1B88013B78
:101ED0009AB2704BB2F5804F1A800CD3B2F5B64F60
:101EE00002D26E4901230B70930B6949C2F30D02B4
:101EF00051F823309854654B1E801CE5664BE21C5C
:101F00001B680A80644A0A33136014E5624B5F4A17
:101F10001B686149128804330B605C4901320A80F6
:101F20005F4A0023137006E521F0170383716EE703
:101F300043F040039371029B029A9B7903F07F0365
:101F4000937155E7514B524F1E88534B55481D68AE
:101F5000029BDC79731C9BB29A0BC3F30D0157F8FB
:101F600022204A4F3B80EB1D4B4D2B60515C04F00F
:101F70000F0201F00F03D31A13F0100F837914BF6F
:101F800043F0100323F01003837181EA0403621A03
:101F90001F0695B273D584EA020318066FD5029B1B
:101FA00002999B7943F004038B71029BDA713D4ADD
:101FB0009379E9054CBF43F0010323F001039371CA
:101FC000029B029A9B79314915F0FF0F14BF23F051
:101FD000400343F040039371029B029A9B792F06C2
:101FE0004CBF63F07F0303F07F039371029BB21C2D
:101FF0009B790A80029A43F0020393719BE4029B4F
:1020000025489978DA78234B00681B8842EA012238
:10201000013B204914B29AB20A801F4900F10B0318
:10202000B2F5804FA0B20B600DD3B2F5B64F02D21D
:102030001A4901230B70930BC2F30D01144A52F895
:102040002320030A5354134B1B88013B9AB2114BB4
:10205000B2F5804F1A800CD3B2F5B64F02D20F49B9
:1020600001230B70930B0A49C2F30D0251F8233080
:102070009C54064B054A1B88013313805BE4029B8A
:1020800002999B7923F004038B718EE7AABD01208E
:1020900044A501204EBC0120B0BD0120A5000020B8
:1020A000DCBC012000BD0120A14BA2481C88029B82
:1020B0009D79631C9BB29A0BA11C50F822009C4A8C
:1020C0001380C3F30D0289B28B0B805C994A52F8DE
:1020D0002320974B1980C1F30D039549D35C00EB86
:1020E00003239EB2EB0738D4934B944A1B881068A5
:1020F000013BE11C9AB200F1110388B28E490A80BB
:102100008E49B2F5804F0B600DD3B2F5B64F02D2B7
:102110008B4901230B70930BC2F30D01854A52F8D2
:102120002320030A5354844B1B88013B9AB2824BF1
:10213000B2F5804F1A800CD3B2F5B64F02D2804967
:1021400001230B70930B7B49C2F30D0251F823302E
:102150009854774B1E80FFF7EEBB784BE21C1B6850
:102160000A80764A0A331360FFF7E5BB704B714C67
:102170001B88724A01339BB2990B106854F82110E6
:102180006B4C029A23806D4CD2790B30C3F30D0354
:102190002060C95C029B18780BF0E0FE644B644A37
:1021A0001B8801331380FFF7C6BB614B1C88634B50
:1021B0001E68029B9D79631C9AB2A31C98B2910B76
:1021C0005C4B53F821105A4B1A8006F10A035B4E00
:1021D000C2F30D023360895C564A830B52F8232008
:1021E000534B1880C0F30D03D35C514A01EB03231A
:1021F000E9079BB248BFE31C1380FFF79CBB4E4B23
:102200001D884E4B1C684A4B1F886B1C98B2A90B4B
:1022100004F10A03474C820B54F82140454951F818
:102220002260464A1360C5F30D03C0F30D01E25C62
:10223000414B029C1880735C42EA03231BB2C3F338
:102240000720E3703C4BA070A91C1980384B7A1C06
:102250001A80FFF770BB029B9B79D8075CD4364B82
:102260001C88364B1D68631C98B2820B05F10B036A
:10227000A10B304D55F8211055F822502F4A13600C
:10228000C4F30D03C0F30D02C95C2B4B1880AB5C8B
:1022900041EA032326490B80274BA21C1A80FFF733
:1022A0004ABB254B22491B880888244A013B99B226
:1022B000431C21481268018020480B32B1F5804F41
:1022C000026098B20DD3B1F5B64F02D21C4A012379
:1022D00013708B0B174AC1F30D0152F82320030A28
:1022E0005354154B1B88013B9AB2134BB2F5804FE8
:1022F0001A800CD3B2F5B64F02D2114901230B70EC
:10230000930B0C49C2F30D0251F823309854084A3C
:1023100008231380FFF70FBB084B08491A68044BCA
:1023200005321B880A60024A01331380FFF703BBA2
:10233000AABD012044A501204EBC0120B0BD012052
:10234000A5000020904B91481F88914B914E1B682F
:102350000393029B9C79DD797B1C9BB29A0BC3F3A0
:102360000D0150F8222088480380039B88480733DA
:102370000360505C05F00F0304F001010B4400F012
:102380000F021A4443191944D3064CBF44F01003FA
:1023900024F01003B37180EA0503DB0940F08A8062
:1023A00085EA01031E0640F18580029B029A9B7913
:1023B00043F004039371774A029BD9719379CD0559
:1023C0004CBF43F0010323F001039371029B029A77
:1023D0009B7911F0FF0F14BF23F0400343F040033B
:1023E0009371029B029A9B790C064CBF63F07F03AA
:1023F00003F07F039371029B63499B79BA1C0A80A7
:10240000029A23F002039371FFF795BA5E4B1C8882
:102410005F4B1D68604B1E88631C9AB2A31C98B268
:10242000910B5A4B53F82110574B1A8005F11103A9
:10243000574DC2F30D022B608D5C544A830B52F84A
:102440002310514B1880C0F30D03721ECB5C05EBBB
:102450000323E11C92B29CB24F4BB2F5804F88B27D
:102460001A800DD3B2F5B64F02D24C4901230B703E
:10247000930BC2F30D01454A52F82320030A53542B
:10248000454B1B88013B9AB2434BB2F5804F1A80F3
:102490000CD3B2F5B64F02D2404901230B70930B17
:1024A0003A49C2F30D0251F823309854364B1C8040
:1024B000FFF741BA029B029A9B7923F004039371C0
:1024C00079E7314B31481C88029B9D79631C9BB294
:1024D0009A0BA11C50F822002B4A1380C3F30D0263
:1024E00089B28B0B805C294A52F82320264B198035
:1024F000C1F30D032449D35C6A0600EB03239EB2AB
:1025000038D5254B224A1B881068013BE11C9AB242
:1025100000F1110388B220490A801D49B2F5804FAD
:102520000B600DD3B2F5B64F02D21C4901230B70DC
:10253000930BC2F30D01154A52F82320030A53549A
:10254000154B1B88013B9AB2134BB2F5804F1A8092
:102550000CD3B2F5B64F02D2104901230B70930B86
:102560000A49C2F30D0251F823309854064B1E80DD
:10257000FFF7E1B9064BE21C1B680A80044A0A33E4
:102580001360FFF7D8B900BFAABD012044A5012000
:10259000B0BD012000BD01204EBC0120A5000020DF
:1025A000874B1D781DB9874B1B78002B59D0864B64
:1025B00086481A88531C99B2931C9AB28B0B940BC1
:1025C00050F82300804B1980C1F30D037F49C0569A
:1025D0007D4B51F824101A80C2F30D03CB5C03F03D
:1025E000F80203F00706382A03F29385DFE812F0B9
:1025F0004E1D911D911D911D911D911D911D911DAE
:102600003C1D911D911D911D911D911D911D911DAF
:10261000391D911D911D911D911D911D911D911DA2
:10262000FA03911D911D911D911D911D911D911DEB
:10263000F803911D911D911D911D911D911D911DDD
:10264000F603911D911D911D911D911D911D911DCF
:10265000F403911D911D911D911D911D911D911DC1
:102660008800594B59481B8801339BB29A0BC3F31E
:102670000D0150F8222054480380535C03F0F80207
:1026800003F00701382A03F27A87DFE812F0721F9D
:10269000781F781F781F781F781F781F781F4D03C9
:1026A000781F781F781F781F781F781F781FEE0219
:1026B000781F781F781F781F781F781F781F3B01BD
:1026C000781F781F781F781F781F781F781FEE00FB
:1026D000781F781F781F781F781F781F781FAB012D
:1026E000781F781F781F781F781F781F781FA50024
:1026F000781F781F781F781F781F781F781F760043
:1027000006212F4B1B78002B50D0029B1A7A5B7A44
:102710002F4943EA022303440C682C4A99B28B0BDD
:10272000C1F30D0052F8232004F11703284C236055
:10273000125C029B9B79D00702984CBF43F00103C7
:1027400023F00103062E83714FEA52001DD0029B35
:102750009855029B9B7998B1029A23F0400393719C
:10276000029B02999A79184B02F06D021B888A71BC
:10277000154A01331380FFF7DEB80E460020C0E78C
:10278000029A43F040039371EAE7B1F5804FE0D33A
:10279000B1F5B64F02D20F4A012313708B0BC1F370
:1027A0000D020A4951F823309854D2E7054B1C78A2
:1027B000002C00F06F81029B9A7ADB7AA8E700BFB9
:1027C0004EBD0120ACBD0120AABD012044A50120C1
:1027D000B0BD0120A50000200E460020A64B1B78AE
:1027E000002B00F0AA81029B1A7A5B7AA34943EA84
:1027F000022303440C68A24A99B28B0BC1F30D006B
:1028000052F8232004F117039C4C2360125C029BB6
:1028100002989B7915064CBF43F0010323F0010396
:102820008371530043F00100062E84B200F07381DF
:10283000029B9855029B02989A79924902F0BF0335
:102840002406837154BF02F03F0363F07F038B7152
:10285000029B02999A798C4B22F012021B888A7192
:10286000894A01331380FFF766B80E460020824B79
:102870001B78002B00F0A280029B1A7A5B7A7F49BA
:1028800043EA022303440C687D4A99B28B0BC1F3DF
:102890000D0052F8232004F11703784C2360125CDA
:1028A000029B02989B7915064CBF43F0010323F06D
:1028B0000103062E83714FEA42006ED0029B9855A9
:1028C000029B029A9B79029910F0FE0F14BF23F02D
:1028D000400343F040039371029B029A9B790406E4
:1028E0004CBF63F07F0303F07F039371029B9A79DF
:1028F000654B22F012021B888A71634A01331380F0
:10290000FFF719B80E4600205B4B1B78002B00F038
:102910006981029B1A7A5B7A584943EA022303448D
:102920000C68574A99B28B0BC1F30D0052F8232063
:1029300004F11703514C2360125C029B9879C30782
:1029400046BF530843F080045408D707029A4CBF8F
:1029500040F0010320F00103062E937100F0308156
:10296000029B9C55029B9B79002C30D00299454AD2
:1029700003F0BF0326068B712DD563F07F0393719F
:10298000029B02999A79404B22F012021B888A71AD
:102990003D4A01331380FEF7CEBFB1F5804F8FD390
:1029A000B1F5B64F02D2394A012313708B0BC1F334
:1029B0000D02334951F82330985481E7344B1C7889
:1029C000002C00F01681029B9A7ADB7A57E7029A74
:1029D00043F040039371029B029A9B7903F07F03BB
:1029E0009371CDE70E460020234B1B78002B00F09F
:1029F0008B80029B1A7A5B7A204943EA02230344C4
:102A00000C681F4A99B28B0BC1F30D0052F82320BA
:102A100004F11703194C2360125C029B9B79D007C9
:102A200002984CBF43F0010323F0010317068371A2
:102A300046BF530843F080005008062E53D0029B37
:102A40009855029B9B7900282FD002990D4A03F0DC
:102A5000BF0306068B712CD563F07F039371029B35
:102A600002999A79084B22F012021B888A71064A51
:102A700001331380FEF75FBF4EBD0120B0BD0120C2
:102A800044A5012000BD0120AABD0120A500002011
:102A9000ACBD0120062913D09D4B029A1B689C48AF
:102AA000525C08332146036043E6029A43F0400338
:102AB0009371029B029A9B7903F07F039371CEE797
:102AC000029B93491A795B790C6843EA02218B0BCC
:102AD000904A52F8232004F10F038D4CC1F30D00EE
:102AE0002360125C25E6B1F5804FAAD3B1F5B64F4D
:102AF00002D2894A012313708B0BC1F30D02854961
:102B000051F8233098549CE7844B1C78E4B1029B25
:102B10009A7ADB7A70E7B1F5804FFFF48BAEB1F5AE
:102B2000B64F02D27C4A012313708B0BC1F30D0206
:102B3000784951F8233098547CE6784B1C7874B16E
:102B4000029B9A7ADB7A51E6062913D0704B029ADF
:102B50001B686F48525C0833214603605DE7062915
:102B60001BD06B4B029A1B686948525C08332146A4
:102B700003604CE6029B66491A795B790C6843EA6C
:102B800002218B0B634A52F8232004F10F03604C9F
:102B9000C1F30D002360125C3FE7029B5C491A7988
:102BA0005B790C6843EA02218B0B5A4A52F82320C6
:102BB00004F10F03564CC1F30D002360125C26E6AE
:102BC000B1F5804FFFF4CEAEB1F5B64F02D2524A06
:102BD000012313708B0BC1F30D024E4951F82330C2
:102BE0009C54BFE64D4B1C7874B1029B9A7ADB7AF9
:102BF00092E6062913D0464B029A1B684448525C61
:102C00000833214603604BE606291BD0404B029A4D
:102C10001B683F48525C0833214603608DE6029BE7
:102C20003B491A795B790C6843EA02218B0B394ADC
:102C300052F8232004F10F03354CC1F30D0023603B
:102C4000125C2DE6029B32491A795B790C6843EAE3
:102C500002218B0B2F4A52F8232004F10F032C4C36
:102C6000C1F30D002360125C67E60E4600202C4B7A
:102C70001B78002B03F09184029B1A7A5B7A24491B
:102C800043EA022303440D6899B2880B214B53F8A1
:102C9000202005F117031E4DC1F30D042B60125DBA
:102CA000029B9B7903F0010343EA4202062E95B290
:102CB00000F08380029B9A55029B029A9B79E9055A
:102CC0004CBF43F0010323F001039371029B029A6E
:102CD0009B79029915F0FF0F14BF23F0400343F0D6
:102CE00040039371029B9B792A06029A4CBF63F0C2
:102CF0007F0303F07F039371029B9A79094B22F0C3
:102D000012021B888A71074A01331380FEF713BE33
:102D1000B0BD012044A50120A5000020ACBD0120CC
:102D20004EBD0120AABD01200E4600209E4B1B78FF
:102D3000002B03F07084029B1A7A5B7A9B4943EA6A
:102D4000022303440C689A4A99B28B0BC1F30D001D
:102D500052F8232004F11703944C2360125C029B69
:102D6000D4079B7943F15084520842F08000029AC4
:102D700043F001039371062E03F05584029B98558E
:102D8000029B9B79002803F010840299894A03F082
:102D9000BF0300068B7143F10C8463F07F039371D2
:102DA000029B02999A79844B22F012021B888A7145
:102DB000814A01331380FEF7BEBDB1F5804FFFF4A9
:102DC0007BAFB1F5B64F02D27C4901230B70784B33
:102DD00053F820301A556FE70621FFE4062103E679
:102DE000062144E506218FE5734B714F1E886F4B1A
:102DF00070481D68029BDC79731C9BB29A0BC3F36D
:102E00000D0157F822206C4F3B80EB1D674D2B6066
:102E1000515C04F00F0201F00F03D31A13F0100FEE
:102E2000837914BF43F0100323F01003837181EA08
:102E30000403621A1F0695B23DD584EA02031C06FC
:102E400039D5029B029A9B7943F004039371029B4C
:102E5000029A9B79E8054CBF43F0010323F001037C
:102E60009371029B029A9B7915F0FF0F14BF23F018
:102E7000400343F040039371029B029A9B79290619
:102E80004CBF63F07F0303F07F039371029B4A49B9
:102E90009B79B21C0A80029A43F002039371FEF7F9
:102EA0004ABD454B44491B885A1C0A80444A0123A9
:102EB0001370FEF746BD029B029A9B7923F0040330
:102EC0009371C4E73C4B3A481C88029B9D79631C74
:102ED0009BB29A0BA11C50F82200374A1380C3F30F
:102EE0000D0289B28B0B805C314A52F82320324BA1
:102EF0001980C1F30D033049D35C00EB03239EB26C
:102F00002B0638D52F4B294A1B881068013BE11C42
:102F10009AB200F1110388B22A490A802349B2F516
:102F2000804F0B600DD3B2F5B64F02D22349012377
:102F30000B70930BC2F30D011D4A52F82320030AB4
:102F40005354204B1B88013B9AB21E4BB2F5804F65
:102F50001A800CD3B2F5B64F02D2184901230B7078
:102F6000930B1349C2F30D0251F823309854124BBE
:102F70001E80FEF7E0BC0D4BE21C1B680A800B4A6A
:102F80000A331360FEF7D7BC084B0B4A1B6807498E
:102F9000128804330B60084901320A800A4A01236F
:102FA0001370FEF7C8BC00BF4EBD0120B0BD0120AC
:102FB00044A5012000BD0120AABD0120A5000020DC
:102FC000ACBD01204EBC0120DCBC01209C4B1C8808
:102FD0009C4B1E68029B9D79631C9AB2A31C98B2FD
:102FE000910B994B53F82110954B1A8006F10A0367
:102FF000944EC2F30D023360895C934A830B52F8FE
:1030000023208F4B1880C0F30D03D35C8C4A01EB57
:10301000032329069BB258BFE31C1380FEF78BBC29
:103020008A4B1B78002B73D0864B1A68029B197A47
:103030005B7A0A3243EA012382490A60844A138098
:103040007F4B7F4A1B8801331380FEF774BC029BC1
:103050009B79180666D57E4B1C887A4B1D68631CCD
:1030600098B2820B05F10B03A10B774D55F8211097
:1030700055F82250734A1360C4F30D03C0F30D02D8
:10308000C95C734B1880AB5C41EA03236C490B802D
:103090006F4BA21C1A80FEF74EBC6D4B68491B8813
:1030A0000888684A013B99B2431C6948126801804C
:1030B00064480B32B1F5804F026098B20DD3B1F580
:1030C000B64F02D2634A012313708B0B5E4AC1F3E1
:1030D0000D0152F82320030A53545D4B1B88013B1A
:1030E0009AB25B4BB2F5804F1A800CD3B2F5B64F53
:1030F00002D2584901230B70930B5349C2F30D02BE
:1031000051F8233098544E4A30231380FEF713BCF5
:10311000514B1B7893B14B4B1A68029B0A32997A38
:10312000DB7A87E7474B47491A68454B05321B88CE
:103130000A60434A01331380FEF7FDBB414B1A6816
:10314000029B063219795B7974E7444A1370FEF7E3
:1031500084B90121424812F07FFA0A9B1B689868E3
:1031600010F09AFA0125FEF72DB9012325468DF8B6
:103170003D30FEF727B93B4810F0FAFEFDF7BCBE24
:10318000029B029A9B7923F001039371FDF7C8BF5C
:10319000029BD879062842D00D2825D00A9B1D68AD
:1031A000A9688B68013B002B8B6012DB0A68531CFB
:1031B0000B6010700A9B1B68986810F06DFAFDF7A1
:1031C000AFBFDDF82080FEF704BDDFF89C80FEF77E
:1031D00000BD8A69934201DB0A28E7D10A4601460D
:1031E000284611F07DFCE5E70A9B1D68A9688B68FD
:1031F000013B002B8B6019DB08680D23421C0A6021
:1032000003700A9B19688A689368013B002B9360DE
:1032100007DB10680A23411C11600370CAE709200C
:10322000BCE708460A2111F05BFCC3E78A699342B8
:10323000E2DA0A460146284611F052FCE1E700BFF7
:10324000AABD0120B0BD012044A501204EBD012032
:103250004EBC0120A5000020ACBD0120DCBC01203B
:103260001861010854BC012000C00010984B994D12
:103270001C88994B1968029BD879631C9BB29A0BE6
:10328000073155F82220924D2B80934DC3F30D0347
:103290002960D35C914A5840029BD87193790028E9
:1032A00002F0AC8203F0BF030506937142F1A982DC
:1032B00063F07F039371029B029D9979884B1A5C9E
:1032C000864801F0EC03AB71002A02F0928243F0D1
:1032D000040383717E4AA31C1380FEF72CBB7C4B36
:1032E0001C887D4B1E68029B9D79631C9AB2A31CAF
:1032F00098B2910B774B53F82110754B1A8006F159
:103300000A03754EC2F30D023360895C714A830B68
:1033100052F823206E4B1880C0F30D03D35C6C4A27
:1033200001EB032329069BB248BFE31C1380FEF781
:1033300002BB029B9B7918065CD46A4B1C88664BC7
:103340001D68631C98B2820B05F10B03A10B614D44
:1033500055F8211055F822505F4A1360C4F30D034D
:10336000C0F30D02C95C5F4B1880AB5C41EA0323DC
:1033700057490B805B4BA21C1A80FEF7DCBA594BF5
:1033800053491B880888544A013B99B2431C55484D
:103390001268018050480B32B1F5804F026098B23C
:1033A0000DD3B1F5B64F02D24F4A012313708B0BE8
:1033B000484AC1F30D0152F82320030A5354494BE4
:1033C0001B88013B9AB2474BB2F5804F1A800CD351
:1033D000B2F5B64F02D2444901230B70930B3D491D
:1033E000C2F30D0251F823309854394A2823138030
:1033F000FEF7A1BA384B38491A68354B05321B889D
:103400000A60334A01331380FEF795BA304B1C88AB
:10341000314B1E68029B9D79631C9AB2A31C98B223
:10342000910B2C4B53F82110294B1A8006F10A03FB
:10343000294EC2F30D023360895C264A830B6D0767
:1034400052F82320224B1880C0F30D03D35C204A8E
:1034500001EB03239BB258BFE31C1380FEF76BBA4A
:10346000224B1B78002B7ED01B4B029A1B68117AD3
:103470001948527A0833036042EA0123144A138040
:10348000FEF759BA029B9B795E077AD5154B1C88CB
:10349000114B1D68631C98B2820B05F10B03A10B45
:1034A0000C4D55F8211055F822500B4A1360C4F307
:1034B0000D03C0F30D02C95C0A4B1880AB5C41EAF6
:1034C000032303490B80074BA21C1A80FEF733BA73
:1034D000AABD012044A50120B0BD012000BD0120EE
:1034E000F45B01084EBC0120A50000204EBD012068
:1034F0006B4B6C491B8808886B4A013B99B2431C93
:1035000067481268018068480B32B1F5804F02604D
:1035100098B20DD3B1F5B64F02D2644A01231370AD
:103520008B0B634AC1F30D0152F82320030A535455
:103530005B4B1B88013B9AB2594BB2F5804F1A8006
:103540000CD3B2F5B64F02D2584901230B70930B3E
:103550005749C2F30D0251F823309854514A2023A1
:103560001380FEF7E8B9534B1B78B3B14E4B029A68
:103570001B68917A4C48D27A0833036042EA0123EF
:103580007CE7494B48491A68464B05321B880A605C
:10359000444A01331380FEF7CEB9434B029A1B68AD
:1035A0001179414852790433036042EA012365E707
:1035B0003C4B3F481C88029B9D79631C9BB29A0B35
:1035C000A11C50F82200374A1380C3F30D0289B2C0
:1035D000805C374A8B0B52F82320324B1980C1F3A1
:1035E0000D033049D35C00EB032368079EB238D546
:1035F0002B4B2D4A1B881068013BE11C9AB200F14D
:10360000110388B226490A802749B2F5804F0B6022
:103610000DD3B2F5B64F02D2244901230B70930BA0
:10362000C2F30D01224A52F82320030A53541C4BC3
:103630001B88013B9AB21A4BB2F5804F1A800CD30B
:10364000B2F5B64F02D2194901230B70930B1849FA
:10365000C2F30D0251F823309854124B1E80FEF72E
:103660006AB9114BE21C1B680A800F4A0A331360C7
:10367000FEF761B90C4B029C19680A4B1A88029B31
:103680005879DB7863710B1D0749E0700B60054BBF
:10369000217901321A80A3782371A170FEF74BB90A
:1036A0004EBC0120AABD0120B0BD0120A500002014
:1036B00044A50120ACBD0120814B82481F887B1CA2
:1036C0009BB29A0BC3F30D0150F822207C48038073
:1036D000525CA2F140037B2B01F2F387DFE813F089
:1036E000C80F990F3C0FD70E8C0E6A0E4C0E2F0E82
:1036F000060EE30D860D4D0D8C0E2B0D1E0D140DBB
:10370000BE0CAA0C4D0CFA0B8C0E6A0EDF0BD00B04
:10371000A60B810BB4076D078C0E6A0E6007560767
:103720001107FD06BB0668068C0E6A0E3106E7051A
:10373000BC05A8051805C8048C0E6A0EB0045C040C
:103740000A0AF8099D094E098C0E6A0E850AF10FC6
:103750005C0A6F081408430B8C0E6A0E360BF10FCF
:10376000F10FF10FF10FF10FF10FF10FF10FF10F59
:10377000F10FF10FF10FF10FF10FF10FF10FF10F49
:10378000F10FF10FF10FF10FF10FF10FF10FF10F39
:10379000F10FF10FF10FF10FF10FF10FF10FF10F29
:1037A000F6089108E50AAE0AF10FF10FF10FF10FDB
:1037B0000404AA031C03E502F10FF10FF10FF10F4E
:1037C000D101920158022A02F10FF10FF10FF10F0E
:1037D0003901FA009F007C00029B1A795B7943EA69
:1037E0000224A30B3749384D51F823300299C4F312
:1037F0000D0249789A5C029B18780AF0AFFB029B95
:103800001B78621E013B94B2029ADBB21370002B4C
:1038100030D02E4B2D4A1B6815331360E1E7029B15
:103820001A795B79012743EA0225B5F5804F4FEA03
:103830009533C5F30D060DD3B5F5B64F3CBF244AFD
:103840001770029A517810781E4A52F823400AF0F5
:10385000DBFAA055029B1C4C1B786A1E013B95B2FB
:10386000029ADBB21370C3B1184B184A1B681533A8
:103870001360DAE7154BAA791968114B6C711B8834
:10388000200A42F042022871AA7110480C4A1031F5
:10389000013301601380FEF74EB80C4BA279196812
:1038A000074B65711B88280A42F042022071A27101
:1038B0000648034A1031013301601380FEF73BB81C
:1038C000AABD012044A5012000BD0120B0BD0120FA
:1038D000A5000020029B029A9B79157854781079F4
:1038E0005179029ED27923F04003B37144EA052551
:1038F00041EA002197B202F00F068B0B9F48C1F3FB
:103900000D0250F823309A5C02F00F03F41ABB1A30
:103910009AB2029B681E9B7985B2E00602984CBF62
:1039200043F0100323F010038371029B94489B79AA
:103930000139140689B240F17C81029A63F07F0359
:103940009371904B002D3FD01B688E4A1533136046
:10395000D3E7029B02995C781D789A78DB78087926
:10396000497944EA052C43EA0222CCEB020341EAFE
:10397000002E9EB274464FF00108A30B7F49C4F39A
:103980000D0051F82310B2F5804F04F1FF33085CAD
:1039900002F1FF374FEA92359CB2C2F30D0109D311
:1039A000B2F5B64F3CBF784B83F80080734B53F8A9
:1039B00025305854BAB2964200F05881714B714983
:1039C0001B6815330B60D8E71A68029B59710B0A04
:1039D00002990B716B4B0D7010324D701A60029B87
:1039E000029A9B7923F004039371029B02999A79BE
:1039F000664B42F002021B888A71644A01331380CD
:103A0000FDF799BF029B029A9B791578547810793B
:103A10005179029ED27923F04003B37144EA05251F
:103A200041EA002197B202F00F068B0B5348C1F315
:103A30000D0250F823309A5C02F00F03F41ABB1AFF
:103A40009AB2029B681E9B7985B2E00602984CBF31
:103A500043F0100323F010038371029B48489B79C5
:103A60000131140689B240F19E81029A63F07F030E
:103A70009371444B002D3FD01B68424A15331360AD
:103A8000D3E7029B02995C781D789A78DB780879F5
:103A9000497944EA052C43EA02220CEB020341EA8D
:103AA000002E9EB274464FF00108A30B3349C4F3B5
:103AB0000D0051F82310B2F5804F04F10103085CAA
:103AC00002F101074FEA92359CB2C2F30D0109D30E
:103AD000B2F5B64F3CBF2C4B83F80080274B53F810
:103AE00025305854BAB2964200F07A81254B2549C8
:103AF0001B6815330B60D8E71A68029B59710B0AD3
:103B000002990B711F4B0D7010324D701A60029BA1
:103B1000029A9B7923F004039371029B02999A798C
:103B20001A4B42F002021B888A71184A0133138033
:103B3000FDF701BF029B1A795B7943EA0224A30BCC
:103B40000E490F4D51F823300299C4F30D02497804
:103B50009A5C029B18780AF001FA029B1B78621C9F
:103B6000013B94B2029ADBB21370002B3BD0054BA1
:103B7000044A1B6815331360E1E700BF44A5012028
:103B800000BD0120B0BD0120A5000020AABD01207C
:103B9000029B1A795B79012743EA0225B5F5804F2C
:103BA0004FEA9533C5F30D060DD3B5F5B64F3CBFBF
:103BB0009B4A1770029A517810789A4A52F823401B
:103BC0000AF022F9A055029B974C1B786A1C013B16
:103BD00095B2029ADBB21370C3B1944B934A1B683F
:103BE00015331360DAE7914BAA791968904B6C7121
:103BF0001B88200A42F042022871AA718B488C4A25
:103C00001031013301601380FDF795BE874BA27917
:103C10001968874B65711B88280A42F0420220719F
:103C2000A2718248824A1031013301601380FDF78E
:103C300082BE03F07F04029B9C71002A7FF481AE58
:103C40007A4B41711A6845700B0A0371774B02F188
:103C50001001196044F040022B0A82710370002D9C
:103C60003FF4BDAE44F044038371BEE66F4A029850
:103C70001468029A029D91796D4AC670CCEB0E03CE
:103C800012889BB2300A21F016016B71A8701B0AD2
:103C90006648A97166492B71103400230132046013
:103CA0000A802B706B70FDF746BE029B5F491A7944
:103CB0005B790C68029943EA0225AB0B594A4978B3
:103CC00052F8232004F11003584CC5F30D00236073
:103CD000029B125C1878544C0AF040F9029B029A3D
:103CE0001B78013BDBB21370002B53D1A37943F057
:103CF0004003A371029A029891794D4A6B1E9BB2C0
:103D0000128843711B0A0371494B41F002010132D1
:103D100081711A80FDF70FBE029A444B11795279D6
:103D20001B6842EA0125414A1033B5F5804F136004
:103D300011D3B5F5B64F02D2394A01231370029A56
:103D4000AB0B51781078374A52F823400AF05CF8F0
:103D5000C5F30D03E054029B334819786B1E9AB2E9
:103D60004B1ED9B2029B5A71130A029A1371117039
:103D70008379A1B943F040038371029B02999A7938
:103D80002B4B42F002021B888A71294A01331380AF
:103D9000FDF7D1BDA37923F04003A371AAE723F077
:103DA00040038371E9E703F07F04029B9C71002AC2
:103DB0007FF45FAE1D4B41711A6845700B0A0371A9
:103DC0001A4B02F11001196044F040022B0A827173
:103DD0000370002D3FF49BAE44F0440383719CE6D6
:103DE000124A02981468029A029D9179104AC6708C
:103DF0000CEB0E0312889BB2300A21F016016B7196
:103E0000A8701B0A0948A97109492B7110340023B5
:103E1000013204600A802B706B70FDF78CBD00BF0F
:103E2000A500002044A5012000BD0120B0BD012057
:103E3000AABD0120029BAE491A795B7908680299F4
:103E400043EA0225AB0BAB4ACC7952F823200E781B
:103E500000F11003A648C5F30D010360535C029AFC
:103E60005078E21A03F00F0104F00F0394B2A24A53
:103E70005B1A13F0100F937914BF43F0100323F073
:103E800010039371029B029A9B7940EA0621260651
:103E90004CBF63F07F0303F07F0393716B1E0298A6
:103EA0009BB24A1E91B21A0A0271934A43710B0ADD
:103EB000037041709379002940F03E8723F004039A
:103EC0009371029B9B79002C61D1029A43F04003CD
:103ED0009371029B89499B79BA1C0A80029A43F02C
:103EE00002039371FDF727BD029B81491A795B7923
:103EF0000F68029943EA0225AB0B7E4A8E7852F88E
:103F00002300029BC9781A7807F11003784F3B60B1
:103F1000029BC5F30D0441EA06215B78005DB1F513
:103F2000804F43EA02240CD3B1F5B64F02D2744A53
:103F3000012313708B0B6F4EC1F30D0256F8233023
:103F400098546A1E631E013994B2029A89B298B2DB
:103F5000D1700B0A02995070220A0A71664A8B705E
:103F6000030A0B704C719379002840F0EA8623F025
:103F700004039371029B02999A79604B22F012021A
:103F80001B888A715D4A01331380FDF7D4BC029A05
:103F900023F0400393719CE7029B02991A79C87938
:103FA0005B7953490F6843EA02218B0B514AC1F3F5
:103FB0000D0552F82340665D00F00F034C4843EABC
:103FC0000612B1F5804F07F11203D2B2036006D397
:103FD000B1F5B64F02D24A4901230B706255029BDC
:103FE000454ADB7923F00F0343EA161358B2029BCC
:103FF000C1B2D9719379002936D143F0400393714E
:10400000029B029A9B790028B4BF63F07F0303F000
:104010007F0393713B4B5B5CFBB1029B029A9B79E4
:1040200043F004039371029B02999A79334B22F077
:1040300012021B888A71314A01331380FDF77BBC61
:104040002B4B2E491A68BB1C0B80294908320A6089
:104050002D4A00231370FDF76EBC029B029A9B79D8
:1040600023F004039371DEE723F040039371C7E765
:10407000BB1C9AB2FB1C99B21E481E4D930B8C0BB5
:1040800050F823001D4B1A80C2F30D03194AC05C7F
:104090001A4B52F824401980C1F30D031B4AE35C0C
:1040A000127800EB032398B2002A00F08280104AB5
:1040B000411C1768820B8B13C1F30D0455F82210B5
:1040C0000B4A55F8236007F114031360C0F30D0386
:1040D000325DCB5C029903EB02239BB21A0A4B724E
:1040E0000A72064B054A1B8801331380FDF723BC77
:1040F000B0BD012044A5012000BD0120AABD0120C2
:10410000A5000020F45B010850BC01204EBD012039
:104110009F4B02991A68029B897918795B799C4DAB
:104120009C4C43EA0020060501F0010302F10F0256
:104130002A6003EB40054CBF41F0100321F010034F
:10414000A37180EA050313F4004F029B029A9B7946
:1041500014BF43F0040323F004039371029A2B0A63
:10416000137155718B4A9379EC034CBF43F00103F3
:1041700023F001039371ABB2002B38D0029B029A5B
:104180009B7923F040039371029B029A9B798249A9
:1041900028044CBF63F07F0303F07F039371029BFD
:1041A000BA1C9B790A80029A23F002039371FDF7EF
:1041B000C2BB7A4B1B78411C03B3754A1768820B4C
:1041C0008B13C1F30D0455F82210714A55F8236082
:1041D00007F114031360C0F30D03325DCB5C029949
:1041E00003EB02239BB21A0ACB728A7279E7029B15
:1041F000029A9B7943F040039371C5E7644A1768BC
:10420000820B8B13C1F30D0455F82210604A55F848
:10421000236007F110031360C0F30D03325DCB5C24
:10422000029903EB02239BB21A0A4B710A7158E7F9
:10423000574B029A1B6802990298554C527949785B
:1042400000780C33236009F089FE534B524A1B88D7
:1042500001331380FDF76FBB4D4B029A1B685178F9
:1042600010784B4A0C33136009F0CEFD029B494A8B
:1042700058719379002875D003F0BF03010693713C
:1042800073D563F07F039371029B029C9979444B31
:104290001A5C404801F0FD03A371002A5ED043F090
:1042A000040383713C4ABB1C1380FDF744BB029B93
:1042B00037481A795B790768029943EA0220830B31
:1042C000384AC97952F82340C0F30D0501F00F01B7
:1042D000665D320942EA01122D4907F11203B0F579
:1042E000804F0B6006D3B0F5B64F02D22E490123A2
:1042F0000B706255029B2749DB7906F00F0223F011
:104300000F031A43029BDA718B79002A3BD143F0E9
:1043100040038B71224B9B5C002B2DD0029B029A99
:104320009B7943F004039371029B02999A791A4B8B
:1043300022F012021B888A71174A01331380FDF79D
:10434000FABA134B14491A68BB1C0B801049083287
:104350000A60164A00231370FDF7EDBA21F0060338
:1043600083719FE743F040039371029B029A9B790C
:1043700003F07F03937187E7029B029A9B7923F0F6
:1043800004039371D0E723F040038B71C2E700BFB1
:10439000B0BD012000BD0120AABD0120ACBD01209F
:1043A000F45B010844A50120A500002050BC0120B9
:1043B000BB1C9E489AB2FB1C99B205689C48930BA3
:1043C00050F823409B4B1A8005F11403974D880B3E
:1043D0002B60974BC2F30D0253F82000954BA45C61
:1043E0001980029AC1F30D031179C25C029B5B79BB
:1043F00004EB022243EA012390B21CB2B0F5804FD5
:10440000A5B223D3B0F5B64F02D28B4A0123137065
:10441000830B874AC0F30D0152F8232045F6FE2393
:104420009842545402DC844A01231370431C9A13AB
:10443000C3F30D017E4B53F822202B0A53547D4BBE
:104440007C4A1B8801331380FDF775BA43F6FF736E
:104450009842F4D1E7E7029A744B92791B68734C47
:10446000764942F300000F33C50423604CBF42F08D
:10447000100322F010038B71029B029A9B7923F0A8
:10448000040393716D4B6D4A0293C4034FEA1023EA
:104490005071137165D5937943F00103937183B221
:1044A000002B57D0029B029A9B7923F04003937113
:1044B000029B029A9B795F4900044CBF63F07F0323
:1044C00003F07F039371029BBA1C9B790A80029AC6
:1044D00043F002039371FDF72EBA544B029A1B6806
:1044E00002990298514C1279497800780C33236074
:1044F00009F034FD4F4B4F4A1B8801331380FDF701
:104500001ABA4A4B029A1B6851781078474A0C3302
:10451000136009F079FC029B484A1871937958B3EB
:1045200003F0BF030606937129D563F07F039371EF
:10453000029B029C9979424B1A5C404801F0FD03B2
:10454000A371AAB143F0040383713A4ABB1C1380E0
:10455000FDF7F1B9029B029A9B7943F040039371F6
:10456000A6E7029B029A9B7923F00103937196E7D9
:1045700021F006038371E8E743F040039371029B47
:10458000029A9B7903F07F039371D1E7274B294966
:104590001B68BA1C0A80254A09331360FDF7CBB9A2
:1045A000224B24491A68BB1C0B80204908320A6040
:1045B000244A02231370FDF7BEB9BB1C1B489AB2F4
:1045C00004681B48930BF91C50F82300194B1A8000
:1045D00004F11403154CC2F30D02236089B2805C10
:1045E000134A134C8B0B3E1D52F82320114B19809C
:1045F000C1F30D03D35C00EB032399B2481C8B0B72
:10460000821354F8225054F82340C0F30D02C1F332
:104610000D03AA5CE35C074903EB02239BB20E8007
:1046200002991A0ACB708A70FDF785B9B0BD0120D6
:1046300044A50120AABD0120A500002000BD012045
:10464000F45B010850BC0120029B9B4D1C795979F9
:104650009A780298DB782D688079039543EA0226E0
:1046600041EA0425C5F30B02C6F30B03134400F023
:1046700001015C18AA19039B11448F4A0F33136080
:10468000E3048E4A4CBF40F0100320F010039371F6
:1046900085EA0603DB0B40F0CA8285EA01031C04AD
:1046A00040F1C582029B029A9B7943F00403937107
:1046B000029A0B0A13715171804A9379C8034CBF57
:1046C00043F0010323F0010393718BB2002B00F040
:1046D000A782029B029A9B7923F040039371029B6D
:1046E0009B790A04029A76494CBF63F07F0303F07A
:1046F0007F039371029BBA1C9B790A80029A23F074
:1047000002039371FDF717B96E49029B0E88029957
:104710001A79887968495B790968039143EA022527
:1047200000F00101C6F30B030B44C5F30B029C1808
:10473000AA19039B1144604A0F331360E3045F4AD4
:104740004CBF40F0100320F01003937185EA06037C
:10475000DB0B4FD185EA01031C044BD5029B029A67
:104760009B7943F004039371029A0B0A1371517100
:10477000524A9379C8034CBF43F0010323F001036D
:1047800093718BB2002B2ED0029B029A9B7923F05F
:1047900040039371029B029A9B7909044CBF63F01A
:1047A0007F0303F07F039371029B45499B79BA1CF9
:1047B0000A80029A23F002039371FDF7BCB83E4BC6
:1047C000029A1B68029902983B4CD279497800788A
:1047D0000C33236009F0C2FB394B394A1B88013383
:1047E0001380FDF7A8B8029B029A9B7943F040031F
:1047F0009371CFE7029B029A9B7923F00403937194
:10480000B2E7029B2C491A795B790868029943EA5E
:104810000225AB0B2C4ACC7952F823200E7800F1FC
:1048200010032548C5F30D010360535C029A5078CC
:10483000E21A03F00F0104F00F0394B21F4A5B1A4F
:1048400013F0100F937914BF43F0100323F01003FB
:104850009371029B9B792206029A4CBF63F07F03FF
:1048600003F07F0340EA062193716B1C02989BB210
:104870004A1E91B21A0A0271104A43710B0A037060
:1048800041709379002940F0A48223F004039371CE
:10489000029B9B79002C6CD1029A43F040039371E8
:1048A000029B07499B79BA1C0A80029A43F00203D3
:1048B0009371FDF740B800BFB0BD012000BD0120DD
:1048C000AABD01204EBC012044A50120029BAB499A
:1048D0001A795B790F68029943EA0225AB0BA84A63
:1048E0008E7852F82300029BC9781A7807F11003DA
:1048F000A24F3B60029BC5F30D0441EA06215B78A1
:10490000005DB1F5804F43EA02240CD3B1F5B64FF8
:1049100002D29C4A012313708B0B994EC1F30D02F6
:1049200056F8233098546A1C631E013194B2029ADF
:1049300089B298B2D1700B0A02995070220A0A719A
:10494000914A8B70030A0B704C719379002840F0E8
:10495000448223F004039371029B02999A798B4B52
:1049600022F012021B888A71884A01331380FCF7F7
:10497000E2BF029A23F04003937191E7BB1C9AB205
:10498000FB1C99B27E48930B8C0B50F823007F4B95
:104990001A80C2F30D037A4A52F82440C25C7B4B62
:1049A0001980C1F30D037549E35C086802EB03232A
:1049B00099B2724A00F11403B1F5804F136027D306
:1049C000B1F5B64F02D26F4A012313706C488B0BBE
:1049D000C1F30D0250F823306D480088985445F615
:1049E000FE23994202DC674A012313704A1C68497E
:1049F000931308886249C2F30D0251F82310030A89
:104A00008B54624B614A1B8801331380FCF793BFC0
:104A100043F6FF739942F4D1E5E75D49029B0E88A6
:104A200002991A795B798879544943EA0225096821
:104A30000391C5F30B02C6F30B03D31A00F0010177
:104A40005C1AAA1B039B511A4C4A0F331360E304F0
:104A50004D4A4CBF40F0100320F01003937186EADA
:104A600005031E0475D585EA01031D0471D5029B5B
:104A7000029A9B7943F004039371029A0B0A137113
:104A80005171414A9379CC034CBF43F0010323F0A9
:104A9000010393718BB2002B54D0029B029A9B7935
:104AA00023F040039371029B029A9B7908044CBF48
:104AB00063F07F0303F07F039371029B33499B797B
:104AC000BA1C0A80029A43F002039371FCF733BFC9
:104AD0002A4B029A1B68294C517810780C3300221B
:104AE000236009F03BFA294B284A1B8801331380C5
:104AF000FCF721BF214B029A1B68517810781F4A9E
:104B0000214C0C33136009F07FF9A379024658B3A6
:104B100003F0BF030106A37129D563F07F03A371DE
:104B2000029B029C99791B4B17489A5C01F0FD038C
:104B3000A371AAB143F004038371144ABB1C138010
:104B4000FCF7F9BE029B029A9B7943F040039371F4
:104B5000A9E7029B029A9B7923F0040393718CE7E7
:104B600021F006038371E8E743F04003A371029B41
:104B700002999B7903F07F038B71D1E7B0BD0120CF
:104B800044A50120A500002000BD0120AABD0120F0
:104B90004EBC0120F45B01089C4B029A1B685178C3
:104BA00010789A4A0C33136009F02EF9029B984A48
:104BB000D871937950B303F0BF030106937128D5E0
:104BC00063F07F039371029B029C9979914B1A5C6D
:104BD0008F4801F0FD03A371A2B143F00403837178
:104BE0008D4ABB1C1380FCF7A6BE884B8A491A6805
:104BF000BB1C0B80854908320A60884A0123137068
:104C0000FCF799BE21F006038371E9E743F0400306
:104C10009371029B029A9B7903F07F039371D2E711
:104C2000029B029A9B7943F04003937157E5029BE4
:104C3000029A9B7923F00403937139E5029B73492F
:104C40001A795B790C68029943EA0225AB0B744A26
:104C5000497852F8232004F110036C4CC5F30D0081
:104C60002360029B125C1878694C09F077F9029B6B
:104C7000029A1B78013BDBB21370002B53D1A3794E
:104C800043F04003A371029A02989179624A6B1C27
:104C90009BB2128843711B0A03715F4B41F0020102
:104CA000013281711A80FCF746BE029A574B117986
:104CB00052791B6842EA0125544A1033B5F5804FFA
:104CC000136011D3B5F5B64F02D2564A01231370C3
:104CD000029AAB0B51781078514A52F8234009F0F0
:104CE00093F8C5F30D03E054029B494819786B1CF7
:104CF0009AB24B1ED9B2029B5A71130A029A1371CF
:104D000011708379A1B943F040038371029B02992A
:104D10009A79414B42F002021B888A713E4A013364
:104D20001380FCF708BEA37923F04003A371AAE720
:104D300023F040038371E9E743F004039371FFF725
:104D4000C0B843F004039371FFF714B92F4B3249F5
:104D50001A68BB1C0B802D4908320A602F4A0223B7
:104D60001370FCF7E8BDBB1C28489AB204682C48B5
:104D7000930BF91C50F82300274B1A8004F11403FD
:104D8000224CC2F30D02236089B2805C244A244C79
:104D90008B0B3E1D52F823201F4B1980C1F30D03CE
:104DA000D35C00EB032399B2481C8B0B821354F89D
:104DB000225054F82340C0F30D02C1F30D03AA5C46
:104DC000E35C154903EB0223174A0E801380FCF7BE
:104DD000B2BD43F0040393715AE543F004039371A9
:104DE000BAE50A4B029A1B6802990298074CD278DE
:104DF000497800780C33236009F0B0F8064B064A76
:104E00001B8801331380FCF796BD00BFB0BD0120A5
:104E100000BD0120F45B0108AABD012050BC0120A7
:104E200044A50120A50000204EBC0120A74B029AFA
:104E30001B6851781078A54A0C33136008F0E4FF22
:104E4000029BA34AD8709379002839D003F0BF039E
:104E50000106937137D563F07F039371029B029C27
:104E600099799C4B1A5C9A4801F0FD03A3711AB31F
:104E700043F004038371984ABB1C1380FCF75BBDAD
:104E8000924B029A1968954B1B78D37101F1090373
:104E90009149BA1C0A808D4A1360FCF74CBD8B4BBC
:104EA0008D491A68BB1C0B80884908320A608C4AFD
:104EB00001231370FCF73FBD21F006038371DAE78D
:104EC00043F040039371029B029A9B7903F07F03A6
:104ED0009371C3E7BB1C7D489AB2FB1C99B205686D
:104EE0008048930B50F823407B4B1A8005F1140344
:104EF000764D880B2B607B4BC2F30D0253F82000DC
:104F0000754BA45C1980029AC1F30D039178C25CC1
:104F1000029BDB7804EB022243EA012390B21CB22D
:104F2000B0F5804FA5B223D3B0F5B64F02D26E4A8A
:104F300001231370830B6B4AC0F30D0152F8232039
:104F400045F6FE239842545402DC674A012313704D
:104F5000431C9A13C3F30D01624B53F822202B0A12
:104F600053545D4B5C4A1B8801331380FCF7E3BC50
:104F700043F6FF739842F4D1E7E7029B534D1C7947
:104F800059799A780298DB782D688079039543EAFD
:104F9000022641EA0425C5F30B02C6F30B03D31A1C
:104FA00000F001015C1AAA1B039B511A474A0F33F8
:104FB0001360E304464A4CBF40F0100320F0100396
:104FC000937186EA05031E0479D585EA01031D0461
:104FD00075D5029B029A9B7943F004039371029A60
:104FE0000B0A137151713A4A9379CC034CBF43F0C9
:104FF000010323F0010393718BB2002B58D0029B65
:10500000029A9B7923F040039371029B029A9B7949
:1050100008044CBF63F07F0303F07F039371029B8E
:105020002D499B79BA1C0A80029A43F002039371BE
:10503000FCF781BC254B029A1B6802990298234C0D
:105040009278497800780C33236008F087FF224B70
:10505000214A1B8801331380FCF76DBC1B4B029A5D
:105060001B6851781078194A0C33136008F0CCFE95
:10507000029B174A9870937900283BD003F0BF0336
:105080000106937139D563F07F039371029B029CF3
:105090009979104B1A5C0E4801F0FD03A3712AB3F5
:1050A00043F0040383710C4ABB1C1380FCF743BC20
:1050B000029B029A9B7943F040039371A5E7029B00
:1050C000029A9B7923F00403937188E7B0BD012015
:1050D00000BD0120F45B0108AABD012019070020D2
:1050E00050BC012044A50120A500002021F00603AA
:1050F0008371D8E743F040039371029B029A9B7936
:1051000003F07F039371C1E7A24BA3491B68BA1C4C
:105110000A80A04A09331360FCF70DBC9D4B9E49E1
:105120001A68BB1C0B809B4908320A609B4A00230B
:105130001370FCF700BC9A4B1C88964B1D68631CCF
:1051400098B2820B05F10E03A10B964D55F8211074
:1051500055F822508F4A1360C4F30D03C0F30D02BB
:10516000C95C8F4B1880AB5C41EA03238A490B80F2
:105170008B4BA21C1A80FCF7DEBBBB1C85489AB285
:1051800004688848930BF91C50F82300824B1A805E
:1051900004F114037F4CC2F30D02236089B2805CDA
:1051A000804A804C8B0B3E1D52F823207A4B19808D
:1051B000C1F30D03D35C00EB032399B2481C8B0BA6
:1051C000821354F8225054F82340C0F30D02C1F367
:1051D0000D03AA5CE35C704903EB02230E809BB2D3
:1051E00002991A0A4B700A70FCF7A5BB029B694D25
:1051F0001C7959791A7802985B782D688079039523
:1052000043EA022641EA0425C5F30B02C6F30B0369
:10521000134400F001015C18AA19039B11445D4A74
:105220000F331360E304604A4CBF40F0100320F0DA
:105230001003937185EA0603DB0B50D185EA010365
:105240001D044CD5029B029A9B7943F00403937191
:10525000029A0B0A13715171534A9379CC034CBFD4
:1052600043F0010323F0010393718BB2002B2FD085
:10527000029B029A9B7923F040039371029B029A4E
:105280009B7908044CBF63F07F0303F07F039371A5
:10529000029B41499B79BA1C0A80029A23F00203BF
:1052A0009371FCF748BB3B4B02991A68029B087844
:1052B0005B7802F10C0419461A46364B1C6008F064
:1052C0004DFE354B344A1B8801331380FCF733BB4A
:1052D000029B029A9B7943F040039371CEE7029BB5
:1052E000029A9B7923F004039371B1E7294B029A48
:1052F0001B6851781078274A0C33136008F084FD3E
:10530000029B294A5870937960B303F0BF030106EA
:1053100093712AD563F07F039371029B029C997964
:10532000224B1A5C204801F0FD03A371B2B143F097
:1053300004038371184ABB1C1380FCF7FCBA154B9D
:105340001B4A1968029BDB79137001F109031249AA
:10535000BA1C0A800F4A1360FCF7EDBA21F006036D
:105360008371E7E743F040039371029B029A9B79B4
:1053700003F07F039371D0E7064B07491A68BB1C03
:105380000B80044908320A60044A00231370FCF7BA
:10539000D2BA00BFB0BD0120AABD012050BC01207F
:1053A0004EBC012044A5012000BD0120F45B010892
:1053B00019070020A84B1C88A84B1D68631C98B2D5
:1053C000820B05F10E03A10BA54D55F8211055F8E0
:1053D0002250A24A1360C4F30D03C0F30D02C95C4E
:1053E0009D4B1880AB5C41EA03239E490B809A4B8E
:1053F000A21C1A80FCF79FBA029A984BD1791B68BD
:105400009648994A08338029036000F098804B42FF
:1054100098B20B0700F09980937943F010039371D1
:10542000029B0E069B7940F18580050640F1828043
:10543000029A43F0040393718B4A029B8949D87105
:105440009379C4054CBF43F0010323F0010393712A
:10545000029B029A9B7910F0FF0F14BF23F04003C8
:1054600043F040039371029B029A9B7900064CBF64
:1054700063F07F0303F07F039371029BBA1C9B7957
:105480000A80029A43F002039371FCF754BABB1CE2
:1054900072489AB2FB1C99B205687148930B50F898
:1054A0002340704B1A8005F114036C4D880B2B6060
:1054B0006B4BC2F30D0253F820006A4BA45C1980B9
:1054C000029AC1F30D031178C25C029B5B7804EB76
:1054D000022243EA012390B21CB2B0F5804FA5B27C
:1054E00023D3B0F5B64F02D2604A01231370830B69
:1054F0005B4AC0F30D0152F8232045F6FE23984283
:10550000545402DC594A01231370431C9A13C3F309
:105510000D01534B53F822202B0A5354514B514A3F
:105520001B8801331380FCF706BA43F6FF739842D9
:10553000F4D1E7E7029A23F0040393717CE79379AF
:1055400043F0040393714FF68070029B029A9B799B
:1055500023F01003937163E7029B404D1C79597946
:105560001A7802985B782D688079039543EA0226C1
:1055700041EA0425C5F30B02C6F30B03D31A00F06E
:1055800001015C1AAA1B039B511A344A0F331360A2
:10559000E304354A4CBF40F0100320F01003937130
:1055A00086EA05031E0450D585EA01031C044CD588
:1055B000029B029A9B7943F004039371029A0B0AAF
:1055C00013715171284A9379C8034CBF43F001030A
:1055D00023F0010393718BB2002B2FD0029B029A10
:1055E0009B7923F040039371029B9B790A04029AF2
:1055F0001C494CBF63F07F0303F07F039371029B50
:10560000BA1C9B790A80029A43F002039371FCF75B
:1056100092B9124B02991A68029B49781B7802F1E1
:105620000C0418461A460D4B1C6008F097FC0D4BF5
:105630000C4A1B8801331380FCF77DB9029B029A48
:105640009B7943F040039371CEE7029B029A9B79CA
:1056500023F004039371B1E74EBC0120B0BD0120DB
:1056600044A50120AABD012000BD0120A500002005
:10567000A24B029A1B6810785178A04A0C33136031
:1056800008F0C2FB029B9E4A1870937940B303F066
:10569000BF030106937126D563F07F039371029BCC
:1056A000029C9979974B1A5C954801F0FD03A37110
:1056B00092B143F004038371934ABB1C1380FCF73F
:1056C0003AB9114691480FF0C7FF0A9B1B689868CA
:1056D0000DF0E2FFFCF72FB921F006038371EBE731
:1056E00043F040039371029B029A9B7903F07F037E
:1056F0009371D4E7029B8148D9799A79844B0068E9
:105700001B8842EA0122013B814914B29AB20A8005
:105710007A4900F10B03B2F5804FA0B20B600DD3B4
:10572000B2F5B64F02D27B4901230B70930BC2F343
:105730000D01794A52F82320030A5354744B1B88F5
:10574000013B9AB2724BB2F5804F1A800CD3B2F57E
:10575000B64F02D26F4901230B70930B6E49C2F30F
:105760000D0251F823309C54674B674A1B88013364
:105770001380FCF7E0B821F0070343F01003A37196
:10578000FCF70DBB43F040039371029B029A9B7997
:1057900003F07F039371FCF7F1BA5D4B1D88574B03
:1057A0001C68594B1F886B1C98B2A90B04F10A03A3
:1057B000594C820B54F82140574951F822604F4A06
:1057C0001360C5F30D03C0F30D01E25C504B029C66
:1057D0001880735C42EA03231BB2C3F30720A37152
:1057E0004B4BE071A91C1980474B7A1C1A80FCF7BF
:1057F000A2B821F017038371FDF76CBD43F040039D
:105800009371029B029A9B7903F07F039371FDF7DA
:1058100052BD3D4B404EB3F800E0384B384F18684E
:10582000029B9C79DD790EF101039BB29A0BC3F3C5
:105830000D0156F82220344E3380C31D2F480360DB
:10584000505C05F00F0200F00F03D11A04F00103C1
:105850002A1AC91AD31ACA069EB24CBF44F01003C2
:1058600024F01003BB7180EA05031B063FD585EACF
:1058700006031F063BD5029B029A9B7943F0040363
:1058800093711F4A029B2049DE719379F5054CBF45
:1058900043F0010323F001039371029B029A9B7969
:1058A00016F0FF0F14BF23F0400343F04003937141
:1058B000029B029A9B7934064CBF63F07F0303F08E
:1058C0007F039371029B0EF102029B790A80029A78
:1058D00043F002039371FCF72EB80B4B0A491B8867
:1058E0005A1C0A800D4A01231370FCF72AB8029B48
:1058F000029A9B7923F004039371C2E7B0BD0120A3
:1059000000BD0120F45B0108AABD0120F46101087B
:105910004EBC0120A500002044A501204EBD012061
:10592000A14BA2481C88029B9D79631C9BB29A0BD9
:10593000A11C50F822009C4A1380C3F30D0289B2C7
:10594000805C9A4A8B0B52F82320974B1980C1F345
:105950000D039549D35C00EB0323E8079EB238D5CD
:10596000934B944A1B881068013BE11C9AB200F1EA
:10597000110388B28E490A808E49B2F5804F0B60C0
:105980000DD3B2F5B64F02D28B4901230B70930BA6
:10599000C2F30D01854A52F82320030A5354844B65
:1059A0001B88013B9AB2824BB2F5804F1A800CD310
:1059B000B2F5B64F02D2804901230B70930B7B499D
:1059C000C2F30D0251F823309854774B1E80FBF739
:1059D000B2BF784BE21C1B680A80764A0A33136018
:1059E000FBF7A9BF704B714D1C88724B1968029B65
:1059F000D879631C9BB29A0B0B3155F822206A4D63
:105A00002B806C4DC3F30D032960D15C08F0FCF9C9
:105A1000029AD071644AA31C1380FBF78CBF624BBF
:105A20001C88644B1E68029B9D79631C9AB2A31C60
:105A300098B2910B5D4B53F821105B4B1A8006F125
:105A40000A035C4EC2F30D023360895C574A830B34
:105A5000ED0752F82320544B1880C0F30D03D35C9C
:105A6000514A01EB03239BB258BFE31C1380FBF7A1
:105A700062BF504B029C19684B4B1A88029B1878E6
:105A80004E4B1B7823700B1D4A490B6046496378C7
:105A900001320A80494A107048485178437083782F
:105AA0004648A2788270C27844486170E178C1703B
:105AB00001794248A370237921714049E270037152
:105AC0006279437963714A71FBF735BF029B9B7919
:105AD000DE075CD5364B1C88364B1D68631C98B2BC
:105AE000820B05F10B03A10B304D55F8211055F831
:105AF0002250304A1360C4F30D03C0F30D02C95C99
:105B00002B4B1880AB5C41EA032327490B80284BC1
:105B1000A21C1A80FBF70FBF254B23491B8808885E
:105B2000244A013B99B2431C214812680180214854
:105B30000B32B1F5804F026098B20DD3B1F5B64F7C
:105B400002D21D4A012313708B0B184AC1F30D01B9
:105B500052F82320030A5354154B1B88013B9AB279
:105B6000134BB2F5804F1A800CD3B2F5B64F02D268
:105B7000114901230B70930B0C49C2F30D0251F82C
:105B800023309854084A10231380FBF7D4BE094BE6
:105B900008491A68044B05321B880A60024A01331F
:105BA0001380FBF7C8BE00BFAABD012044A5012099
:105BB0004EBC0120B0BD0120A5000020E0BC0120AA
:105BC0008C4B1C888C4B1E68029B9D79631C9AB27F
:105BD000A31C98B2910B894B53F82110854B1A8066
:105BE00006F10A03844EC2F30D023360895C834AD6
:105BF000830B52F823207F4B1880C0F30D03D35C36
:105C00007C4A01EB032369079BB248BFE31C138066
:105C1000FBF791BE7A4B1B78002B00F08E80794BFE
:105C20001C88754B1D68631C98B2A10B05F10E030F
:105C3000724D820B55F82150704951F822606E4A1E
:105C40001360C4F30D03C0F30D01EA5C6D4B1880C3
:105C5000735C029842EA03231BB2C3F30721437229
:105C6000684B0172A21C1A80624B624A1B88013386
:105C70001380FBF760BE029B9B79580700F1878079
:105C8000604B1C885C4B1D68631C98B2820B05F14D
:105C90000B03A10B594D55F8211055F82250564AC7
:105CA0001360C4F30D03C0F30D02C95C554B18809B
:105CB000AB5C41EA03234F490B80524BA21C1A8074
:105CC000FBF739BE4F4B4B491B8808884A4A013BBA
:105CD00099B2431C4B481268018047480B32B1F51A
:105CE000804F026098B20DD3B1F5B64F02D2464A4A
:105CF000012313708B0B414AC1F30D0152F823208D
:105D0000030A53543F4B1B88013B9AB23D4BB2F5FB
:105D1000804F1A800CD3B2F5B64F02D23A49012314
:105D20000B70930B3549C2F30D0251F82330985490
:105D3000304A18231380FBF7FEBD344B1B78002B31
:105D400031D0304B1C882C4B1D68631C98B2A10BC2
:105D500005F10E03294D820B55F82150274951F8C2
:105D60002260254A1360C4F30D03C0F30D01EA5C01
:105D7000244B1880735C029842EA03231BB2C3F3DE
:105D80000721C3721F4B8172A21C1A806CE71A4B49
:105D900019491A68174B05321B880A60154A0133E6
:105DA0001380FBF7C8BD174B1C88134B1D68631C81
:105DB00098B2A10B05F10A03104D820B55F8215042
:105DC0000E4951F822600C4A1360C4F30D03C0F36E
:105DD0000D01EA5C0B4B1880735C029842EA0323C6
:105DE0001BB2C3F307214371064B0171A21C1A8039
:105DF0003AE700BFAABD0120B0BD012044A50120A3
:105E00004EBD01204EBC0120A5000020ACBD0120EC
:105E1000974B98481C88029B9D79631C9BB29A0BF8
:105E2000A11C50F82200924A1380C3F30D0289B2DC
:105E30008B0B805C8F4A52F823208D4B1980C1F365
:105E40000D038B49D35C00EB03239EB26B0738D460
:105E5000894B8A4A1B881068013BE11C9AB200F109
:105E6000110388B284490A808449B2F5804F0B60DF
:105E70000DD3B2F5B64F02D2814901230B70930BBB
:105E8000C2F30D017B4A52F82320030A53547A4B84
:105E90001B88013B9AB2784BB2F5804F1A800CD325
:105EA000B2F5B64F02D2764901230B70930B7149BC
:105EB000C2F30D0251F8233098546D4B1E80FBF74E
:105EC0003ABD6E4BE21C1B680A806C4A0A331360B1
:105ED000FBF731BD6B4B93F80080B8F1000F43D056
:105EE000664B029A1B68557A92F808E0634A1733AA
:105EF0001360614B5F481A88531C9F13C3F30D0C4A
:105F00005C4B910B53F8273050F8210013F80C60CC
:105F1000C2F30D03B2F5804F0393C45C07D3B2F50F
:105F2000B64F02D2564901230B70039BC55443F66A
:105F3000FE739A420BDD45F6FE239A4202DC504A7C
:105F4000012313704B4B53F8273003F80CE0B8F1E2
:105F5000000F16D0029B5C721E72454B444A1B8890
:105F600001331380FBF7E7BC474B1B7883B1434BEE
:105F7000029A1B68D57A92F80AE0404A17331360F8
:105F8000B7E7414B1B786BB1029BDC729E72E4E772
:105F90003A4B029A1B68557992F804E0374A13335A
:105FA0001360A6E7029B5C711E71D6E7354B1B7828
:105FB000002B3DD0314B029A1B68117A2F48527A40
:105FC0000F33036042EA01202B4B1B88013B9AB23E
:105FD000294BB2F5804F1A800DD3B2F5B64F02D2DD
:105FE000274901230B70930BC2F30D01214A52F88C
:105FF0002320030A5354204B1B88013B9AB21E4BAB
:10600000B2F5804F1A800CD3B2F5B64F02D21C49BC
:1060100001230B70930B1749C2F30D0251F8233083
:106020009854134B124A1B8801331380FBF783BC2F
:10603000154B1B7853B1114B029A1B68917A0F488C
:10604000D27A0F33036042EA0120BDE70B4B029A7C
:106050001B681179094852790B33036042EA012029
:10606000B2E70621FCF703BE0621FCF75FBE00BFC6
:10607000AABD012044A501204EBC0120B0BD0120D5
:10608000A50000204EBD0120ACBD0120002D00F078
:106090009A81029B1A7A5B7AA34943EA022303445A
:1060A00098B20C68A14A830BC0F30D0152F823206B
:1060B00004F117039C4C2360525C029B170600F10D
:1060C00078819B79520002F0FE01029A23F00103CD
:1060D0009371062E00F05B81029B9955029B9B7980
:1060E000002957D00298924A03F0BF030D0683712E
:1060F00054D563F07F039371029B02999A798D4B7B
:1061000022F012021B888A718A4A01331380FBF73E
:1061100012BC062103F0C002802AC3F3C2076CD070
:10612000C02A42D0402A7BF406AC834B1B78002B5C
:1061300000F08B80029B1A7A5B7A7B4943EA022348
:1061400003449BB20C6878489A0BC3F30D01774B5C
:1061500053F8222004F114030360525C42FA07F35F
:1061600013F0010F029B029A9B7914BF23F04403A2
:1061700043F044039371029B6E4A9B79118823F08C
:10618000020343F010024B1C02998A71694A138082
:10619000FBF7D1BB029A43F040039371029B029A32
:1061A0009B7903F07F039371A6E7634B1B78002B69
:1061B0006CD0029B1A7A5B7A5B4943EA0223034460
:1061C0000D6899B2880B594B53F8202005F117033D
:1061D000554DC1F30D042B60125D012505FA07F33F
:1061E0001343062E1AB244D0029B9A55514B514A82
:1061F0001B8801331380FBF79EBB4F4B1B78002B92
:106200004BD0029B1A7A5B7A474943EA0223034444
:106210000D6899B2880B454B53F8202005F1170300
:10622000414DC1F30D042B60125D012505FA07F302
:10623000062E22EA03020FD0029B9A553D4B3D4A9F
:106240001B8801331380FBF776BB3C4B1B785BB399
:10625000029B9A7ADB7A70E7B1F5804FEED3B1F505
:10626000B64F3CBF364B1D70304B53F820301A559B
:10627000E4E7B1F5804FB9D3B1F5B64F3CBF304B31
:106280001D702A4B53F820301A55AFE72B4B1B7863
:10629000A3B1029B9A7ADB7A8EE7284B1B78F3B185
:1062A000029B9A7ADB7AAFE706292AD01E4B029A24
:1062B0001B68525C1C4908330B604FE70629029BA0
:1062C00040D05A5C184B19680123BB401A4301F1B6
:1062D00008031549062E12B20B6085D186E7062900
:1062E00042D0114B1868029B595C012303FA07F254
:1062F00021EA02020C4900F10803062E0B609BD133
:106300009CE7029B08491A795B79086843EA0223F3
:106310009A0BC3F30D01054B53F8222000F10C0337
:1063200001480360525C19E7B0BD012044A501207B
:1063300000BD0120AABD01204EBD0120ACBD012041
:10634000A50000201A799F495B790D6843EA022174
:10635000880B9D4B53F8202005F10F03994DC1F395
:106360000D042B60125D38E7029B96491A795B7920
:106370000D6843EA0221880B934B53F8202005F166
:106380000F03904DC1F30D042B60125D4DE7B0F586
:10639000804FFFF4A3AEB0F5B64F02D28B4A012373
:1063A0001370830BC0F30D02874850F823309954C3
:1063B00094E69979530043F0010241F00103D1B210
:1063C000029A937185E6824B1B78002B00F0BE8009
:1063D000029B9A7ADB7A5FE67E4B1C88794B1E68BB
:1063E000029B9D79631C9AB2A31C98B2910B764BC9
:1063F00053F82110774B1A8006F10A03714EC2F34D
:106400000D023360895C704A830B52F82320714B74
:106410001880C0F30D03D35C6E4A01EB03236906B9
:106420009BB258BFE31C1380FBF785BA029B9B7994
:1064300058065CD5684B1C88624B1D68631C98B27B
:10644000820B05F10B03A10B5F4D55F8211055F898
:1064500022505C4A1360C4F30D03C0F30D02C95C03
:106460005D4B1880AB5C41EA03235A490B805A4BC1
:10647000A21C1A80FBF75FBA574B56491B88088845
:10648000504A013B99B2431C5348126801804D4861
:106490000B32B1F5804F026098B20DD3B1F5B64F13
:1064A00002D24A4A012313708B0B474AC1F30D01F4
:1064B00052F82320030A5354474B1B88013B9AB2DE
:1064C000454BB2F5804F1A800CD3B2F5B64F02D2CD
:1064D0003E4901230B70930B3B49C2F30D0251F867
:1064E000233098543B4A00231380FBF724BA354BE2
:1064F00034491A68374B05321B880A60354A013324
:106500001380FBF718BA344B1C882E4B1D68631C94
:1065100098B2820B05F10A03A10B2B4D55F82110FF
:1065200055F82250274A1360C4F30D03C0F30D023F
:10653000C95C294B1880AB5C41EA032325490B80D9
:10654000254BA21C1A80FBF7F6B90E46029B1D498B
:106550001A795B790C6843EA0220830B1A4A52F8D5
:10656000232004F10F03174CC0F30D012360525C8C
:10657000A3E5174B187828B10E46002028E70E46F1
:106580000020C7E50629E0D00E4B029A1B680D4C8F
:10659000525C083323600E468FE50D4B1B78EBB140
:1065A000029B9A7ADB7AFCF76ABB029A43F04003BB
:1065B0009371029B029A9B7903F07F039371FCF71E
:1065C000EFBB00BFB0BD012044A50120A500002005
:1065D000ACBD0120AABD01204EBC01200629029BB2
:1065E00034D0029A9B79525C8D49096803F001030B
:1065F00043EA420201F108038949062E95B20B6075
:106600007CF458ABFCF758BB5008029A23F0010306
:106610009371FCF7B0BB834B1C7854B3029B9A7AFE
:10662000DB7AFCF78BBBB1F5804FFCF4A9ABB1F57D
:10663000B64F02D27C4A012313708B0BC1F30D02BB
:106640007A4951F823309854FCF79ABB1A79744967
:106650005B790D6843EA0221880B744B53F82020C4
:1066600005F10F036E4DC1F30D042B60125DFCF7B5
:1066700017BB062901F0B685694B029A1B6868486A
:10668000525C083321460360FCF769BB684B674FD7
:106690001E88634B67481D68029BDC79731C9BB2A4
:1066A0009A0BC3F30D0157F82220614F3B80EB1D7D
:1066B0005B4D2B60515C04F00F0201F00F0313449B
:1066C00013F0100F837914BF43F0100323F010036D
:1066D000837181EA04036218DB0995B245F04F80AB
:1066E00084EA02031B0645F14A80029B02999B79CA
:1066F00043F004038B71029B4D49DA714D4A937943
:10670000EF054CBF43F0010323F001039371029B9B
:10671000029A9B7915F0FF0F14BF23F0400343F05A
:1067200040039371029B029A9B792C064CBF63F045
:106730007F0303F07F039371029BB21C9B790A8055
:10674000029A23F002039371FBF7F5B83A4B1B78DA
:10675000002B01F03C82324B314A1B680B33136033
:106760000824334B31491D886B1C9BB29A0BC3F331
:106770000D0051F822102E4A13800B5C02990B5524
:106780002B4BAA1C1A80FBF7D6B82B4B1B7804F0B6
:106790000701A3B1224B22481B6803F108020B1F1B
:1067A000012B026000D80431214B1A88029B5B5CEC
:1067B0000299CB70531C1E4A1380FBF7BCB8194BCF
:1067C0001B78002B04F05882154B15481A680B1FD4
:1067D000DBB20832012B0260E6D88B1DD9B2E3E7A9
:1067E000154B1B783BB90F4B1B7823B90C4B0C4A4C
:1067F0001B68073313600E4B0C491C88631C9BB24B
:106800009A0BC3F30D0051F82210094A13800B5C58
:1068100002990B70064BA21C1A80FBF78CB800BFC4
:10682000B0BD0120ACBD0120A500002044A5012081
:10683000AABD012000BD01204EBD0120A14B1B7847
:106840001BB9A14B1B78002B43D0A04B9F4A1B6860
:1068500008331360029B9E49187800F00F035A1EFC
:10686000431E9CB28B79D7064CBF43F0100323F034
:1068700010038B71C30932D080EA04031E062ED5A3
:10688000029B029A9B7943F004039371904A029B06
:1068900002991C70937914F0FF0F14BF23F040038A
:1068A00043F040039371029B029A9B7925064CBFEB
:1068B00063F07F0303F07F039371029B9A79854B0A
:1068C00042F002021B888A71824A01331380FBF76F
:1068D00032B87E4B7D4A1B6804331360BAE7029BD3
:1068E000029A9B7923F004039371CFE7754B1B78D1
:1068F00004F00704002B5DD0744B74491B6803F14E
:106900000802231F012B0A6000D80434029B704E3A
:10691000DD79195D987905F00F0201F00F03D21AA5
:1069200000F00103D21A691ACB1AD70699B24CBFEC
:1069300040F0100320F01003B371029B644A1B5D0A
:106940006B401E0642F1978385EA01031C0642F163
:106950009283937943F0040393715D4A029BD9714A
:106960009379C8054CBF43F0010323F001039371F1
:10697000029B029A9B7911F0FF0F14BF23F0400392
:1069800043F040039371029B9B790A06029A029995
:106990004CBF63F07F0303F07F039371029B9A79EE
:1069A0004C4B42F002021B888A714A4A0133138021
:1069B000FAF7C1BF444B1B78002B04F0E384434B30
:1069C00042491A68231FDBB20832012B0A609DD8A6
:1069D000A31DDCB29AE73B4B1B783BB93A4B1B78C3
:1069E00023B93A4B394A1B6807331360394B3A498C
:1069F0001C88631C9BB29A0BC3F30D0051F8221044
:106A0000344A13800B5C02998B70324BA21C1A80A3
:106A1000FAF791BF2B4B1B781BB92B4B1B78002B24
:106A200043D02A4B294A1B6808331360029B28492C
:106A3000987800F00F035A1E431E9CB28B79D5063E
:106A40004CBF43F0100323F010038B71C30932D005
:106A500080EA040319062ED5029B029A9B7943F023
:106A6000040393711A4A029B02999C70937914F063
:106A7000FF0F14BF23F0400343F040039371029BC8
:106A80009B792206029A4CBF63F07F0303F07F03D9
:106A90009371029B9A790F4B42F002021B888A7114
:106AA0000C4A01331380FAF746BF084B074A1B68AC
:106AB00004331360BAE7029B029A9B7923F0040324
:106AC0009371CFE74EBD0120ACBD0120B0BD0120C8
:106AD00000BD0120AABD012044A50120844B1B78E4
:106AE000002B3DD0834B844A1B881168029A83484F
:106AF000147A01339BB29A0B133150F822007D4A6D
:106B00001380C3F30D027C4B1960029B82565B7AA3
:106B100043EA0423134498B2764B784C1B88013324
:106B20009BB29A0BC3F30D0154F82220714CB0F5BF
:106B3000804F2380515C0CD3B0F5B64F02D2704A1F
:106B400001231370830BC0F30D026C4850F82330FF
:106B50009954684B674A1B8801331380FAF7EBBEE0
:106B6000684B1B78002B00F0AC80624B624A1B889C
:106B70001168029A6148947A01339BB29A0B1331DF
:106B800050F822005B4A1380C3F30D025A4B196080
:106B9000029B8256DB7A43EA0423134498B2BBE794
:106BA000534B1B78002B6ED0524B534A1B881168F5
:106BB000029A5248147A01339BB29A0B173150F85B
:106BC00022004C4A1380C3F30D024B4B1960029B09
:106BD00082565B7A43EA0423134498B2830B474AF4
:106BE000C0F30D0652F82350A95D01F00F035A1EA1
:106BF0004B1E9CB2029B9B79D206029A4CBF43F07B
:106C0000100323F010039371CB0935D081EA0403FC
:106C10001F0631D5029B029A9B7943F004039371BE
:106C2000B0F5804F06D3B0F5B64F02D2344A0123F7
:106C30001370AC55029B029A9B79029914F0FF0FD6
:106C400014BF23F0400343F040039371029B029A68
:106C50009B7920064CBF63F07F0303F07F039371A1
:106C6000029B9A79234B42F002021B888A71214AC7
:106C700001331380FAF75FBE029B029A9B7923F0DF
:106C800004039371CCE71F4B1B782BB3194B1A4AA3
:106C90001B881168029A1948947A01339BB29A0BA7
:106CA000173150F82200134A1380C3F30D02124B20
:106CB0001960029B8256DB7A43EA0423134498B29C
:106CC0008CE70D4B029A1B6811790B4852790A33F5
:106CD000036042EA01201FE7074B029A1B68117903
:106CE000054852790B33036042EA012076E700BF82
:106CF0004EBD0120AABD0120B0BD012044A5012048
:106D0000A5000020ACBD0120A44B1B78002B6DD04A
:106D1000A34BA44A1B881168029AA348147A013332
:106D20009BB29A0B173150F822009D4A1380C3F38F
:106D30000D029C4B1960029B82565B7A43EA042346
:106D4000134499B28B0B984A029E52F82340C1F328
:106D50000D05625D02F00F03013313F0100F029B6B
:106D60009B7914BF43F0100323F01003B371D309D0
:106D700002F1010033D182EA00031E062FD5029BE7
:106D8000029A9B7943F004039371B1F5804F06D3C7
:106D9000B1F5B64F02D2854A012313706055029BAC
:106DA000029C9A79824902F0FD0310F0FF0FA37153
:106DB00014BF22F0420343F040038B71029B029AFE
:106DC0009B7901064CBF63F07F0303F07F0393714F
:106DD000734B734A1B8801331380FAF7ACBD029BD7
:106DE000029A9B7923F004039371CEE7714B1B78D1
:106DF000002B2BD06A4B6B4A1B881168029A6A4899
:106E0000947A01339BB29A0B173150F82200644AEE
:106E10001380C3F30D02634B1960029B8256DB7A29
:106E200043EA0423134499B28CE75E4B5D4819682A
:106E3000614B06311A885A4B01605F491B88013249
:106E40000A80574A01331380FAF775BD554B029AF1
:106E50001B681179534852790B33036042EA0121D0
:106E600070E74F4B504C19884E4B1D684B1C9AB223
:106E70008B1C99B2930B880B54F82340484B1A8013
:106E800005F10D03474D2B60474BC2F30D0253F83C
:106E90002000434BA25C1980C1F30D03C35C02EBDD
:106EA00003239AB2B2F5804F0ED3B2F5B64F02D299
:106EB0003E4901230B70930BC2F30D013A4A52F87D
:106EC0002320029BDB795354354B354A1B88013311
:106ED0001380FAF730BD324B33481C88314B1D68A4
:106EE000631C9BB29A0BA11C50F822002C4A138001
:106EF000C3F30D0205F10A032A4D89B22B60855CAC
:106F0000294A8B0B52F82300254B1980C1F30D033E
:106F10002349C35CE21C0A80274A05EB0323138044
:106F2000FAF709BD1E4B1E4C1888029B1E499D791D
:106F3000431C9BB29A0B238051F82210C3F30D031C
:106F4000821CCB5692B21344EF079BB21DD4154A54
:106F50002380126802F10C03124A1360FAF7EBBCAB
:106F6000104B104C1868029B0430D9799A790C4B5D
:106F7000206002981B8842F012028271084AC943BD
:106F80000133C1711380FAF7D6BC064B22801B680F
:106F9000044A07331360FAF7CEBC00BF4EBD012090
:106FA000AABD0120B0BD012044A50120A5000020FC
:106FB00000BD0120ACBD01204EBC0120A44B1B78BC
:106FC000002B63D0A34BA34A1B680B331360092427
:106FD000A14BA2491D886B1C9BB29A0BC3F30D00F9
:106FE00051F822109C4A13800B5C02990B559A4B66
:106FF000AA1C1A80FAF79FBC954B1B78002B00F057
:107000004C82944B934A1B68083313600924029BFB
:1070100093481A5D02F00F03591E531E9DB28379E7
:107020008F4ACE064CBF43F0100323F01003837148
:10703000029B1B5DD90935D06B40190632D5937977
:1070400043F004039371029B854A1D55937902997D
:1070500015F0FF0F14BF23F0400343F0400393717A
:10706000029B9B792A06029A4CBF63F07F0303F0D0
:107070007F039371029B9A79774B42F002021B883F
:107080008A71754A01331380FAF755BC754B1B782A
:10709000002B00F00C826F4B6E4A1B680B331360A1
:1070A0000B2495E7029B029A9B7923F004039371CA
:1070B000C9E7694B69481988654B684D1E784B1CB8
:1070C0009AB28B1C99B2930B8C0B50F82300624B35
:1070D0001A80C2F30D03614AC05C5F4B52F8242052
:1070E0001980C1F30D03D35C00EB032398B2002E8B
:1070F00054D0584A411C1768820B8B13C1F30D04FE
:1071000055F82210534A55F8236007F11403136011
:10711000C0F30D03325DCB5C029903EB02239BB2FB
:107120001A0A4B720A724C4B4B4A1B88013313806C
:10713000FAF701BC464B1B78002B4ED0029B454909
:107140001A7A0C685B7A4649424D43EA022204F1FE
:107150000F032B608B7917054FEA42004CBF43F0B9
:10716000100323F01003029A8B71030A0446507235
:107170001372029B02989A79394902F0FD038371D8
:10718000E00354BF22F0030343F001038B71324B41
:10719000314A1B8801331380FAF7CDBB314B1B7882
:1071A000411C002B39D02B4A1768820B8B13C1F37B
:1071B0000D0455F82210274A55F8236007F11403EF
:1071C0001360C0F30D03325DCB5C029903EB022325
:1071D0009BB21A0ACB728A72A5E7224B1B78002B4E
:1071E00042D0029B1B499A7A0C68DB7A1C49194DE4
:1071F00043EA022204F10F032B608B7916054FEA54
:1072000042004CBF43F0100323F01003029A8B712D
:10721000030A0446D0729372ABE70E4A1768820BDA
:107220008B13C1F30D0455F822100A4A55F8236058
:1072300007F110031360C0F30D03325DCB5C0299BC
:1072400003EB02239BB21A0A4B710A716BE700BF72
:107250004EBD0120B0BD0120AABD012044A50120E2
:1072600000BD0120ACBD0120029B9D491A790C682C
:107270005B799C499A4D43EA022204F10B032B608F
:107280008B7915054FEA42004CBF43F0100323F001
:107290001003029A8B71030A04465071137168E758
:1072A000914B914C1888029B90499D79431C9BB24D
:1072B0009A0B238051F82210C3F30D03821CCB5686
:1072C00092B2134469069BB262D5854A2380126844
:1072D00002F10C03824A1360FAF72DBB029A804B2D
:1072E00091791B687E487F4A0433CF06036057D4E8
:1072F000D37903F00F03092B8CBF06240024CE079B
:1073000003D4029BDB79992B06D904F16002D4B235
:10731000029A41F001039371029B724A997901F03C
:107320001203022B4BD0122BD37903F00F0344D05E
:10733000092B44D941F010039371029B694A987953
:10734000DB79850746BF1B1B99B21919029BCCB28A
:10735000DC71002C2DD020F040039371029B029A27
:107360009B7908064CBF63F07F0303F07F039371A2
:107370005F4B1B5DB3B1029B029A9B7943F0040300
:107380009371594B584A1B8801331380FAF7D3BACB
:10739000534B22801B68524A07331360FAF7CBBA6B
:1073A0000624ACE7029B029A9B7923F004039371B5
:1073B000E7E740F040039371D0E7052BBAD921F0FD
:1073C00010039371B9E74B4B1B78002B7DD0444BD6
:1073D000434A1B68083313600920029B41491A5C29
:1073E00002F00F03013313F0100F8B7914BF43F039
:1073F000100323F010038B71029B1B5CD90902F16F
:107400000104384A42D163401B063FD5937943F0CB
:1074100004039371029B33491C549A79029802F039
:10742000FD0314F0FF0F837114BF22F0420343F0F9
:1074300040038B71029B029A9B7927064CBF63F035
:107440007F0303F07F039371274B274A1B88013387
:107450001380FAF770BA274B1B78002B4ED0029B93
:107460001F491A7A5B7A0298096843EA0223013BB2
:107470009AB2130A03721A4B42720A3119601A4BFC
:10748000194A1B8801331380FAF755BA029B029AF6
:107490009B7923F004039371BCE7174B1B786BB106
:1074A0000F4B0F4A1B68083313600B24AFE50C4BDE
:1074B0000B4A1B6807331360052489E5084B084A0B
:1074C0001B68043313600524A1E50B4B1B784BB3F9
:1074D000034B034A1B68083313600B207DE700BF92
:1074E000B0BD012000BD0120AABD012044A501209E
:1074F000F45B01084EBD0120ACBD01209C4B1B7804
:10750000BBB1029B9B499A7ADB7A0298096843EAED
:107510000223013B9AB2130A8372964BC2720A315C
:107520001960ACE7934B934A1B6804331360052042
:1075300053E7029B8F491A795B790298096843EAFD
:107540000223013B9AB2130A03718A4B427106313E
:10755000196094E7884B1B783BB9854B1B7823B99E
:10756000844B844A1B6807331360844B84491C880E
:10757000631C9BB29A0BC3F30D0051F822107F4A93
:1075800013800B5C0299CB717C4BA21C1A80FAF71A
:10759000D2B9794B1B781BB9754B1B78002B43D0A4
:1075A000744B744A1B6808331360029B7549D87981
:1075B00000F00F035A1E431E9CB28B79D5064CBFB8
:1075C00043F0100323F010038B71C30932D080EA1B
:1075D000040319062ED5029B029A9B7943F00403FB
:1075E0009371684A029B0299DC71937914F0FF0F42
:1075F00014BF23F0400343F040039371029B9B7937
:107600002206029A4CBF63F07F0303F07F0393715D
:10761000029B9A79594B42F002021B888A71574AA1
:1076200001331380FAF787B9524B524A1B6804336F
:107630001360BAE7029B029A9B7923F004039371CB
:10764000CFE74D4B1B781BB9494B1B78002B53D010
:10765000484B484A1B6808331360029B494AD97952
:1076600001F00F03013313F0100F937914BF43F0AF
:10767000100323F010039371CB0901F1010041D1F4
:1076800081EA00031F063DD5029B029A9B7943F0D5
:1076900004039371029B029A9979D87101F0FD035A
:1076A000937110F0FF0F374A14BF21F0420343F0EB
:1076B00040039371029B029A9B7906064CBF63F0CC
:1076C0007F0303F07F0393712C4B2C4A1B880133FB
:1076D0001380FAF730B9274B264819682A4B063130
:1076E0001A88264B016028491B88013A0A80234AE0
:1076F00001331380FAF71FB91E4B1E4A1B6804336F
:107700001360AAE7029B029A9B7923F0040393710A
:10771000C0E71A4B1A4C1888164B1D68431C9BB2C5
:107720009A0B811C54F82240144A1380C3F30D02B3
:1077300005F10D030F4D89B22B60A45C104A8B0B31
:10774000033052F823200D4B1980C1F30D03D35C95
:1077500004EB03239BB2C3F30D02990B084B53F8C0
:1077600021309B5C029AD371044B1880FAF7E3B87E
:10777000ACBD0120B0BD01204EBD0120AABD01203D
:1077800044A5012000BD01204EBC01209F4B1B7869
:10779000002B67D0029B9E491A7A9E485B7A098823
:1077A00005689D4843EA02235C18C3F30B02C1F34A
:1077B0000B0398491A4405F10F030B608379D20437
:1077C0004CBF43F0100323F01003029A8371230A85
:1077D000254654721372029B02989A798E4902F0E0
:1077E000FD038371E80354BF22F0030343F0010358
:1077F0008B718A4B894A1B8801331380FAF79BB837
:10780000864B864C1888029B85499D79431C9BB208
:107810009A0B238051F82210C3F30D03821CCB5620
:1078200092B21344E9079BB241D57A4A2380126889
:1078300002F10C03774A1360FAF77DB8029B77498F
:107840009B790888734A23F0120343F00101431C1B
:107850000298126881716F4904320A606F4A13807E
:10786000FAF769B86F4B1B784BB3029B68499A7A59
:107870006848DB7A09880568674843EA02235C1890
:10788000C3F30B02C1F30B0362491A4405F10F0362
:107890000B608379D7044CBF43F0100323F010032F
:1078A000029A8371230A2546D472937293E7594B47
:1078B00022801B68574A07331360FAF73CB8029BD3
:1078C00053491A7953485B7909880568524843EA55
:1078D00002235C18C3F30B02C1F30B034D491A4496
:1078E00005F10B030B608379D6044CBF43F0100302
:1078F00023F01003029A8371230A254654711371F1
:1079000069E7424B1B7804F00701A3B1414B4148A2
:107910001B6803F108020B1F012B026000D8043121
:107920003E4B1A88029B5B5C02994B70531C3B4A8E
:107930001380FAF700B83B4B1B78002B00F0EE8069
:10794000344B34481A680B1FDBB20832012B02603B
:10795000E6D88B1DD9B2E3E72C4B1B78002B00F047
:10796000E3802E4B2B4A1B881168029A2C48147A0C
:1079700001339BB29A0B133150F82200274A13802F
:10798000C3F30D02234B1960029B82565B7A43EAD4
:10799000042313449BB29A0BC3F30D01204B53F8FD
:1079A00022301E4A5B5C128802990B70531C1B4AE2
:1079B0001380F9F7C0BF154B1B7804F00701A3B182
:1079C000144B14481B6803F108020B1F012B0260C3
:1079D00000D80431114B1A88029B5B5C02998B70B2
:1079E000531C0E4A1380F9F7A6BF0E4B1B78002BD1
:1079F00000F0E780074B07481A680B1FDBB208321C
:107A0000012B0260E6D88B1DD9B2E3E74EBD012001
:107A10004EBC0120B0BD012000BD0120AABD012047
:107A200044A50120ACBD0120974B1B78002B00F032
:107A3000EC80964B964A1B881168029A9548147AF6
:107A400001339BB29A0B133150F822008F4A1380F6
:107A5000C3F30D028E4B1960029B82565B7A43EA98
:107A6000042313449BB29A0BC3F30D01894B53F8C3
:107A70002230864A5B5C128802994B70531C834A01
:107A80001380F9F758BF804B1B7804F00701A3B1AE
:107A90007F4B7F481B6803F108020B1F012B02601C
:107AA00000D80431794B1A88029B5B5C02990B70F9
:107AB000531C764A1380F9F73EBF774B1B783BB3D4
:107AC000734B73481A680B1FDBB20832012B02603C
:107AD000E8D88B1DD9B2E5E76D4B029A1B68927905
:107AE0006B486E4904330360D3074CBF22F0010397
:107AF00042F001038B71029B02999A79634B22F049
:107B000002021B888A71614A01331380F9F713BF9F
:107B10005F4B5F4A1B6804331360C3E75C4B5C4AEE
:107B20001B6804331360FBE65B4B1B78002B59D0BA
:107B3000564B574A1B881168029A5648947A01336B
:107B40009BB29A0B133150F82200504A1380C3F3B2
:107B50000D024F4B1960029B8256DB7A43EA0423E5
:107B600013449BB217E7484B1B78002B6CD0474B54
:107B7000474A1B881168029A4648147A01339BB21F
:107B80009A0B133150F82200404A1380C3F30D02C0
:107B90003F4B1960029B82565B7A43EA04231344ED
:107BA0009BB29A0BC3F30D013A4B53F82230374A7C
:107BB0005B5C128802998B70531C344A1380F9F76E
:107BC000BABE334B324A1B680433136002E7324BB0
:107BD0001B7893B12E4B2E4A1B680B3313600A247B
:107BE000FEF7BFBD2A4B029A1B68117928485279CB
:107BF0000733036042EA0123CDE6254B244A1B6884
:107C0000073313600424FEF7ACBD234B1B78002B15
:107C100046D01E4B1E4A1B881168029A1D48947A52
:107C200001339BB29A0B133150F82200174A13808C
:107C3000C3F30D02164B1960029B8256DB7A43EAAE
:107C4000042313449BB20EE7134B1B78002B32D056
:107C50000E4B0F4A1B881168029A0E48947A013322
:107C60009BB29A0B133150F82200084A1380C3F3D9
:107C70000D02074B1960029B8256DB7A43EA04230C
:107C800013449BB28DE700BF4EBD0120AABD012069
:107C9000B0BD012044A50120ACBD012000BD0120E4
:107CA0009C4B029A1B6811799A48527907330360FA
:107CB00042EA0123D7E6974B029A1B68117995484F
:107CC00052790733036042EA01236AE7924B1B783B
:107CD00004F00704002B59D08E4B8E491B6803F12A
:107CE0000802231F012B0A6000D80434029B8B4832
:107CF000DD79195D05F00F0201F00F03D31A13F0BF
:107D0000100F8379854A14BF43F0100323F010034A
:107D10008371029B1B5D6B40691A1C068EB240F199
:107D2000AC8485EA0103180640F1A784937943F0F7
:107D300004039371029B029A9B79F1054CBF43F0B7
:107D4000010323F001039371029B029A9B7902992C
:107D500016F0FF0F14BF23F0400343F0400393716C
:107D6000029B9B793206029A4CBF63F07F0303F0BB
:107D70007F039371029B9A79694B42F002021B8840
:107D80008A71674A01331380F9F7D5BD654B1B78BB
:107D9000002B01F085835F4B5E491A68231FDBB21D
:107DA0000832012B0A60A1D8A31DDCB29EE75A4B12
:107DB0001B7804F00701A3B1564B56481B6803F12A
:107DC00008020B1F012B026000D80431544B1A88A3
:107DD000029B5B5C0299CB71531C514A1380F9F7EB
:107DE000AABD504B1B7893B14A4B4A481A680B1FE7
:107DF000DBB20832012B0260E8D88B1DD9B2E5E76F
:107E0000444B444A1B6804331360F9F794BD414B5B
:107E1000404A1B6804331360D8E7414B1C883D4B34
:107E20001E68029B9D79631C9AB2A31C98B2910BA9
:107E30003D4B53F821103A4B1A8006F10A03354E98
:107E4000C2F30D023360895C374A830B52F823205A
:107E5000334B1880C0F30D03D35C314A01EB03238D
:107E600069069BB248BFE31C1380F9F764BD2F4B32
:107E70001D88284B1C682A4B1F886B1C98B2A90BC5
:107E800004F10A03284C820B54F82140264951F88A
:107E90002260204A1360C5F30D03C0F30D01E25CBC
:107EA000224B029C1880735C42EA03231BB2C3F38B
:107EB000072063701D4B2070A91C1980184B7A1C79
:107EC0001A80F9F738BD029B9B79580600F1A38010
:107ED000164B1C880F4B1D68631C98B2820B05F172
:107EE0000B03A10B104D55F8211055F82250094AEB
:107EF0001360C4F30D03C0F30D02C95C0B4B188073
:107F0000AB5C41EA032306490B80084BA21C1A8094
:107F1000F9F711BDB0BD01204EBD012000BD01200B
:107F2000AABD0120ACBD012044A501204EBC01200A
:107F3000A44B1B78002B00F08180A34BA34A1B8825
:107F40001168029AA248147A01339BB29A0B13313A
:107F500050F822009C4A1380C3F30D029B4B19601A
:107F6000029B82565B7A43EA042313449BB29A0B2A
:107F7000C3F30D01964B53F82230029A585CD47922
:107F8000944900F00F0204F00F039B1A13F0100F36
:107F90008B7914BF43F0100323F010038B7180EA38
:107FA0000403221A1B0695B241D584EA02031F0678
:107FB0003DD5029B029A9B7943F004039371029B87
:107FC000029A9B790299EE054CBF43F0010323F01E
:107FD00001039371029B029A9B7915F0FF0F14BF66
:107FE00023F0400343F040039371029B029A9B7974
:107FF0002C064CBF63F07F0303F07F039371029B59
:108000009A79714B42F002021B888A716E4A0133E1
:108010001380F9F790BC6D4B6C491A686A4B0532B6
:108020001B880A60684A01331380F9F784BC029BFD
:10803000029A9B7923F004039371C0E7664B1B7887
:10804000002B00F00781604B604A1B881168029A80
:108050005F48947A01339BB29A0B133150F8220097
:10806000594A1380C3F30D02584B1960029B825684
:10807000DB7A43EA042313449BB278E7524B54481B
:108080001C88029B9D79631C9BB29A0BA11C50F823
:1080900022004D4A1380C3F30D0289B28B0B805C22
:1080A0004B4A52F82320484B1980C1F30D0346492F
:1080B000D35C6A0600EB03239EB238D4474B434A95
:1080C0001B881068013BE11C9AB200F1110388B2D1
:1080D00042490A803D49B2F5804F0B600DD3B2F59D
:1080E000B64F02D23E4901230B70930BC2F30D0130
:1080F000374A52F82320030A5354384B1B88013B5C
:108100009AB2364BB2F5804F1A800CD3B2F5B64F07
:1081100002D2334901230B70930B2D49C2F30D0298
:1081200051F823309854284B1E80F9F704BC274B94
:10813000E21C1B680A80254A0A331360F9F7FBBB6F
:10814000029B224819785A78244B00681B8842EA1F
:108150000122013B214914B29AB20A801B4900F165
:108160000B03B2F5804FA0B20B600DD3B2F5B64F42
:1081700002D21B4901230B70930BC2F30D01144A69
:1081800052F82320030A5354144B1B88013B9AB224
:10819000124BB2F5804F1A800CD3B2F5B64F02D213
:1081A0000F4901230B70930B0949C2F30D0251F8DB
:1081B00023309C54044B044A1B8801331380F9F785
:1081C000BABB00BF4EBD0120AABD0120B0BD012039
:1081D00044A5012000BD0120ACBD01204EBC012002
:1081E000A5000020029B71491A795B790C6843EA6B
:1081F00002218B0B6E4A52F8232004F10F036B4CC3
:10820000C1F30D002360125CFAF7A9BD694B684CFD
:108210001988664B1D684B1C9AB28B1C99B2930B44
:10822000880B54F82340634B1A8005F10A035F4D15
:108230002B605F4BC2F30D0253F820005D4BA25C34
:108240001980C1F30D03C35C02EB0323594A138069
:10825000F9F771BB554B029A1B6811795348527953
:108260000733036042EA012381E6534B1B7804F095
:108270000701002B33D04D4B4C481B6803F108021B
:108280000B1F012B026000D80431029B5A5CDB7982
:108290004A495A40029BDA718B79002A00F0AF827A
:1082A00003F0BF0310068B7140F1AC8263F07F03D3
:1082B0008B71029B029C9979414B40489A5C01F07A
:1082C000EC03A371002A00F0688243F00403837179
:1082D000384B384A1B8801331380F9F72CBB394BD4
:1082E0001B78002B56D0314B30481A680B1FDBB27D
:1082F0000832012B0260C8D88B1DD9B2C5E72E4BBE
:108300001B7804F00701002B35D0284B27481B6849
:1083100003F108020B1F012B026000D80431029BFD
:108320005A5CDB7925491A40029BDA718B79002A65
:1083300000F0EB8003F0BF0315068B7140F1E8807D
:1083400063F07F038B71029B029D99791C4B1B4C40
:10835000985C01F0FC0242F01003AB71002800F0C1
:10836000A98042F01403A371124B124A1B880133F7
:108370001380F9F7E0BA134B1B788BB10B4B0B480A
:108380001A680B1FDBB20832012B0260C7D88B1DA5
:10839000D9B2C4E7054B054A1B680433136074E780
:1083A000024B024A1B6804331360B8E7B0BD0120DA
:1083B00044A50120AABD01204EBD012000BD012021
:1083C000F45B0108ACBD0120804B1B78002B7ED0F4
:1083D0007F4B804A1B881168029A7F48147A0133C8
:1083E0009BB29A0B133150F82200794A1380C3F3E1
:1083F0000D02784B1960029B82565B7A43EA042394
:1084000013449BB29A0BC3F30D01734B734E53F895
:108410002230029A5D5CD479907904F00F0305F064
:108420000F02991A00F00103621BC91AD31A9FB2F6
:10843000CB064CBF40F0100320F01003B37185EA67
:1084400004031D063CD584EA0703180638D5029BB1
:10845000029A9B7943F004039371604A029BDF7197
:108460009379F9054CBF43F0010323F001039371A5
:10847000029B029A9B79029917F0FF0F14BF23F019
:10848000400343F040039371029B029A9B793E069E
:108490004CBF63F07F0303F07F039371029B9A79D3
:1084A0004B4B42F002021B888A71494A0133138008
:1084B000F9F741BA21F0070343F01003A37153E722
:1084C000029B029A9B7923F004039371C5E7444B06
:1084D0001B7823B33E4B3F4A1B881168029A3E48E3
:1084E000947A01339BB29A0B133150F82200384A28
:1084F0001380C3F30D02374B1960029B8256DB7A5F
:1085000043EA042313449BB27CE743F040038B719E
:10851000029B02999B7903F07F038B7113E72D4B2C
:10852000029A1B6811792B4852790733036042EA9B
:10853000012367E7254B1B7804F00701002B33D09C
:10854000244B24481B6803F108020B1F012B026017
:1085500000D80431029B5A5CDB7920491A43029B04
:10856000DA718B79002A00F0E68103F0BF0316066A
:108570008B7140F1E38163F07F038B71029B029C5E
:108580009979184B15489A5C01F0EC03A371002A05
:1085900000F0A18143F0040383710D4B0C4A1B884A
:1085A00001331380F9F7C7B90D4B1B78002B00F08E
:1085B0009880084B07481A680B1FDBB20832012B62
:1085C0000260C7D88B1DD9B2C4E700BF4EBD0120E1
:1085D000AABD0120B0BD012044A5012000BD01209D
:1085E000ACBD0120F45B01088F4B1B78002B5AD0E7
:1085F0008E4B8F4A1B881168029A8E48147A013379
:108600009BB29A0B133150F82200884A1380C3F3AF
:108610000D02874B1960029B82565B7A43EA042362
:1086200013449BB29A0BC3F30D01824B53F82230D3
:10863000029A5B5CD27980491A43029BDA718B798A
:108640003AB303F0BF0315068B7125D563F07F03A2
:108650008B71029B029C9979784B77489A5C01F068
:10866000EC03A3718AB143F0040383716F4B6F4A2B
:108670001B8801331380F9F75EB9029B029A9B793C
:1086800023F004039371FFF755BB21F017038371A7
:10869000ECE743F040038B71029B02999B7903F056
:1086A0007F038B71D5E7664B1B7803B35F4B604A42
:1086B0001B881168029A5F48947A01339BB29A0B27
:1086C000133150F82200594A1380C3F30D02584B5E
:1086D0001960029B8256DB7A43EA042313449BB25F
:1086E000A0E7534B524A1B680433136032E7504BE8
:1086F000029A1B6811794E4852790733036042EAA7
:1087000001238FE7484B1B78002B5AD0474B484A30
:108710001B881168029A4748147A01339BB29A0B5E
:10872000133150F82200414A1380C3F30D02404B2D
:108730001960029B82565B7A43EA042313449BB27E
:108740009A0BC3F30D013B4B53F82230029A5B5C4A
:10875000D27939491A40029BDA718B793AB303F026
:10876000BF0314068B7125D563F07F038B71029BC9
:10877000029D9979314B304C985C01F0FC0242F03B
:108780001003AB7168B142F01403A371274B274A61
:108790001B8801331380F9F7CEB821F017038371DA
:1087A00096E521F0070343F01003A371EEE743F0D1
:1087B00040038B71029B02999B7903F07F038B71BD
:1087C000D5E71F4B1B7823B3184B194A1B88116838
:1087D000029A1848947A01339BB29A0B133150F8DD
:1087E0002200124A1380C3F30D02114B1960029B41
:1087F0008256DB7A43EA042313449BB2A0E743F09A
:1088000040038B71029B02999B7903F07F038B716C
:108810004FE5074B029A1B681179054852790733D7
:10882000036042EA01238BE74EBD0120AABD01206F
:10883000B0BD012044A5012000BD0120F45B01086A
:10884000ACBD01208E4B1B78002B56D08D4B8E4A31
:108850001B881168029A8D48147A01339BB29A0BD7
:10886000133150F82200874A1380C3F30D02864B60
:108870001960029B82565B7A43EA042313449BB23D
:108880009A0BC3F30D01814B53F82230029A5B5CC3
:10889000D2797F495A40029BDA718B791AB303F07F
:1088A000BF0317068B7121D563F07F038B71029B89
:1088B000029C9979774B76489A5C01F0EC03A3719E
:1088C0006AB143F0040383716E4B6E4A1B88013317
:1088D0001380F9F730B821F0170383715DE621F0BA
:1088E00017038371F0E743F040038B71029B0299F9
:1088F0009B7903F07F038B71D9E7674B1B7823B318
:10890000604B614A1B881168029A6048947A01336F
:108910009BB29A0B133150F822005A4A1380C3F3CA
:108920000D02594B1960029B8256DB7A43EA0423FD
:1089300013449BB2A4E743F040038B71029B02995E
:108940009B7903F07F038B7118E64F4B029A1B68EB
:1089500011794D4852790733036042EA01238FE7CA
:10896000474B1B7804F00705002B5CD0464B46496B
:108970001B6803F108022B1F012B0A6000D8043585
:10898000029B434F9879DE795C5D00F0010106F0AF
:108990000F03CA1804F00F031A4433191944D306FD
:1089A0004CBF40F0100320F01003BB71029B384A0B
:1089B0005B5D7340DB0940F0178586EA01031C0606
:1089C00040F11285937943F004039371304A029B7E
:1089D000D9719379C8054CBF43F0010323F001031B
:1089E0009371029B029A9B7911F0FF0F14BF23F041
:1089F000400343F040039371029B9B790A06029A5D
:108A000002994CBF63F07F0303F07F039371029BD5
:108A10009A791C4B22F002021B888A71194A013391
:108A20001380F8F788BF1C4B1B78002B00F046859D
:108A3000154B15491A682B1FDBB20832012B0A604F
:108A40009ED8AB1DDDB29BE70D4B1B7804F00700F1
:108A5000002B54D00C4B0C491B6803F10802031F78
:108A6000012B0A6048D90922064B1988029B1B5C1E
:108A700002988354034A4B1C1380F8F75CBF00BF75
:108A80004EBD0120AABD0120B0BD012044A501209A
:108A900000BD0120F45B0108ACBD01209E4B1B789A
:108AA000002B3BD09D4B9E4A1B881168029A9D4823
:108AB000147A01339BB29A0B133150F82200974A73
:108AC0001380C3F30D02964B1960029B82565B7AAA
:108AD00043EA042313449BB29A0BC3F30D01914B59
:108AE00053F822308D4A5B5C128802990B71531C3B
:108AF0008A4A1380F8F71FBF04300922B4E78A4B73
:108B00001B78002B2CD0864B85491A68031FDBB2DB
:108B10000832012B0A601FD90B22A5E7824B1B7874
:108B20002BB37E4B7E4A1B881168029A7D48947A4B
:108B300001339BB29A0B133150F82200774A13800D
:108B4000C3F30D02764B1960029B8256DB7A43EA2F
:108B5000042313449BB2BFE7831DD8B20B2283E7E3
:108B60006F4B6F4A1B680433136005227CE76C4B24
:108B7000029A1B6811796A4852790733036042EA06
:108B80000123A9E7644B1B7804F00704002B5AD09B
:108B9000634B63491B6803F10802231F012B0A6022
:108BA00000D80434029B6148DD79195D05F00F029D
:108BB00001F00F03D31A13F0100F83795B4A14BF2F
:108BC00043F0100323F010038371029B1B5D6B4085
:108BD000691A1C068EB240F1F38285EA0103180679
:108BE00040F1EE82937943F0040393714F4A029B64
:108BF000D9719379F1054CBF43F0010323F00103D0
:108C00009371029B029A9B79029916F0FF0F14BF91
:108C100023F0400343F040039371029B029A9B7937
:108C200037064CBF63F07F0303F07F039371029B11
:108C30009A793A4B42F002021B888A71374A013313
:108C40001380F8F778BE384B1B78002B00F02F8488
:108C5000334B33491A68231FDBB20832012B0A60F9
:108C6000A0D8A31DDCB29DE72B4B1B7804F00705B1
:108C7000002B32D0294B2A4A1B881168029A2948B6
:108C8000147A01339BB29A0B133150F82200234A15
:108C90001380C3F30D02224B1960029B82565B7A4C
:108CA00043EA042313449AB2B2F5804F0ED3B2F5CF
:108CB000B64F02D21E4901230B70930BC2F30D0174
:108CC000184A52F82320029B5B5D5354134B134AFE
:108CD0001B8801331380F8F72EBE134B1B78002B33
:108CE00056D00E4B0E4A1B881168029A0D48947A92
:108CF00001339BB29A0B133150F82200074A1380BC
:108D0000C3F30D02064B1960029B8256DB7A43EADD
:108D1000042313449AB2C7E74EBD0120AABD012027
:108D2000B0BD012044A50120ACBD012000BD012043
:108D3000A5000020904B1B78002B34D08F4B904A1D
:108D40001B881168029A8F48147A01339BB29A0BE0
:108D5000133150F82200894A1380C3F30D02884B67
:108D60001960029B82565B7A43EA042313449BB248
:108D70009A0BC3F30D01834B53F822307F4A5B5C9F
:108D8000128802994B71531C7C4A1380F8F7D3BDAB
:108D90007B4B029A1B68117979485279073303603B
:108DA00042EA012280E7784B1B78002B00F0F28228
:108DB000724B734A1B881168029A7248947A013385
:108DC0009BB29A0B133150F822006C4A1380C3F304
:108DD0000D026B4B1960029B8256DB7A43EA042337
:108DE00013449BB2C4E7644B1B7804F00704002BC8
:108DF00058D0634B62491B6803F10802231F012B03
:108E00000A6000D80434029B6048DD79195D05F0E2
:108E10000F0201F00F03134413F0100F83795B4A24
:108E200014BF43F0100323F010038371029B1B5DFA
:108E30006B402944DB098EB243D185EA01031F064A
:108E40003FD5937943F004039371504A029BD97143
:108E500093790299F5054CBF43F0010323F0010318
:108E60009371029B029A9B7916F0FF0F14BF23F0B7
:108E7000400343F040039371029B029A9B793406AE
:108E80004CBF63F07F0303F07F039371029B9A79D9
:108E90003A4B22F002021B888A71384A0133138050
:108EA000F8F749BD384B1B7893B1354B34491A68F4
:108EB000231FDBB20832012B0A60A4D8A31DDCB249
:108EC000A1E7029B029A9B7923F004039371BCE70C
:108ED0002B4B2B4A1B680433136094E7264B1B78FB
:108EE00004F00700002B00F0F082254B24491B689A
:108EF00003F10802031F012B0A603AD908221F4B15
:108F00001988029B1B5C029883541C4A4B1C1380DB
:108F1000F8F711BD184B1B78002B00F0E582174BBA
:108F2000174A1B881168029A1648147A01339BB2BB
:108F30009A0B133150F82200104A1380C3F30D022C
:108F40000F4B1960029B82565B7A43EA0423134459
:108F50009BB29A0BC3F30D010A4B53F82230074A18
:108F60005B5C12880299CB70531C044A1380F8F79B
:108F7000E2BC04300822C2E74EBD0120AABD012098
:108F8000B0BD012044A50120ACBD012000BD0120E1
:108F9000984B1B78002B7DD0974B984A1B88116803
:108FA000029A9748147A01339BB29A0B133150F806
:108FB0002200914A1380C3F30D02904B1960029B6B
:108FC00082565B7A43EA042313449BB29A0BC3F3A1
:108FD0000D018B4B53F82230029A585CD4798949A1
:108FE00000F00F0204F00F039B1A13F0100F8B799F
:108FF00014BF43F0100323F010038B7180EA0403C5
:10900000221A1E0695B23ED584EA020318063AD506
:10901000029B02999B7943F004038B71029BDA71E6
:10902000784A9379E9054CBF43F0010323F001032B
:109030009371029B029A9B79029915F0FF0F14BF5E
:1090400023F0400343F040039371029B9B792A066F
:10905000029A4CBF63F07F0303F07F039371029B7E
:109060009A79654B42F002021B888A71624A013389
:109070001380F8F760BC029B029A9B7923F00403EB
:109080009371FDF76ABC029B02999B7923F004035C
:109090008B71C3E75C4B1B78002B00F09880564B1C
:1090A000564A1B881168029A5548947A01339BB23C
:1090B0009A0B133150F822004F4A1380C3F30D026C
:1090C0004E4B1960029B8256DB7A43EA0423134419
:1090D0009BB27BE7474B1B78002B00F09780464BF9
:1090E000464A1B881168029A4548147A01339BB29C
:1090F0009A0B133150F822003F4A1380C3F30D023C
:109100003E4B1960029B82565B7A43EA0423134468
:109110009BB29A0BC3F30D01394B3A4E53F82230F0
:10912000029A5C5C9079D57900F0010105F00F039B
:109130000B4404F00F021A4463191944D3064CBFC0
:1091400040F0100320F01003B37184EA0503DB093B
:1091500048D185EA01031F0644D5029B029A9B79F8
:1091600043F004039371274A029BD9719379CE058A
:109170004CBF43F0010323F001039371029B029A59
:109180009B7911F0FF0F14BF23F0400343F040031D
:109190009371029B029A9B790D064CBF63F07F038B
:1091A00003F07F039371029B02999A79124B22F08C
:1091B00002021B888A71104A01331380F8F7BBBB87
:1091C000029B029A9B7923F0040393710EE50B4BEB
:1091D000029A1B681179094852790733036042EA01
:1091E0000123F3E6029B029A9B7923F00403937117
:1091F000B9E700BF4EBD0120AABD0120B0BD0120CE
:1092000044A5012000BD0120ACBD01209E4B1B7870
:10921000002B00F017819D4B9D4A1B881168029A14
:109220009C48947A01339BB29A0B133150F8220078
:10923000964A1380C3F30D02954B1960029B825628
:10924000DB7A43EA042313449BB262E7924B1B7818
:10925000002B00F0D8808D4B8D4A1B881168029A34
:109260008C48147A01339BB29A0B133150F82200C8
:10927000864A1380C3F30D02854B1960029B825608
:109280005B7A43EA042313449BB29A0BC3F30D01A8
:10929000804B53F82230029A585CD4797F4900F011
:1092A0000F0204F00F03134413F0100F8B7914BF57
:1092B00043F0100323F010038B7180EA040322189B
:1092C000DB0995B240F0988084EA0203180640F169
:1092D0009380029B02999B7943F004038B71029B5C
:1092E000DA716E4A9379E9054CBF43F0010323F02C
:1092F00001039371029B029A9B79029915F0FF0F6B
:1093000014BF23F0400343F040039371029B9B7909
:109310002A06029A4CBF63F07F0303F07F03937128
:10932000029B9A79594B22F002021B888A71574A94
:1093300001331380F8F7FFBA574B1B78002B34D05A
:10934000524B534A1B881168029A5248147A0133CF
:109350009BB29A0B133150F822004C4A1380C3F38E
:109360000D024B4B1960029B82565B7A43EA042341
:1093700013449BB29A0BC3F30D01464B53F82230B2
:10938000424A5B5C12880299CB71531C3F4A13809E
:10939000F8F7D1BA3E4B029A1B6811793C485279D2
:1093A0000733036042EA0123E2E4374B1B78002BCA
:1093B00053D0364B364A1B881168029A3548947A46
:1093C00001339BB29A0B133150F822002F4A1380BD
:1093D000C3F30D022E4B1960029B8256DB7A43EADF
:1093E000042313449BB2C5E7029B029A9B7923F0A6
:1093F00004039371FFF7EABA029B02999B7923F069
:1094000004038B716BE7204B1B78002B30D01F4B74
:109410001F4A1B881168029A1E48947A01339BB236
:109420009A0B133150F82200184A1380C3F30D022F
:10943000174B1960029B8256DB7A43EA04231344DC
:109440009BB222E7124B029A1B681179104852799D
:109450000733036042EA01235BE60D4B029A1B6867
:1094600011790B4852790733036042EA012381E7FF
:10947000074B029A1B68117905485279073303603C
:1094800042EA012301E700BFACBD0120AABD0120D3
:10949000B0BD012044A501204EBD012000BD01202A
:1094A000744B744A1B6804331360FEF71FBC714B86
:1094B000704A1B6804331360FFF774BB6D4B6D4A31
:1094C0001B6804331360FFF75BBA6B4B1B78002BF0
:1094D0002CD0684B67491A68031FDBB20832012B96
:1094E0000A601FD90A220AE5634B1B782BB3634B32
:1094F000604A1B881168029A6148947A01339BB2D2
:109500009A0B133150F822005C4A1380C3F30D020A
:10951000584B1960029B8256DB7A43EA04231344BA
:109520009BB216E5831DD8B20A22E8E4514B514A9A
:109530001B68043313600422E1E44E4B029A1B685B
:1095400011794C4852790733036042EA012300E560
:109550000A9B4C481B680D22DB6801210BF07CFD47
:10956000F7F7D6B801340A2003F046F80A2C77F44E
:109570005EA8454B0A931B68444A4549D8680BF0DE
:109580000BFD0A9B43481B681B22DB6801210BF083
:1095900063FDF7F7BDB80A9B3F481B681122DB68E3
:1095A00001210BF059FDF7F7B3B80A9B3B481B6844
:1095B0003622DB6801210BF04FFDF7F7A9B80A9BB3
:1095C00037481B681B22DB6801210BF045FDF7F7CC
:1095D0009FB80A9B33481B680E22DB6801210BF001
:1095E0003BFDF7F795B8284B2F480A9321460CF01E
:1095F00033F801233B60F7F78BB82C4803F0DAF817
:1096000011ADF7F707B8C9003231A3FB0113C3F35B
:10961000421343EA0201F6F702BF254BEB60312308
:109620008DF861708DF862708DF863808DF8603010
:10963000F6F71CBF59685A685B684C024CBF1D495D
:109640001D4902F03F02B1FBF2F21C494968C3F325
:10965000881302FB03F2C1F30141194B01314900A8
:10966000B2FBF1F21A60F6F709BE154B114A1A6007
:10967000F6F704BEB0BD0120ACBD0120AABD01209B
:1096800044A501202C5E010828010020B45D0108DA
:10969000BC5D0108105E0108FC5D0108C45D0108A5
:1096A0007C60010898600108905D01085C5D01081C
:1096B0000006FA0500127A000024F4000038024087
:1096C000700000200B6009F001FB2B6B6C4C43F029
:1096D00002032B632B6B43F002032B63204618A974
:1096E0004FF480758DF864808DF866808DF8676022
:1096F0008DF86560189503F0CBF84FF400732046A1
:1097000018A918938DF866608DF864608DF867600D
:109710008DF8656003F0BCF823699A0503D465836E
:10972000404602F069FF4FF48076554C37460925D4
:109730000120278302F060FF23699B054FF00100A1
:1097400004D4668302F058FF013DF1D14C4C4D4DDD
:109750004FF480762683012002F04EFF23692B6BA5
:1097600043F002032B632B6B43F002032B632B6A42
:1097700043F400132B622B6A23F400132B62636AF9
:1097800023F00F036362636A43F004036362636A56
:1097900023F0F0036362636A43F0400363620222D2
:1097A0000123204618A98DF864208DF865208DF8D6
:1097B00066308DF86730189603F06AF84FF400733E
:1097C00018A92046189303F063F8296C2E4B2F4AF2
:1097D00041F4001129641A6006F062FCF6F7FDBE40
:1097E00018A803F0A9F8F6F754BEFB22022118A826
:1097F0008DF861308DF8602009F012FB002876F4B6
:10980000FAAEFA23012118A88DF8603009F008FBA0
:10981000002876F4F0AE4FF4003009F063FA002827
:10982000F9D11B4C1B4823889BB243F480732380DF
:1098300009F0E0FA002836F4DEAEA52323821648AC
:1098400009F0D8FA002836F4D6AE238B23889BB2D1
:1098500043F4806318AD238027462E4601240F4829
:1098600009F0C8FA631C0A4A002836F4C4AE398AE3
:1098700006F8011B062B00F06B871C46EFE700BFC4
:10988000000402400038024064220020801A0600D2
:1098900000540040010000100200001040000010C1
:1098A000C34FDFF83CB3DFF83CA30A234FF00008B6
:1098B000B9463E460293DAF83030BE4C43F001031D
:1098C000CAF830304FF4C053032218A92046189329
:1098D00002238DF865208DF864308DF866808DF850
:1098E000678002F0D5FF4FF480524FF4006363832A
:1098F0006420628302F080FE636A23F47043636233
:10990000636A43F420436362636A23F470236362EF
:10991000636A43F420236362DAF8443043F48043FB
:10992000CAF84430DAF8343043F08003CAF83430EF
:1099300009F0DCFAA04BCBF87C30A04BCBF88030A0
:10994000C7F81083002202F1C40307EB830302F17E
:10995000D401C3F80480BB1801320F2A47F82180D4
:1099600083F88C83EFD108230122A6F8B233337039
:109970004023B270F272B38004224FF4A07372706D
:10998000F38002228E4B32728E4A336103F54073AC
:10999000B261736520322033F261B3652032203327
:1099A0003262F3652032203372623366A2F5AC6214
:1099B000A3F5E4637261C6F8CC3002F58072E0333F
:1099C000C6F89020C6F8943040324033C6F898204C
:1099D000C6F89C3040324033C6F8A020C6F8A43008
:1099E000403240334FF0A041C6F8A820C6F8AC3052
:1099F00002F5246203F5D1534FF00000C6F8D020E1
:109A0000C6F8D43002F5005203F50053F070F1604F
:109A1000C6F8D820C6F8DC308A6803F50053C6F8CB
:109A2000E43022F001038B60CA68674BC6F8E83067
:109A300042F04003CB60654A654BC6F8EC204FF01E
:109A40005021C6F8E010C6F80C3104F015F9737A0D
:109A5000FA68002B0CBF4FF434134FF47413936364
:109A6000142005F083F9FB78012B07D1F9688B6886
:109A7000052262F3440343F020038B60FA68D36845
:109A80006FF39E7343F00053D360322005F06EF9FC
:109A9000D7F80C3100241C603B7A012B254601F0DD
:109AA0003981D9F814100B68012262F301030B60AD
:109AB0003F4805F073F97A6913686FF38203136006
:109AC000FB7A012B0FD18021E023D9F80C2061F320
:109AD0000F0463F30F05C0F26004C0F26005516229
:109AE0009462C2F80051CDF85880169BF96843F093
:109AF00020031693169B102262F38A131693169B6B
:109B00000B610B69334A1693169B9C0603D50B69B0
:109B10001693013AF8D104F0A5F8CDF85080149BC3
:109B2000FA682C4943F010031493149B13611369D2
:109B30001493149BD80603D5136914930139F8D1F3
:109B400004F090F83B786BB12333234A09EB830090
:109B50004FF0FF3152F8043F996013688242C3F816
:109B60000C80F7D1D7F8CC201C4C13686FF382031C
:109B70006FF341036FF3C3036FF34513D9045CBF65
:109B800043F480531360C82005F0F0F8FA68F878C1
:109B9000002393614FF0FF3353615360F96800284D
:109BA00014BF002310236FF080424A611CE000BF05
:109BB000ECBD012000000240000000201400002045
:109BC0000008005000090050007000500080005054
:109BD000000E0050400D030078BE012000080080F8
:109BE00098C301200038024043F00C538C618A690D
:109BF00043F4001343F0080313438B618B6843F075
:109C000001038B60DBF880301B689847A34BA449A5
:109C1000D96001224321032318A88DF861208DF813
:109C200063208DF860108DF8623002F085FE3220DE
:109C300002F0E2FC942403F08BFC9A4B1B78012B7E
:109C40004FF0050037F41DA902F0D6FC013CF2D11B
:109C5000944B1B78012B37F414A9029B013B029310
:109C60007FF429AEF7F70DB9029A8F4B117852782D
:109C70001B6842EA01228C490733B2F5804F0B6022
:109C80000ED3B2F5B64F02D2884901230B70930B65
:109C9000C2F30D01864A52F82320029BDB7953540C
:109CA000844B844A1B8801331380F7F744BE8249F2
:109CB000824809F05DFE0446002800F0CE80804B0B
:109CC000029A1B78D07921465D000BF049F8029B7F
:109CD000214698790BF044F8029B214658780BF006
:109CE0003FF8029B214618780BF03AF8029B214678
:109CF00058790BF035F8029B214618790BF030F8B3
:109D0000214600200BF02CF8214600200BF028F80B
:109D10006C4B2046198808F069FE6B4B2146187879
:109D20000BF01EF8214600200BF01AF8214605F032
:109D3000FE000BF015F8029B2146D8780BF010F8C6
:109D4000029B214698780BF00BF8604B214658781F
:109D50000BF006F85D4B214618780BF001F85B4BD1
:109D60002146D8780AF0FCFF584B214698780AF033
:109D7000F7FF564B214658790AF0F2FF534B214624
:109D800018790AF0EDFF514B2146D8790AF0E8FF27
:109D90004E4B214698790AF0E3FF029B2146D87A80
:109DA0000AF0DEFF029B2146987A0AF0D9FF029B57
:109DB0002146587A0AF0D4FF029B2146187A0AF00D
:109DC000CFFF434B214618780AF0CAFF414B21468A
:109DD00018780AF0C5FF404B214618780AF0C0FFFA
:109DE0003621204608F002FE324B2046198808F042
:109DF000FDFD0025012608E0022B33D00AF0B0FF5C
:109E0000342E1AD0731C9EB2013521460020ABB20D
:109E1000002DF1D1314B1B68B3F5804F0CBF0346C9
:109E2000042326E0052F37F615AD2D4B01373846B4
:109E3000196807F023FDF7F70DBD284B1B68B3F534
:109E4000804F1DD00025E9B22046013508F096FD6F
:109E5000082DF8D1204609F065FB224A0023136043
:109E6000F7F7D9B81D4B1B68B3F5804F06D01E4BD2
:109E70001B78184621460AF073FFC3E70023F8E772
:109E80002046012108F07AFD2046022108F076FDE7
:109E90000521204608F072FDDCE700BF00ED00E080
:109EA0000006FA05A8BD0120B0BD0120A5000020D4
:109EB00044A50120AABD0120D86101085C01002051
:109EC00054A501204EBC012019070020E0BC012050
:109ED000DCBC01201C1F002050BC0120F0BC012074
:109EE000EC030020201F002070A50120029BA04A47
:109EF0001C7A587A9978DB78126843EA012A029B27
:109F000040EA042893F807B0002A7ED1029B029A07
:109F10009B7923F001039371964B974C1888431C4F
:109F2000820B99B28B0B54F82240934A52F823507B
:109F3000C0F30D03C1F30D02E45C8E4B1980AB5CE2
:109F40008E4944EA03230B808A4B821C1A80F7F760
:109F500056B8029B1E7A5D7A9C78D878884B99799E
:109F6000DA79884B1B6812F1000845EA062B40EAB3
:109F7000042A01F0010918BF4FF00108002BC5D0D9
:109F8000814B824A1B6814787F4E002B00F0AB8215
:109F9000012C00F0B682022CB8D100247A4B1A684A
:109FA0001D465368013B002B5360C0F28A82116842
:109FB0004B1C13600A78A2F11003222B00F26E8270
:109FC000DFE813F06B01610153016C0201016C02C7
:109FD0006C026C026C026C026C026C026C026C0211
:109FE0006C026C022902EB018B016C026C026C02A8
:109FF0006C026C026C026C026C026C026C026C02F1
:10A000006C026C02E8006C02C700614B604D1B687B
:10A01000002B00F000835E4B19680A9B18688B6860
:10A02000013B002B8B60C0F2ED8208681023421CBC
:10A030000A600370564B1C680A9B1A68A3680AF1F1
:10A040000205013B4FEA2529002BA3605FFA89F73F
:10A05000EEB2C0F2CD822168E8234A1C22600B7068
:10A06000A3680A9A013B002B1268A360C0F2B68273
:10A07000216803234A1C22600B70A3680A9A013BE3
:10A08000002B1268A360C0F289822268531C2360EF
:10A090001570A3680A9A013B002B1268A360C0F2F6
:10A0A00067822268531C236082F80090A3680A9A92
:10A0B000013BBBF1FF0F0CBFFF260026002B1268EF
:10A0C000A360C0F261822268531C23601670BAF14B
:10A0D000000F1DD008EB0A039FB227494FEA9833BF
:10A0E000C8F30D0251F82330A1689D5C0A9B1868E3
:10A0F0004B1E002B86EA0506A36020DB2268531C5A
:10A100002360157008F101031FFA83F84745E4D175
:10A11000A3680A9A013B002B1068A360C0F24A8230
:10A120002268531C23601670194B186809F0B4FAA2
:10A13000029B029A9B7943F001039371ECE6A269BA
:10A1400093422946224601DB0A2DD7D10AF0C8FCEA
:10A15000D8E70D4B18681D4604F0E4FE04460028BD
:10A160007FF41BAF286809F0DDF92C60CEE600BF54
:10A17000F80600204EBC012044A50120AABD012004
:10A18000E0BC01201407002060020020FC06002033
:10A19000C0B70120B34B1C680DF14201204604F00A
:10A1A000A7FE00283FF4F9AE9DF84220531E18A9DF
:10A1B00020468DF84230002A3FF4EFAE04F098FEBE
:10A1C0000028F1D1E9E6A74B1D6810A9284604F044
:10A1D0005FFE00283FF4E1AE0DF14201284604F095
:10A1E00057FE00283FF4D9AE0DF13E01284604F099
:10A1F0007FFE00283FF4D1AE18A9284604F048FE9F
:10A2000000283FF4CAAE0DF13D01284604F070FE6F
:10A2100000283FF4C2AE0DF13D0128469DF83D6097
:10A2200004F066FED8B19DF83D300DF13D012846A1
:10A230001C0204F05DFE00283FF4AFAE9DF83D30F7
:10A2400044EA03431E430AD000240DF13F0128468F
:10A2500004F04EFE631C9CB208B1A642F5D80A9BDE
:10A260001B68986809F018FA97E67E4B1C6818A9D5
:10A27000204604F00DFE00283FF48FAE204618A9BA
:10A2800004F006FE89E6774B1C6818A9204604F006
:10A29000FFFD034658BB1C4680E6724B1C6818A99C
:10A2A000204604F0F5FD03460028F4D00DF14201EC
:10A2B000204604F0EDFD03460028ECD0BDF8423006
:10A2C000CDF80080204601934B465246594604F093
:10A2D0005BFE012804467FF461AE029B02999B79E4
:10A2E00043F0010200238A718B70CB7014E618A929
:10A2F000204604F0CDFD03460028CCD018A9204606
:10A3000004F0C6FD03460028C5D018A9204604F075
:10A31000BFFD03460028BED018A9204604F0B8FDB2
:10A3200003460028B7D018A9204604F0B1FD034623
:10A330000028B0D00DF14201204604F0D9FD0346BB
:10A340000028A8D018A9204604F0A2FD0346002842
:10A35000A1D06168013900296160C0F2948022684F
:10A36000531C23601678013900296160C0F2808097
:10A370002268531C236015784B1E002B636068DB3A
:10A380002268531C23601278CDF8008046EA05232A
:10A3900043EA02430193204696E7324B1F680DF1D2
:10A3A0004201384604F0A4FD034600283FF473AF91
:10A3B0009DF842102C480BF04FF99DF84230E3B164
:10A3C000002618A9384604F093FD034600283FF400
:10A3D00062AF0A9B9DF8605018688468A368013BCF
:10A3E000002BA36026DB2268531C23601570721CAF
:10A3F0009DF84230D6B2B342E3D80A9B19688A6806
:10A400009368013B002B93601EDB10680A23411CFC
:10A410001160037061E7134B18A9186804F038FD48
:10A42000034600283FF437AFBDF860100F480BF02B
:10A4300013F952E7A26993422946224601DB0A2D0D
:10A44000D1D10AF04DFBD2E708460A210AF048FBB9
:10A4500043E70A9B2146186809F094FF0246013041
:10A4600092D19AE5600200209C6101089061010888
:10A470000A9B2146186809F085FF471C05463FF4F2
:10A480008CAD616878E70A9B2146186809F07AFF6D
:10A49000431C06463FF481AD616864E70A9B9C4912
:10A4A0001B68D8680AF078FD0A9B1B68D86809F019
:10A4B000F3F8984B186809F035F8964A00231360B2
:10A4C00024E50A9B1146186809F05CFF411C02460E
:10A4D0007FF471AD286809F025F800232B60002C6B
:10A4E0003FF414ADF9E68C498C4809F041FA054671
:10A4F000306000283FF40AAD022C18D0012C7FF404
:10A5000005AD844B1D6818A9284604F0C1FC00283D
:10A510003FF4FCACBDF860400194CDF800804B46A0
:10A5200052465946284604F02FFD0446D7E718AC9A
:10A530002146284604F0DCFC013400283FF4E6AC58
:10A540000DF16A039C42F3D10722754918A80AF05D
:10A5500091FD002839D19DF867301A2B3FF41DADCD
:10A560000A9A70491268D0681A460AF015FDCDE4BF
:10A57000A1698B4202DB0A2F7FF493AD3946104666
:10A5800022460AF0ADFA91E5A1698B42BFF69BAD78
:10A590001046314622460AF0A3FA98E5A1698B429B
:10A5A00002DB0A2E7FF471AD3146104622460AF0D6
:10A5B00097FA6EE5A269934202DB0A2E7FF4B0ADF2
:10A5C000224631460AF08CFAAEE50A9B56481B68D3
:10A5D0001622DB6801210AF03FFD97E4A1698B4256
:10A5E000BFF646AD1046032122460AF079FA44E54B
:10A5F000A1698B42BFF62FAD1046E82122460AF032
:10A600006FFA2DE58A699342BFF60FAD0A46102115
:10A610000AF066FA0EE54549454809F0A9F90446ED
:10A62000286000283FF472AC0346072201213C4811
:10A630000AF012FD21461A200AF092FB2146012061
:10A640000AF08EFB214610200AF08AFBE3E43B214E
:10A6500018A80BF0CBF8002836F4ACAA0470F6F773
:10A66000A9BA03F80119C34276F4ADAAF6F7B9BA4C
:10A67000204630490BF09CF8002876F488AA2E4A30
:10A6800082F88000F6F783BA21463F222B480BF070
:10A69000D5F8294B83F87F60F6F779BA21463F2237
:10A6A00025480BF0CBF8244B83F83F60F6F76FBAE0
:10A6B000234918A80BF07CF80646002800F01B81FF
:10A6C000204918A80BF074F8002840F0F7801E49C4
:10A6D00020460BF06DF848B9174B174AD3F8C43031
:10A6E00043F00103C2F8C430F6F751BA17492046C7
:10A6F0000BF05EF8002840F0D0800F4B0E4AD3F8E4
:10A70000C43043F00203C2F8C430F6F740BA00BFC9
:10A71000B06101086002002014610108241F0020BC
:10A72000486101086861010850610108D8610108A9
:10A7300064020020DC60010874A50120B4A501209A
:10A74000E0600108EC600108F8600108FC600108A5
:10A75000138823F480631B041B0C138013889BB2A3
:10A7600043F4007313804FF4003008F0BBFA002864
:10A77000F9D1B34808F03EFB002835F43CAFB14BAB
:10A7800018A91A8A0A551A8892B242F480621A806D
:10A7900012A806220AF06EFC002840F0B680AA4EED
:10A7A00001233360A74CA948A588A94BDFF804937F
:10A7B000A84FA949A94ADFF80083ADB245F4006566
:10A7C000A580046BA64D44F400140463186820F0BF
:10A7D000010018601868002420F001004FF0210AE1
:10A7E00018601C605C609C60DC601C61C3F814A095
:10A7F000C9F80C70186801400A431A605A699949EF
:10A800000D9122F0070242F001025A615C60C3F828
:10A810000880DD601A6811AD42F010021A6001274D
:10A82000112328462B706C70AC70EF7002F084F826
:10A830008D4B8E491A6822F001021A601A6822F0C4
:10A8400001021A603D221C605C609C60DC601C613F
:10A85000C3F814A0C9F8082018687F4A024042F0E3
:10A86000007242F482321A605A6922F007023A43B7
:10A870005A615C60C3F80880D9601A6842F010021F
:10A880001A6028460B232B706C70AC70EF7002F0CE
:10A8900053F80D9B1F60F5F7B6BE204674490AF0C9
:10A8A00087FF002876F473A9724B724AD3F8C4303C
:10A8B00043F00403C2F8C430F6F769B96E4918A82A
:10A8C0000AF076FF002841D06C4918A80AF070FF02
:10A8D000002876F45CA9204608F0B4FD684B654A70
:10A8E0000340002B03DA013B63F00103013382F8DC
:10A8F000C830F6F74CB921463F2262480AF09EFF65
:10A900005C4B83F8C060F6F742B9062218A914A878
:10A910000AF0B0FB28B1062218A916A80AF0AAFB73
:10A9200018B9494E022333603CE7574801F042FF13
:10A930000DF1660415F8011B544801F019FFAC42F3
:10A94000F8D1534801F036FFF5F755BE204608F020
:10A9500079FD504B474A0340002B03DA013B63F07B
:10A960000303013382F8C930F6F711B9012007F06B
:10A97000C9F800283AD0014647480AF04FFF474A35
:10A9800001231360012004F027FA454BFF201968CA
:10A9900006F074FF0D9B43491A6800230B600AB14F
:10A9A00006F044FF404A01231370F6F72FBB314BEA
:10A9B00093F88030B3B1002388F88030384B0620FC
:10A9C000196806F05BFFF6F745BF354B1C681D465E
:10A9D0009CB1364B00241C60354B1C7004F04CFAC3
:10A9E0002C60CFE7012388F88030E7E72C4B052067
:10A9F000196806F043FFF6F72DBF204607F082F8EE
:10AA00000546B0B1294B1C60294B1C7004F034FA88
:10AA100028460AF00BFF0428244C06D92946FF22B9
:10AA200023480AF00BFF012323601D4A0123136012
:10AA3000A8E7DAF80010042006F020FFF6F70ABFB6
:10AA4000400000100054004044B80120003802408B
:10AA5000A060024000003D203F801CF04004010245
:10AA60002420002018B801201060024008070020B0
:10AA70000061010874A5012004610108106101084A
:10AA800001000080F5A501200C5D0108245D01088E
:10AA90004C710108030000805C010020201F002091
:10AAA000EC03002040B8012074000020F8060020CC
:10AAB000640200200060024010540040002007F0B3
:10AAC00015F90646002848D00AF0B0FE04287FF6A3
:10AAD00059AF9E4B9E4A9E4F126800241C609D4BAE
:10AAE0001C709D4B051F1C601AB1104608F01AFD22
:10AAF0003C607419204699490AF05AFE00283FD05C
:10AB0000974920460AF054FE70B3204695490AF052
:10AB10004FFE00287FF436AF934C8E480323FF226C
:10AB2000314623700AF08AFE8B4A0123136029E71D
:10AB3000012007F0DBF8044600283ED00AF076FE3C
:10AB400004287FF61FAF2146802288480AF076FE4F
:10AB500007F05AFF03F06CFA14E7854B03201968DD
:10AB600006F08CFEF6F776BE7F4C7A480223FF2271
:10AB7000314623700AF062FE744A0123136001E734
:10AB8000794B744801243146FF221C700AF056FEAE
:10AB90006E4B1C60F6E6774B764A1B780133DBB2CE
:10ABA000042B137004BF002389F80030704B002081
:10ABB000196806F063FEF6F74DBE6D4B022019686A
:10ABC00006F05CFEF6F746BE6B4B1B781BB96B4B71
:10ABD0001B78002B6ED06A4B694A1B6808331360E0
:10ABE000029B684A197801F00F03013313F0100F2C
:10ABF000937914BF43F0100323F010039371CB0932
:10AC000001F1010040F09B8081EA0003190640F148
:10AC10009680029B029A9B7943F004039371029BF6
:10AC2000029A9979187001F0FD03937110F0FF0FEB
:10AC3000544A14BF21F0420343F040039371029B36
:10AC40009B790206029A4CBF63F07F0303F07F03F7
:10AC500093714D4B4C4A1B8801331380F6F76BBE42
:10AC6000474B47491A68484B04321B880A60464ADA
:10AC700001331380F6F75FBE414B414A1B68043332
:10AC80001360FBF791BD029B02981A785B783C49F0
:10AC900043EA022301339BB209683B4A43701B0A13
:10ACA0000370374B128806311960374B01321A8016
:10ACB000F6F741BE324B324A1B68043313608FE70C
:10ACC000314B32481C882E4B1D68631C9BB29A0B7B
:10ACD000A11C50F822002C4A1380C3F30D0205F189
:10ACE0000A03274D89B22B60855C284A8B0B52F8EA
:10ACF0002300254B1980C1F30D032349C35CE21CDB
:10AD000005EB03230A809BB202991A0A4B700A7062
:10AD1000F6F711BED9F81420136864F30103136029
:10AD2000FEF7C6BE1A4B1B481A8821460AF094FC4F
:10AD30000A9B1B68986808F0AFFCF6F7FCBD029B05
:10AD4000029A9B7923F00403937168E714070020AB
:10AD500060020020241F002000070020DC610108A1
:10AD6000E4610108EC610108FC06002054BC0120EC
:10AD7000EC030020C40000204EBD0120ACBD01202A
:10AD8000B0BD012000BD0120AABD012044A50120C5
:10AD9000F4BC0120186201088E4B1B783BB98E4B26
:10ADA0001B7823B98D4B8D4A1B68073313608C4B7E
:10ADB0008C491C88631C9BB29A0BC3F30D0051F89D
:10ADC0002210874A13800B5C0299CB70844BA21C23
:10ADD0001A80F6F7B0BD7F4B1B783BB97E4B1B78D2
:10ADE00023B97E4B7D4A1B68073313607C4B7D493A
:10ADF0001C88631C9BB29A0BC3F30D0051F8221000
:10AE0000774A13800B5C02994B70754BA21C1A8019
:10AE1000F6F791BD6F4B1B781BB96F4B1B78002B5E
:10AE200043D06E4B6D4A1B6808331360029B6E491A
:10AE3000587800F00F035A1E431E9CB28B79D5063A
:10AE40004CBF43F0100323F010038B71C30932D0C1
:10AE500080EA040319062ED5029B029A9B7943F0DF
:10AE600004039371604A029B02995C70937914F019
:10AE7000FF0F14BF23F0400343F040039371029B84
:10AE80009B792206029A4CBF63F07F0303F07F0395
:10AE90009371029B9A79524B42F002021B888A718D
:10AEA0004F4A01331380F6F746BD4C4B4B4A1B68A3
:10AEB00004331360BAE7029B029A9B7923F00403E0
:10AEC0009371CFE7434B1B781BB9434B1B78002B87
:10AED00059D0424B414A1B6808331360029B424AD7
:10AEE000597801F00F03013313F0100F937914BF59
:10AEF00043F0100323F010039371CB0901F101001B
:10AF000047D181EA00031F0643D5029B029A9B7931
:10AF100043F004039371029B029A9979587001F0EF
:10AF2000FD03937110F0FF0F2F4A14BF21F042036D
:10AF300043F040039371029B029A9B7906064CBF33
:10AF400063F07F0303F07F039371254B244A1B8832
:10AF500001331380F6F7EFBC029B02981A785B78F6
:10AF60001E4943EA0223013B9BB209681C4A437015
:10AF70001B0A0370194B128806311960184B0132F5
:10AF80001A80F6F7D8BC154B144A1B6804331360BB
:10AF9000A4E7029B029A9B7923F004039371BAE71A
:10AFA000029B0E491A785B780C680D4943EA02232C
:10AFB00008889A0BC3F30D010A4B53F82220E31DB6
:10AFC000064C2360535C029AD371054A431C1380DC
:10AFD000F6F7B1BC4EBD0120ACBD0120B0BD0120D3
:10AFE000AABD012044A5012000BD0120029BA64A64
:10AFF00018785978A54B1B7841EA0024002B67D0BC
:10B00000A348117A537A056843EA0123C3F30B007E
:10B0100005F10F011D19C4F30B03034413F4805F02
:10B0200093799B4814BF43F0100323F010039371EE
:10B03000029A01602B0A55721372029B02989A7948
:10B04000914902F0FD038371E80354BF22F003032A
:10B0500043F001038B718F4B8E4A1B8801331380A1
:10B06000F6F769BC8A4B029C19688A4B1A88029BC6
:10B07000D879894BDB79E3710B1D85490B60854BD2
:10B08000A17901321A80844B834A9B79D0719171E6
:10B09000A371F6F750BC7E4B029A1B68D2797C48AC
:10B0A000794904331406036033D48B79520023F0BA
:10B0B0000103CA718B71029B02999A79754B22F038
:10B0C00012021B888A71734A01331380F6F733BC6E
:10B0D000724B1B7833B36E48917AD37A056843EA92
:10B0E0000123C3F30B0005F10F011D19C4F30B037A
:10B0F000034413F4805F9379654814BF43F0100351
:10B1000023F010039371029A01602B0AD572937297
:10B1100093E78879530043F0010240F00103CA71BC
:10B120008B71C8E75A4811795379056843EA0123BE
:10B13000C3F30B0005F10B011D19C4F30B0303440A
:10B1400013F4805F9379524814BF43F0100323F047
:10B1500010039371029A01602B0A557113716CE709
:10B16000029A4B4B9178D2781B6842EA01224849F7
:10B170000733B2F5804F0B600ED3B2F5B64F02D253
:10B18000474901230B70930BC2F30D01454A52F856
:10B190002320029BDB7953543E4B3E4A1B880133EC
:10B1A0001380F6F7C8BB3B4B3E481C88384B1D68E4
:10B1B000631C9BB29A0BA11C50F82200354A1380E5
:10B1C000C3F30D0205F10A03314D89B22B60855C92
:10B1D000344A8B0B52F823002E4B1980C1F30D0318
:10B1E0002C49C35CE21C05EB03230A809BB2029945
:10B1F0001A0ACB708A70F6F79EBB264B294918882D
:10B20000029B244D1C78431C9BB29A0B2B8051F857
:10B210002210C3F30D02831C8A56029899B2631E52
:10B220000A44DBB292B2037033B3194B2A801B6815
:10B23000174A0D331360F6F77EBB154B029A1B6855
:10B24000D2791348104904330360D3072CD5887989
:10B25000530863F07F0240F00103CA718B71029BB7
:10B2600002999A790B4B22F012021B888A71094AC3
:10B2700001331380F6F75FBB054B054A1B68298035
:10B2800008331360F6F757BB00BD01204EBD012007
:10B29000B0BD0120AABD0120E0BC0120ACBD012051
:10B2A000A500002044A501208B79520823F001035A
:10B2B000CA718B71D3E7984B1B781BB9974B1B78DE
:10B2C000002B59D0964B964A1B6808331360029B9B
:10B2D000944A997801F00F03013313F0100F93791A
:10B2E00014BF43F0100323F010039371CB0901F155
:10B2F00001004ED181EA00031F064AD5029B029A43
:10B300009B7943F004039371029B029A9979987098
:10B3100001F0FD03937110F0FF0F824A14BF21F07A
:10B32000420343F040039371029B029A9B79060605
:10B330004CBF63F07F0303F07F0393717A4B7A4A2B
:10B340001B8801331380F6F7F6BA029B02989A78AD
:10B35000DB78734943EA022301339BB20968724ADE
:10B36000C3701B0A83706E4B1288063119606E4BD6
:10B3700001321A80F6F7DFBA694B694A1B68043359
:10B380001360A4E7664B664A1B6804331360FBF73F
:10B39000BDBA029B029A9B7923F004039371B3E731
:10B3A000614B624C19885C4B1D784B1C9AB28B1C0C
:10B3B00099B2930B880B54F823405B4B1A80C2F36D
:10B3C0000D035A4A52F82000E25C574B1980C1F332
:10B3D0000D03C35C02EB032398B2002D32D0504B17
:10B3E000029A1B68547A157A4D4A14331360B0F5EB
:10B3F000804F22D3B0F5B64F02D24D4A01231370CD
:10B40000830B4A4AC0F30D0152F8232045F6FE2370
:10B410009842545402DC464A01231370431C99138A
:10B42000C3F30D02414B53F821309D543E4B3E4A2D
:10B430001B8801331380F6F77EBA43F6FF739842F8
:10B44000F4D1E8E7354B1B78002B35D0344B029A0A
:10B450001B68D47A957A324A14331360C7E72E4BAF
:10B460001B78002B31D0304B30481A882C4B1D688C
:10B47000531C9BB2911C9A0B89B250F822402A4A65
:10B48000C3F30D00138005F10E03254D2B60235CE3
:10B4900026488A0B50F82220029843722248C1F3B2
:10B4A0000D030180D35C029A13721F4B1E4A1B8846
:10B4B00001331380F6F73FBA194B029A1B6854798F
:10B4C0001579174A1033136091E7144B1B78002B42
:10B4D00075D0154B15481A88114B1D68531C9BB22B
:10B4E000911C9A0B89B250F822400F4AC3F30D0009
:10B4F000138005F10E030A4D2B60235C0B488A0B69
:10B5000050F822200298C3720748C1F30D0301804E
:10B51000D35C029A9372C8E74EBD0120ACBD0120F6
:10B52000B0BD012000BD0120AABD012044A501201D
:10B53000A50000209F4B9F4C1888029B9E499D7937
:10B54000431C9BB29A0B238051F82210C3F30D03C6
:10B55000821CCB5692B2134469069BB252D4974ACE
:10B560002380126802F10C03944A1360F6F7E3B9E2
:10B57000924B029A1B6891799048914A0433036078
:10B58000D3798F4ACD0746BF5B0843F08000580847
:10B59000029BDB79DC074CBF41F0010321F0010382
:10B5A0009371029B02999A79824BC8711B8822F091
:10B5B00012028A717F4A01331380F6F7BCB97D4BC2
:10B5C0007D481A887D4B1D68531C9BB2911C9A0BB9
:10B5D00089B250F82240774AC3F30D00138005F179
:10B5E0000A03764D2B60235C73488A0B50F82220A7
:10B5F000029843716F48C1F30D030180D35C029A36
:10B60000137152E76D4B22801B686C4A073313603D
:10B61000F6F791B96B4B1B78002B00F0D780674B86
:10B62000664A1B68083313600820029B64491A5C51
:10B6300002F00F03013313F0100F8B7914BF43F0A6
:10B64000100323F010038B71029B1B5CD90902F1DC
:10B6500001045B4A43D163401B0640D5937943F014
:10B6600004039371029B56491C549A79029802F084
:10B67000FD0314F0FF0F837114BF22F0420343F067
:10B6800040038B71029B029A9B7927064CBF63F0A3
:10B690007F0303F07F039371464B464A1B880133B7
:10B6A0001380F6F748B9474B1B78002B00F09880C1
:10B6B000029B42491A7A5B7A0298096843EA02239C
:10B6C00001339AB2130A03723C4B42720A31196079
:10B6D000384B384A1B8801331380F6F72CB9029B8C
:10B6E000029A9B7923F004039371BBE7354B1B78D7
:10B6F000002B53D0314B314A1B68083313600824A8
:10B70000029B2F481A5D02F00F03591E531E9DB273
:10B7100083792B4ACE064CBF43F0100323F010036D
:10B720008371029B1B5DD90931D06B4019062ED560
:10B73000937943F004039371029B214A1D55937939
:10B74000029915F0FF0F14BF23F0400343F04003AC
:10B750009371029B9B792A06029A4CBF63F07F0388
:10B7600003F07F039371029B9A79124B42F002021D
:10B770001B888A710F4A01331380F6F7DCB8029BED
:10B7800002999B7923F004038B71FAF7B4BF029BF3
:10B79000029A9B7923F004039371CDE70A4B1B783F
:10B7A000002B31D0054B054A1B68083313600A246F
:10B7B000A6E700BFAABD012044A50120B0BD01201D
:10B7C00000BD01204EBD0120ACBD0120A14B1B7866
:10B7D0000BB3A14BA04A1B68083313600A2024E76F
:10B7E0009C4B1B78F3B1029B9B499A7ADB7A0298B7
:10B7F000096843EA022301339AB2130A8372964B13
:10B80000C2720A31196063E7934B934A1B68043391
:10B810001360042474E7904B8F4A1B680433136051
:10B82000042002E7029B8C491A795B790298096827
:10B8300043EA022301339AB2130A0371864B427121
:10B840000631196044E7029B83499A78DB780C68DB
:10B85000824943EA022308889A0BC3F30D01804B07
:10B8600053F82220E31D7C4C2360535C029AD37171
:10B870007A4A431C1380F6F75EB8029B794A98789F
:10B88000D978794B1B7841EA0024002B6FD072489D
:10B89000117A537A056843EA0123C3F30B0005F1DB
:10B8A0000F011D19C4F30B03034413F4805F937954
:10B8B000694814BF43F0100323F010039371029AF8
:10B8C00001602B0A55721372029B02989A7965499E
:10B8D00002F0FD03ED03837154BF22F0030343F034
:10B8E00001038B715D4B5D4A1B8801331380F6F7B2
:10B8F00022B85A4B5A4C1888574B1968431C9BB2B4
:10B900009A0B0C3154F82220544C2380524CC3F330
:10B910000D032160D256831C1344504A1380F6F75E
:10B920000AB84D4B029A02991B688979D2794A4824
:10B930000433CF0703604FEA4203029A48BF43F043
:10B940000103D371DE05474A4CBF41F0010321F0EA
:10B9500001039371029B02999A79404B22F01202E3
:10B960001B888A713D4A01331380F5F7E4BF394BD8
:10B970001B78002B00F0E9803748917AD37A05686C
:10B9800043EA0123C3F30B0005F10F011D19C4F3B2
:10B990000B03034413F4805F93792F4814BF43F0E3
:10B9A000100323F010039371029A01602B0AD572E1
:10B9B000937289E72C4B1B781BB9264B1B78002B05
:10B9C00042D0254B244A1B6808331360029B254A4A
:10B9D000D97801F00F03013313F0100F937914BFDE
:10B9E00043F0100323F010039371CB0901F1010020
:10B9F0003CD181EA00031C0638D5029B029A9B7950
:10BA000043F004039371029B029A9979D87001F074
:10BA1000FD03937110F0FF0F124A14BF21F042038F
:10BA200043F040039371029B029A9B7901064CBF3D
:10BA300063F07F0303F07F039371084B074A1B8871
:10BA400001331380F5F777BF034B034A1B680433B8
:10BA50001360BBE7ACBD0120B0BD0120AABD012031
:10BA600044A5012000BD01204EBD0120029B029A89
:10BA70009B7923F004039371C5E7464B1B781BB9F0
:10BA8000454B1B78002B5AD0444B444A1B68083363
:10BA90001360029B4249D87800F00F035A1E431EE0
:10BAA0009CB28B79D2064CBF43F0100323F01003F5
:10BAB0008B71C30967D080EA04031F0663D5029B1C
:10BAC000029A9B7943F004039371354A029B0299D1
:10BAD000DC70937914F0FF0F14BF23F0400343F0A0
:10BAE00040039371029B029A9B7926064CBF63F038
:10BAF0007F0303F07F039371029B9A79294B42F0F5
:10BB000002021B888A71274A01331380F5F713BF9D
:10BB1000029B02989A78DB78204943EA0223013B92
:10BB20009BB209681F4AC3701B0A83701B4B1288A3
:10BB3000063119601B4B01321A80F5F7FCBE174B1A
:10BB4000164A1B6804331360A3E71448117953792C
:10BB5000056843EA0123C3F30B0005F10B011D192E
:10BB6000C4F30B03034413F4805F93790B4814BFB1
:10BB700043F0100323F010039371029A01602B0A23
:10BB800055711371A0E6029B029A9B7923F004037E
:10BB900093719AE74EBD0120ACBD0120B0BD0120DC
:10BBA00000BD0120AABD0120016809B310B40C78C2
:10BBB000202C09D93A2C16D00A4601E03A2B07D09E
:10BBC00012F8013F202BF9D800205DF8044B704794
:10BBD00001318A4207D1302C05D1013202605DF873
:10BBE000044B002070474FF0FF305DF8044B704766
:10BBF0004FF0FF30704700BF2DE9F04107468846FF
:10BC0000066861BBF5681DB3B3699D4228BF012575
:10BC100033690BB3B3692C4606E0012815D0013017
:10BC200058D0AC4218D0B36901349C4202D3012DE4
:10BC300012D902242146386806F0DAF90028ECD13E
:10BC4000012C02D9B3699C422CD30120BDE8F081BC
:10BC500033690125002BDDD10020BDE8F08130469D
:10BC600006F0C6F90128F0D9421C33D0B3699842D6
:10BC700043D33269002AEFD008F10104A34298BFF0
:10BC800002242146386806F0B3F90128DDD0431CB0
:10BC900020D0A0B3F568B369012D33D99D4228BFE8
:10BCA0004546B8E74FF0FF322146304606F002FA2B
:10BCB00070B9B8F1000F11D0B8F1010FC5D9B3694F
:10BCC0009845C2D241462246304606F0F3F928B1E3
:10BCD0000128BAD14FF0FF30BDE8F081B369326975
:10BCE000F460023B9A4201D8013A3261337943F061
:10BCF000010333712046BDE8F081BDE8F081002CDE
:10BD00009ED1B369454686E708B1042070472DE906
:10BD1000F04FDFF86892904E904C914D30704FF09C
:10BD2000010E2060C5F800E0C9F82C00D9F83C707D
:10BD3000DFF854828B4BDFF854C247F44A7747F060
:10BD40000207C9F83C704FF07469C8F808901F6882
:10BD500027F001071F601F6827F001071F602127D8
:10BD6000186058609860D86018615F61C8F80890E2
:10BD7000D3F800907C487D4F09EA0C0C4CEA000097
:10BD80001860D3F814C07A48A8F59B38A8F5C07895
:10BD90004CF0070C4FF40079C3F814C0C3F80490BA
:10BDA000C3F80880D960196841F01001196019685A
:10BDB00041F020011960196841EA0E011960C7F8C5
:10BDC00000E0036883B05202022B009200F0A380CF
:10BDD000684F00224FF0100B4FF4007A4FF04009EB
:10BDE0004FF48068FA6087E8000CC7F80890C7F83D
:10BDF000108006F095FF584603F03AFB002841D02A
:10BE00005D490B687BB923686BB933785BB94FF038
:10BE1000FF3305E0226832B9327822B9013B02D003
:10BE20000A68002AF6D00023544A0B60536B13F4BF
:10BE3000805400F086804FF0FF3401E0002C6DD07C
:10BE4000536B13F4805704F1FF34F7D12A68444D43
:10BE5000012A6ED0002C6AD03846484B3E4940F249
:10BE6000FF529A6333785BB10878C4B205F054FC92
:10BE70000028FBD1201C18BF012003B0BDE8F08FC3
:10BE80000446F3E73E4AF8601268C7F8089002FAE1
:10BE90000BF24FF0370BC7F8108087E8040806F064
:10BEA0003FFF584603F0E4FA0028A9D117224FF0CB
:10BEB000010BF8607A600192C7F80890C7F810800B
:10BEC000C7F800B006F02CFF019A104603F0D0FA34
:10BED000002895D11922009BF8607A6000923B609F
:10BEE000C7F80890C7F8108006F01AFF009A1046AD
:10BEF00003F0BEFA002883D1224B4FF0FF3190228D
:10BF0000C3F804A0D8601861C3F814B019609A602F
:10BF100006F020FF74E7530A009359E72B68104D91
:10BF2000012B04D105F0E2FB2C60002895D1042000
:10BF300093E705F0DBFB2F60002C8ED100288CD11D
:10BF4000F5E72B68064D012B01D0204685E705F06B
:10BF5000CDFB2C6081E700BFB4B70120C4B701203E
:10BF600098240020586402404054A3088C85254240
:10BF70009C240020C0BD0120B0B70120002C01404E
:10BF800000B80120D4BD0120006402403F801CF0B5
:10BF900083690BB9042070472DE9F04F05692035FE
:10BFA000B5F5001F83B003D3042003B0BDE8F08FC4
:10BFB000C5F308068846044607684EBB416901334D
:10BFC000836161B3B7F80A9009F1FF3919EA55297D
:10BFD0001ED1384606F00CF80128824627D9B0F168
:10BFE000FF3F34D0BB69984223D2831E019307F1EF
:10BFF0003408C4F814A0BB690199023B994204D2E9
:10C00000B7F80A90FB6A01FB0939C4F8189001E0FF
:10C0100007F134084644E66125610020C5E73B8905
:10C02000B3EB551FF4D80023A3610420BDE7022021
:10C03000BBE7B8F1000FF6D061692046FFF7DCFDE1
:10C04000824630B90720B0E778898345D1D00120F6
:10C05000ABE70128EBD0B0F1FF3FF8D0FB7843BB52
:10C06000BB69AAF10202023B9A42019227D3002344
:10C070000093009B3B6307F13408434607F50D71BD
:10C08000002203F8012B9942FBD14FF0000B06E090
:10C090007878FFF739FE0028D6D10BF1010B7889AB
:10C0A000009B834503EB0B0241464FF00103EFD3A6
:10C0B000CBE7384606F08CF80028D1D0C7E77A895C
:10C0C000FB6A019901FB02330093D2E708B1042017
:10C0D00070472DE9F04FDFF810927B4D7B4C7C4E82
:10C0E00028704FF0010C2060C6F800C0C9F82C0081
:10C0F000D9F83CE0DFF8F481764B774F4EF44A7E76
:10C100004EF0020EC9F83CE04FF07469C8F8089090
:10C11000D3F800E02EF0010EC3F800E0D3F800E001
:10C120002EF0010EC3F800E04FF0210E18605860A9
:10C130009860D8601861C3F814E0C8F808901868CF
:10C14000DFF8AC91DFF8ACE1DFF8AC81074047F0F5
:10C150000A6040F45530186058694FF4007740F099
:10C16000070058615F60C3F80890D96019685B4F99
:10C1700041F010011960196841F020011960196837
:10C1800041EA0C011960C8F800C0DEF8003083B045
:10C19000022B4FEA422B4FF000034FF400724FF096
:10C1A00010084FF0400A4FF480693A60019208BFCE
:10C1B0004FEA5B2BFB60C7F80480C7F808A0C7F8FC
:10C1C000109006F0ADFD404603F052F9019AF8B91F
:10C1D000434B01905A604FF0FF31902219609A60F2
:10C1E000022101221861D9604FF012085A6106F04D
:10C1F000B1FD0198F860C7F800B0C7F808A0C7F80B
:10C200001090C7F8048006F08BFD404603F030F92B
:10C2100034490B687BB923686BB92B785BB94FF055
:10C22000FF3305E0226832B92A7822B9013B02D0F7
:10C230000A68002AF6D000232B4A0B60536B13F4D4
:10C24000005437D04FF0FF3400E004B3536B13F4C5
:10C25000005704F1FF34F8D132681D4E012A21D075
:10C26000F4B13846204B184940F2FF529A632B78BC
:10C270005BB10878C4B205F04FFA0028FBD1201C4E
:10C2800018BF012003B0BDE8F08F0446F3E7336820
:10C290000F4E012B04D105F029FA34600028E1D1BA
:10C2A0000420DFE705F022FA3760002CDAD10028FD
:10C2B000D8D1F5E73368064E012B01D02046D1E7EF
:10C2C00005F014FA3460CDE7B4B70120C4B70120FB
:10C2D00098240020586402403F801CF0C0BD01201B
:10C2E000D4BD0120B0B70120002C01400064024001
:10C2F000802C01409C2400208C85254238B5036B9E
:10C300008B4218D0C37804460D467BB92A460123D8
:10C3100004F134016078FFF7D9FE002818BF4FF010
:10C32000FF3525630CBF0020012038BD05F050FF0C
:10C330000028EBD038BD002038BD00BF00224FF0F0
:10C34000FF3310B5C27003630446FFF7D7FF08B18F
:10C35000042010BD94F8331294F832324AF6552274
:10C3600043EA0123934201D0032010BD94F83430F6
:10C37000EB2B05D01833DBB2012B01D9022010BD05
:10C3800094F86A30462B07D194F86B30412B03D1D7
:10C3900094F86C30542B15D094F886300A4904F187
:10C3A0008702463B8B34002BE8D112F8013B11F891
:10C3B000010FA242A3EB0003F5D1002B14BF022012
:10C3C000002010BD002010BDC06201082DE9F84F0B
:10C3D0000B78D0F800902F2B0C46824641D05C2B76
:10C3E0003FD0D9F81430836023781F2B43D90AF14A
:10C3F00020080AF12B062025434603F8015BB342CF
:10C40000FBD123782E2B3ED00027384604F1FF3E87
:10C410004FF0080C1EF8013F202B00F1010040F204
:10C42000C9802F2B4AD05C2B48D02E2B3AD0BC454C
:10C4300035D91A063DD4222B31D06D4901E09A42FC
:10C440002DD011F8012F002AF9D1A3F16102192A88
:10C4500001D8203BDBB208F807300137DAE714F8DF
:10C46000013F2F2BFBD05C2BF9D00023CAF80830FA
:10C4700023781F2BBBD880238AF82B305046BDE889
:10C48000F84F06F081BC8AF8203063782E2B40F0FC
:10C490009E808AF82130A3782E2B40F092800620CF
:10C4A000BDE8F88FBCF10B0FF9D008274FF00B0C4B
:10C4B000B0E703F07F034F4AD35CBCE72044044657
:10C4C00010F8012B2F2AFAD05C2AF8D0002FE6D0E2
:10C4D0009AF82020E52A04BF05228AF82020202B84
:10C4E0008CBF002304238AF82B305046DAF8007002
:10C4F00006F04AFC60BBDAF818103846FFF7FEFE7B
:10C5000030BBDAF81C201378002B49D092F80BC00E
:10C510000CF03F038AF80630D37A1B0712D49646F4
:10C520009AF820101EF80B3B01325B1A0AF1210128
:10C5300043B912F8013B11F801BB9645CBEB03035D
:10C54000F6D1A3B100215046FFF722FD0028D2D03A
:10C5500004289AF82B302FD198063CD559077FF53F
:10C560004BAF80238AF82B300020BDE8F88F9AF873
:10C570002B305B072DD41CF0100F1FD0DAF81030D1
:10C5800099F8001009F13402C3F308031344032996
:10C59000D87E9A7E42EA002205D0CAF808202BE70E
:10C5A0009AF82B30D8E7597D1B7D43EA012342EAF4
:10C5B0000342F2E7044489E7BDE8F88F0520BDE8AF
:10C5C000F88F03222F2B0BD1144420238BE7022258
:10C5D000F8E7BDE8F88F5A07F0D50420BDE8F88FDA
:10C5E0005C2BF1D0202B3FF65AAF144424237AE77A
:10C5F000C862010840620108044B054A1B6803FB3E
:10C6000000F010601368002BFCD170477800002008
:10C6100084240020064B074A1B68012B18BFB0FB7F
:10C62000F3F0013010601368002BFCD1704700BF9D
:10C630001000002084240020034B1A6812B11A68ED
:10C64000013A1A60704700BF8424002030B42B4B9D
:10C6500099891A888C0602D592B2900623D4274A6B
:10C660009189138809069BB201D51B0601D430BC01
:10C6700070474FF67F73224913800B68002B31D02F
:10C680002048214B02689B5C0132FE2A026004BFF5
:10C69000002202600A681948DBB29BB2013A0A60C4
:10C6A000838030BC70474FF6DF71184A19809B8831
:10C6B00012689BB212B9DAB2032A1AD0144A11686E
:10C6C0007F29CCD81349144D0C68DBB2601C2B5564
:10C6D0007F2888BF0023086088BF0B601368013380
:10C6E0001360BCE70D4A136823F08003136030BC6D
:10C6F00070470B4A01211160E0E700BF0044004091
:10C700008824002080240020802200207C0000203B
:10C71000100700208C2400206C0300200C440040F3
:10C72000942400200E4A1368FD2BFCD830B40D4B26
:10C730000D4D1C68611CFD291960C0B288BF002125
:10C74000285588BF196072B613680133136062B64A
:10C75000064A136843F08003136030BC704700BF83
:10C760008824002090240020802200200C440040D7
:10C770000FB430B583B006AB0D4C53F8042B0193C6
:10C780004FF48071204609F097F8204609F04EF8E2
:10C790000546207828B1FFF7C5FF14F8010F0028DF
:10C7A000F9D1284603B0BDE8304004B0704700BF5F
:10C7B0008023002010B50446007828B1FFF7B2FFAF
:10C7C00014F8010F0028F9D110BD00BF034B5B6BBB
:10C7D000034214BF01200020704700BF002C01401D
:10C7E000044B82B00344002201920193019B18681C
:10C7F00002B07047142C014010B4214CA36803F020
:10C800000C03042B1BD0082B1CD01E4B03601C4AAE
:10C810001D499468C4F303140C5DE34043609468BD
:10C82000C4F382240C5D23FA04F4846092685DF8FA
:10C83000044BC2F342328A5CD340C3607047134B4F
:10C840000360E4E76368616813F4800F636818BFEE
:10C850000E4C01F03F020CBF0A49B4FBF2F1C3F3E6
:10C86000881308BFB1FBF2F101FB03F2044B5B68D4
:10C87000C3F3014301335B00B2FBF3F30360C6E78C
:10C88000003802400024F4008000002000127A00EA
:10C890000022F0B513460126032704E00133102BD4
:10C8A00002F102022FD00D6806FA03F434EA0505FE
:10C8B000F4D1D0F800E007FA02F5ED430EEA050ED8
:10C8C000C0F800E091F804E0D0F800C00EFA02FED3
:10C8D0004EEA0C0EC0F800E091F804E00EF1FF3EC5
:10C8E000BEF1010F07FA02FC0ED9C46824EA0C0459
:10C8F000C460CC79C568944001332C43102BC460CC
:10C9000002F10202CFD1F0BDD0F808E005EA0E0531
:10C91000856091F805E085680EFA02FE4EEA05058D
:10C920008560456825EA040444608C7945689C402C
:10C93000A4B22C434460D8E7F0B4114B4578D968D1
:10C94000827807780F4EC943C1F30221C1F1040474
:10C95000E4B20F2305FA04F40B41E4B2134023437D
:10C96000F2191B01DBB282F800330378012203F0D5
:10C970001F015B098A4046F82320F0BC704700BFC6
:10C9800000ED00E000E100E02DE9F04F00238FB062
:10C990000B600C46FFF708F9002813DB784B53F8BF
:10C9A00020509DB125602B781BB16B78002B00F0D7
:10C9B000D480C0B2002368702B7058B103200FB030
:10C9C000BDE8F08F0B200FB0BDE8F08F0C200FB04A
:10C9D000BDE8F08F6B4B6C4E596A706041F400619A
:10C9E0005962596A694AB06021F400615962306045
:10C9F0005368674F674CF06023F4FD4323F07F03D7
:10CA000043F0760353600321012311603B607622DB
:10CA10004FF4806323613061327520606060A060F4
:10CA2000E06006F07DF94FF480330893089B2BB942
:10CA300009E0089B013B0893089B23B18020FFF786
:10CA4000C5FE0028F5D0089B002BB7D04F4F40F211
:10CA5000FF53BB634FF4D5730820402100222360AD
:10CA60004FF4806323616060A160E26006F058F9D2
:10CA70004FF4803309937B6B13F0450F0CD1099A67
:10CA800052B1394601E0099A32B1099B013B099341
:10CA90004B6B13F0450FF6D0099A12B1580740F1CD
:10CAA000FF833A4B04229A6300274FF03708402255
:10CAB0004FF480632760E760C4F80480A2602361BC
:10CAC00006F02EF94046019702F0D2FC00233727EA
:10CAD00040214FF480622360E3606760A1602261BF
:10CAE00006F01EF9384602F0C3FC00287FF466AF5A
:10CAF000284FDFF898A00695804600234FF03709AD
:10CB00004FF0400B4FF480652360E360C4F804905D
:10CB1000C4F808B0256106F003F9484602F0A8FC05
:10CB200000287FF44BAF019BC7F808B043F00043E7
:10CB300043F480132922F8603D613B607A6006F07F
:10CB4000EFF8DAF8340010F0450FFAD010F00400D6
:10CB500005D00E4B04229A6330E718462FE740F2C7
:10CB6000FF53CAF83830FFF73BFE002808F10108F0
:10CB7000064B11DB4FF6FF739845BED11EE700BF91
:10CB80007C220020003802401C250020002C01409F
:10CB9000A0802542C0BD01204FF6FF729045069D42
:10CBA0003FF40CAF420040F1AB82DFF8A8830222D1
:10CBB000C8F800201B689F073FF400AF9146002390
:10CBC0000221C0222360E3604FF480636160A260B1
:10CBD000236106F0A5F802F033FC00287FF4EEAEE6
:10CBE000FFF7FEFDD64F38600420FFF7F9FD7860AF
:10CBF0000820FFF7F5FDB8600C20FFF7F1FDB9F153
:10CC0000020FF86003D9B9F1060F40F0EE8300235C
:10CC1000402203212360E3604FF48063A2606160DF
:10CC2000236106F07DF8C74A536B13F0450FFBD024
:10CC300058078ED413F0010040F0D083C14A136925
:10CC4000DBB2032B7FF4BAAE40F2FF539363FFF7DE
:10CC5000C7FD10F4604F7FF4B1AE030CBA4A0692E0
:10CC6000190413600922C0236260A36000224FF4FC
:10CC700080632160E260236106F052F802F0E0FB7D
:10CC800000287FF49BAEB14B0193FFF7A9FDAF4B9A
:10CC900081460420C3F80090FFF7A2FDAB4B58601B
:10CCA0000820FFF79DFDA94B98600C20FFF798FD29
:10CCB000A64BD8600023A34833604268337522F442
:10CCC000FD4222F07F024260019AA1495268D8F8E1
:10CCD000008073604FEA196E5FFA8EF04FEA901A87
:10CCE0004FEA126C81F800A0C9F3074BC9F3072A79
:10CCF0004FEA0C1CCEF3830E00F003005FFA89F9B3
:10CD000081F801E0887081F803B0069881F804A0EA
:10CD100081F80590A1F806C0B1F806C0D0F800B0BF
:10CD2000B360100AC2F307491FFA8CFC5FFA80FE59
:10CD30004CEA191C4FEADE1A09F00F09A1F806C0E7
:10CD4000B8F1010F81F80890C0F3801C81F809A0A8
:10CD5000C0F34019C0F3001A81F80AC0F36081F8EB
:10CD60000B90336181F80CA081F85680A1F854B083
:10CD7000DFF8D8C14B7340F2D582B8F1020F00F052
:10CD80009B82DCF80800019A4FEA4E0303F07E0311
:10CD9000CEF3801E81F819E0D2F80CA08B7691F8C2
:10CDA0001AE03A684FEA1A63C0B24EEAD01E4FEA60
:10CDB000830C00F07F0081F81AE00CF00C0CC876B0
:10CDC0004FEAD31EC3F34110C3F3820381F81CE082
:10CDD00048778B7781F81FC091F81FE04FEA1A4C13
:10CDE0005FFA8CF94FEA1A234EEA991ECCF3401CE5
:10CDF00081F81FE009F0010981F820C05FFA83FE85
:10CE00004FF0000C81F821C081F822904FEADE1922
:10CE100081F82390C3F3801981F82490C3F340195B
:10CE200081F82590CAF34600C3F30019C2F3074AFC
:10CE3000C3F3810381F826904FEA0A2A81F827304C
:10CE40000EF0030E130E4FF0010981F828E081F86F
:10CE5000290081F82A9081F82C30A1F82EA0CB8DE2
:10CE60007868DFF8F4A01FFA83FEC2F307234EEAC6
:10CE700003031206CB850A630A6B4FEA106E42EA7F
:10CE80000E420A630B6BC4F80CC04FEA102C0CF472
:10CE90007F4C4CEA03030B630B6BBA68FF68C0F36B
:10CEA000072C4CEA030C4FEA124EC1F830C04FEA8F
:10CEB0000E634FEA126CC0B281F8340081F835C0BD
:10CEC0008B63886B4FEA022E0EF47F0E4EEA000051
:10CED0008863886B120202F47F4202438A638A6B82
:10CEE00042EA17628A6391F83CE03A0CC2F30310FD
:10CEF00012024EEA000002F4706281F83C00CA8718
:10CF0000CA8FC7F3072E92B24FEA0B4042EA0E02D5
:10CF10004FF0070BC7F3460E40234FF48067CA87D4
:10CF2000206081F840E0C4F804B0A36081F841902B
:10CF3000276105F0F5FE584602F09AFA0EE000BFB0
:10CF400008250020002C014000B80120F824002012
:10CF5000A02400209C240020C0BD012000287FF4D4
:10CF60002DADB8F1030F3FF429ADB8F1020F00F277
:10CF7000BA80FFF735FC10F000707FF41FAD4FF062
:10CF8000100B40234FF008080A900B90CAF80C00D1
:10CF9000CAF80830CAF810708AE8000905F0C0FE27
:10CFA000584602F065FA00287FF408AD069BCAF8DF
:10CFB0000C001A68CAF8107002FA0BF240234FF006
:10CFC000370B8AE80408CAF8083005F0A9FE58466D
:10CFD00002F04EFA834600287FF4F0ACC84A3020B5
:10CFE0004FF0FF330221C2F8048013609060C2F852
:10CFF00010B0C2F814904FF03308D16005F0AAFECB
:10D000004023CAF800B0CAF80830CAF80CB0CAF811
:10D010001070CAF8048005F083FE404602F028FA3A
:10D0200000287FF4CBACDFF8DC820DF12409C24686
:10D0300004E0FFF7CBFB002840F0D981D8F834207A
:10D04000B04F40F22A6313404FF40010002BF0D091
:10D050000820FFF7BBFB002800F013820823BB6306
:10D06000ACE440F2FF53BB630A9B1BBA59037FF544
:10D07000A5AC069BE0601B684FF0370A1B044FF01D
:10D0800040094FF4806884E80804C4F80890C4F8A4
:10D09000108005F045FE504602F0EAF99A4B002850
:10D0A0007FF48CAC02220624D860C3F80890C3F841
:10D0B000108083E8140005F033FE204602F0D8F912
:10D0C00000287FF47BAC30607B68307523F4FD432F
:10D0D00023F07F0343F400634FF400627060B0609C
:10D0E00030617B60F26000212846FFF727F90228B3
:10D0F0001AD0042838D0012840F200810D205EE4C7
:10D100001B689B073FF45AACDFF81082D8F80090F8
:10D11000B9F1040F7FF453AD7C4B0193D3F8009029
:10D120007B4B7C4F0693C5E50AAC264605F5FE70A1
:10D1300005F50F7710F8063C43B1018810F8012C73
:10D1400010F8023C42EA012243EA02231030B842BE
:10D1500046F8043BEED10EAF54F8046B36B9032009
:10D16000A742F9D10428C9D1012028E43146284634
:10D17000FFF7E4F80128F3D895F8402095F83F3000
:10D1800043EA0223B3F5007FB8D195F84B1095F828
:10D190004A3053EA012340F02681B5F85A1095F839
:10D1A000593095F8582043EA012342EA032195F8C3
:10D1B0004470E9617B1E012BAF709FD895F8413018
:10D1C0009AB201FB07F76A81002A97D05A1E1A42C9
:10D1D00094D195F8452095F8464042EA0424220768
:10D1E0002C818BD195F8480095F8472052EA00220F
:10D1F00009D1B5F856E095F8550095F8542040EA65
:10D200000E2042EA002295F843E095F8420050EAE9
:10D210000E203FF473AF00EB141EBE447245FFF4C2
:10D220006DAFDFF8FCC0CEEB0202B2FBF3F35A1E87
:10D2300062453FF663AF4FF6F572934200F2EC8021
:10D2400040F6F572934200F2D780023330440EEB81
:10D250000602AB616862EA622E62002C3FF44EAFB8
:10D2600003EB4302384403F0010303EB5203A862CB
:10D27000012203F2FF13B1EB532FFFF43FAF4FF046
:10D28000FF3380212B61EB60297123492A700B88C1
:10D2900001339BB200200B80EB806861FFF78FBBEE
:10D2A000590602D5174B40229A631C4B01221A6083
:10D2B0004FF08043019309E4130403F47C130B61E2
:10D2C000DCF808000B69020E43EA02230B610B69CC
:10D2D000C0F3074213430B610A690023013243F193
:10D2E0000003DB0443EA52334FF4007CD204CB64E6
:10D2F0008A64C0F3072EC1F850C044E500263BE71E
:10D30000D4BD0120002C0140C0BD0120F824002024
:10D3100000B8012008250020182500209C240020AA
:10D32000F4FFFF0F830203F440630B610B69DCF829
:10D330000800920002F47F7213430B61D1F810C011
:10D34000020E030C5FFA82FE4FEA43094CEA9E1C70
:10D350000EF0070A09F00609C2F3C20EC3F3421227
:10D36000C3F38203C1F810C081F814E081F815A05E
:10D370008A75CB7581F818900B7EC0F3072E43EAAF
:10D38000DE130B760B6907930B7E91F808904FF034
:10D39000010C02330CFA03F30CFA09FC4FEAE37AAE
:10D3A000A3FB0C23CDE90423CDE90223079BC1F89D
:10D3B00050C003F10109059B0CFB0A330393029B48
:10D3C000A3FB0923CDE90423059A039B09FB03234F
:10D3D0000593DDE90423C1E91223D4E45A4B012269
:10D3E0009A63FFF7EBBA1946E1E6012336E4DAF86F
:10D3F000803049F8043F21E6023330440EEB060248
:10D40000AB616862EA622E62002C3FF477AE38446A
:10D41000A8625B0002222CE795F85F7095F85E2009
:10D420002E6202333044B64452EA0722AB6168628E
:10D43000C5F82CE07FF462AE002C7FF45FAEB5F847
:10D44000627095F8610095F860209B0040EA072023
:10D4500003F2FF1342EA0022B1EB532FAA62FFF45A
:10D460004DAE95F8651095F8643043EA01234FF00E
:10D47000FF328021012B2A61EA6029710AD0032240
:10D4800003E70220FFF7A2F9002849D00223BB637B
:10D49000FFF794BA711C2846FEF730FF0028EED142
:10D4A00095F8332295F832322C7143EA02234AF67A
:10D4B00055229342E3D1E88E95F8352095F8343023
:10D4C000224942EA002243EA02238B42D7D1B5F82F
:10D4D0001A0295F8192295F8183201F1FF5101F559
:10D4E000005142EA0022203143EA02238B42C6D196
:10D4F000B5F81E6295F81D02B5F8224295F8211282
:10D5000095F81C2295F8203240EA062041EA0421D1
:10D5100042EA002243EA01232A61EB600322B4E6D7
:10D520002020FFF753F918B12023BB63FFF746BA59
:10D530004FF40070FFF74AF900283FF492AD4FF422
:10D540000073BB63FFF73ABA002C014052526141AD
:10D550002DE9F04194B00223AD4D8DF80F30D5F890
:10D560001023AC4C2ABB2278002A3FD09A4200D02C
:10D570002370D4F880301B69984705F0B7FCD4F8C5
:10D5800080305B689847E36FA3495B68A048984781
:10D590000023A5F89035A5F89235A5F89435A5F89F
:10D5A0009635A5F89835A5F89A35237014B0BDE8DE
:10D5B000F08123780A2BF9D801A252F823F000BF9A
:10D5C000EDD5000849D6000873D50008ADD5000890
:10D5D000C5D60008E5D6000801D7000823D6000804
:10D5E00001D60008ADD500081DD70008D5F81033C6
:10D5F000002BDBD001236420237001F0B7FBD5E7BB
:10D60000D4F88030834C9B6B98470128CED1E36FD0
:10D610007F481B68214698470028C7D105232370FF
:10D62000C4E7237F0022013BA2740A2BBED8DFE8A7
:10D6300013F0C7010402E501620236027A02190200
:10D64000AB018C017A016D01D4F880309B6898475A
:10D6500000216F4802F078FE802160716C4802F072
:10D6600073FE20716A4801F099FBD4F88030DB68C2
:10D670009847D5F8CC20D4F880301068C0F34140EA
:10D6800084F821000422227000F003009B6998476F
:10D690000025A07994F8213094F820202179019078
:10D6A00000955B4802F06AFEA079019094F8213061
:10D6B00094F8202061790095554802F05FFE14B07F
:10D6C000BDE8F081A378092B3FF670AFDFE813F0D7
:10D6D000F500E700AF00A600770063004F003B00B5
:10D6E0008B003400E36F4B4C9B68494821469847B8
:10D6F0008DF80F009DF80F304BB90623237055E7C6
:10D70000E36F4449DB68424898478DF80F009DF865
:10D710000F0005F01BFC14B0BDE8F08105F0E6FB3E
:10D72000D4F880305B689847E36F3B495B683848C2
:10D73000984714B0BDE8F081D4F880305B6B98470F
:10D740000823237032E794F83200324C002800F0AE
:10D75000178204A905F012FC00287FF427AFD4F843
:10D76000803004A81B6B98470823A3701EE794F829
:10D770003100284C002800F0F38104A905F0FEFBDD
:10D7800000287FF413AFD4F8803004A8DB6A9847F0
:10D790000723A3700AE794F830001E4C002800F01D
:10D7A000E78104A905F0EAFB00287FF4FFAED4F876
:10D7B000803004A89B6A98470623A370F6E6E08EA3
:10D7C000144C05F013FC00287FF4F0AED4F8803040
:10D7D00004F150025B6A04F13E0104F13400984701
:10D7E0000523A370E2E60B4E94F83930E38200255E
:10D7F00009270748257531462B462A462583658328
:10D80000677505F0A7F900287FF4D0AEB770CDE6B4
:10D81000ECBD012098C30120B8C30120092005F008
:10D82000E5FB00287FF4C2AE0423A370BEE6C64E1B
:10D83000C64F00252B462A464FF0050E2575258339
:10D84000658331460125384684F815E0E58205F008
:10D8500081F900287FF4AAAE022001F087FAD6F8F9
:10D86000803086F820501B6A984796F8203031792E
:10D870000322B2701BB107EB411787F8AC33B34DED
:10D88000284601F0CDF994F8203061791BB105EB01
:10D89000411585F8AC33AD4801F0C2F986E6122097
:10D8A00005F0C2FC00287FF481AED4F88030A8488F
:10D8B000DB6998470223A37078E6082005F0B4FCE2
:10D8C00000287FF473AE94F82930A048A37101F0CA
:10D8D00065FA6179A37905EB41120126B2F8B2032A
:10D8E000A670984202D00BB1A2F8B233974801F06B
:10D8F00097F92179A37905EB4115B5F8B2239A423E
:10D90000C9D0002BC7D0A5F8B233C4E7A37B8E4A99
:10D910000133DBB2022BA37340F23F81082153781D
:10D920009174137042E66379874A1D4495F89B33DE
:10D93000DBB2012B00F02C81022B00F04C81032B79
:10D940007FF434AE0B23237730E661797F4801F111
:10D95000150205EB4212022305EB411682F8143141
:10D960000023C2F818316F18012286F8AE33C6F8CA
:10D97000BC33C6F8C03386F8C52387F89B3301F063
:10D98000A9F80A23237711E623796F496F4A1D44CA
:10D9900095F89B33DBB2012B00F0FA80032BD1D03A
:10D9A00052696C4892680D8A008892B2521B82427A
:10D9B000C8D8042B7FF4FAAD4A788B740A70F5E569
:10D9C0006179654F614801F1150305EB431305EBE0
:10D9D0004112032683F814610D44C3F81871082618
:10D9E000002382F8AE33C2F8C033C2F8BC6385F8B6
:10D9F0009B3301F06FF802232377D7E52179A268E2
:10DA0000A789524801F1150305EB4313022683F859
:10DA1000146105EB4116C3F818210D4400230122BF
:10DA2000C6F8C03386F8AE23C6F8BC7385F89B33BE
:10DA300001F050F804232377B8E56379474A2B4473
:10DA4000116893F89B33DBB28B4218BF1360012B34
:10DA500000F0A680032B7FF4A9AD0B2205232277CB
:10DA6000A374A3E52179394801F1150205EB4212AF
:10DA70006F18022605EB4115002382F81461012678
:10DA8000C2F81831C5F8BC33C5F8C03385F8AE63A9
:10DA900087F89B3301F01EF80823237786E5617928
:10DAA000A789A6684B0105EB030E01F115024FF0A3
:10DAB000000801F11E008EF8AE8305EB42182B44DE
:10DAC00005EB401005EB42124FF0010CCEF8BC7391
:10DAD000C8F818610D440026022780F805C0C3F875
:10DAE000C0631A4882F8147185F89B6300F0F2FF56
:10DAF000062323775AE52379134A2B4493F89B3363
:10DB0000DBB2012B5ED0042B5FD0032B3FF41AAFA6
:10DB10006B69104A9B68218A12889BB25B1A9342F8
:10DB20003FF610AF42E56379074A1D4495F89B33F1
:10DB3000DBB2012B4CD0042B50D0022B7FF4FFAE74
:10DB40000523137732E500BF98C30120ECBD012007
:10DB5000BAC3012044A60120ACC30120A0000020CC
:10DB6000D4F880302648DB6A98470723A3701DE568
:10DB7000D4F8803022489B6A98470623A37015E5A5
:10DB8000D4F880301E481B6B98470823A3700DE51E
:10DB9000637823700D23237708E50123137705E5C8
:10DBA000237D618B174A23F07F03DBB2D9B116497D
:10DBB00041F288300880EBB9052313776B699B68C5
:10DBC0002382F3E409231377A2E753781370EDE47B
:10DBD00007231377EAE409231377E7E453781370F4
:10DBE0000C231377E2E40849322008802BB907237D
:10DBF0001377E3E703231377E0E709231377DDE7E0
:10DC0000D862010898C3012044A6012070B5134DC5
:10DC1000134C82B0002628464FF6FF734FF416725D
:10DC20003421009600F0BAFE284607F0FFFD4FF4BD
:10DC30007843C50005F516722046009334214FF64F
:10DC4000FF7300F0ABFE009605F5187220464FF604
:10DC5000FF73342100F0A2FE02B070BD60A5012068
:10DC6000DC62010882B000230193019B0133332B56
:10DC70000193FAD902B0704700B583B0002315486C
:10DC80000193154AFFF7EEFFC3681969019106E099
:10DC9000FFF7E8FFC368013A1969019115D00199AE
:10DCA0000029F5DA01990C4A41F00101019101992D
:10DCB00019611969019103E019690191013A02D0D2
:10DCC0000199C907F8D4FFF7CDFF002003B05DF834
:10DCD00004FB00BFECBD0120400D0300184A92F880
:10DCE000C83092F8C910B3FA83F302294FEA5313EC
:10DCF00023D003291ED0012919D0002182F8C91090
:10DD0000104913F0010F0B6014BF0022082299077D
:10DD100048BF42F002025B0748BF42F001024FF0E9
:10DD2000C041094B92B2362008801A80704743F0F8
:10DD30000403E5E743F00603E2E743F00203DFE70D
:10DD400074A5012094000020000008600C4A0D4BCF
:10DD500070B4136003F5804603F5004503F54043B6
:10DD6000D360B0F5804F084B084C56604FF000016F
:10DD7000956006BF01221A601960216070BC70476F
:10DD800044A501200000001058A5012040A5012055
:10DD90000209130700F00F000AD410B40949012347
:10DDA0008C5C03FA00F0204388545DF8044B704704
:10DDB000054901220B7802FA00F023EA00000870FE
:10DDC000704700BF980000203C25002003091A0777
:10DDD00000F00F000BD410B4094C0121E25C01FAF1
:10DDE00000F022EA0000E0545DF8044B704705495A
:10DDF00001220B7802FA00F018430870704700BF48
:10DE0000980000203C250020FE2907D01F2900F0A3
:10DE10008D807F2900F08480FF207047F0B54A4B49
:10DE2000D3F8C420C0435207C3B262D513F0010E29
:10DE30001CBF464A107803F0020208BFFF2002F020
:10DE4000FF0712B1414A5278104003F0040202F079
:10DE5000FF0612B13D4A9278104003F0080202F02A
:10DE6000FF0512B1394AD278104003F0100202F0D7
:10DE7000FF0412B1354A1279104003F0200202F07B
:10DE8000FF0112B1314A5279104003F0400C0CF0FE
:10DE9000FF02BCF1000F05D0DFF8B0C09CF806C04F
:10DEA00000EA0C005BB2002B47DBBEF1000F05D08F
:10DEB000DFF89CE09EF800E000EA0E0017B1244F66
:10DEC0007F78384016B1224EB678304015B1204DDB
:10DED000ED78284014B11E4C2479204011B11C4922
:10DEE0004979084012B11A4A92791040002B20DB80
:10DEF000F0BD03F0020703F0040603F0080503F089
:10DF0000100403F0200103F0400203F0010EFFB201
:10DF1000F6B2EDB2E4B2C9B2D2B25BB2FF20C4E74E
:10DF2000FF287FF479AF0B4B187870470A4B1878AD
:10DF30007047074BDB791840F0BDDFF810C09CF844
:10DF400007C000EA0C00B0E774A5012034250020CA
:10DF500098000020900000203C250020FE2904D0DD
:10DF60007F2917D07F281DD07047264B02F007016C
:10DF700002F01002197002F0FF01234B002A34D086
:10DF80001A68002AF0D121494FF400500122088379
:10DF90001A607047FF28E7D11D4B02F003021A7088
:10DFA00004F09EBCFD29DFD11A490B68002BDBD1A0
:10DFB00070B4194D194C1A48227002F0070602F08D
:10DFC000080355F82650C56003F0FF04B3B1154BA4
:10DFD00001241C60D4064CBF134B144B0360930602
:10DFE00044BF01230B6070BCBEE71A68002ABBD097
:10DFF000064A4FF40050508319607047094B1C606B
:10E00000E8E700BF54A501205CA5012000080240FC
:10E010009000002058A50120E062010870A50120B1
:10E0200044A5012040A5012040250020000000104B
:10E0300008B5044B03221A7004F052FCBDE80840F6
:10E0400004F044BD90000020104B114A186811687C
:10E05000890600D47047C106FCD510B420210D48B4
:10E06000916002880C490D4C92B242F40072028019
:10E070001A6822F001021A600B6823F001030B609A
:10E08000002222605DF8044B704700BF1060024020
:10E090000060024000540040A0600240ECB7012044
:10E0A000094A0A4B11685A68900201D5CA0600D481
:10E0B0007047074A4FF40011D96013889BB243F4AC
:10E0C00000731380704700BFA060024000600240F0
:10E0D0000054004038B52B4C2368012B00D038BDCC
:10E0E000294804F0FFFD012809D1284B1B7813B300
:10E0F000274B284A1B6803F0FE03138238BD254DC9
:10E10000254AAB8A288B9BB243EA004311461A404A
:10E110008A4218D0214804F0E5FD0028DFD01B4BCF
:10E120001A78002ADBD01E4A127802F0FF01A2B151
:10E130000023236038BD164B164A1B6843F00103C9
:10E14000DBB2138238BD114B1B78002BC7D0154AA8
:10E15000136843F00103136038BD1348026842F0AE
:10E1600001020260AA8892B242F480524FF6FB701C
:10E17000AA801970A8822B889BB243F480732B80ED
:10E1800038BD00BFECB7012001000010DAB7012054
:10E19000E8B701200054004082000700040000108E
:10E1A000DBB70120A06002401060024002288CBF53
:10E1B00000200120704700BF022838B51ADD03385F
:10E1C000072817DC124C4FF40B7505FB0040D0F804
:10E1D0002842E3070ED5012A0B4614D0022A0FD09D
:10E1E00062B904F03DF848B105F030F94FF4FA6334
:10E1F000036003E005F02AF909230360002038BD1D
:10E20000C1681944EDE74169194404F029F8EAE7C7
:10E210004CA6012000286AD0F0B5012883B00C4636
:10E22000154624D002284BD00338072862DC3A4B2D
:10E230004FF40B7606FB0036D6F82832DB0759D5AB
:10E240000027B5F5007F5ADD01AB4FF4007221467F
:10E25000304604F0C1F850BB019BB3F5007FA5EB3D
:10E2600003051C441F44ECD2384603B0F0BD002A1D
:10E270001ADD2A4E8F1806E0FEF754FA14F8013B17
:10E280003360A74210D020780A28F5D133680D2BCF
:10E29000F2D00D20FEF746FA2078FEF743FA14F884
:10E2A000013B3360A742EED1284603B0F0BD05F034
:10E2B000CDF84FF4FA6303604FF0FF3003B0F0BDC8
:10E2C000002AF1DD164E8F1806E0FEF72BFA14F83F
:10E2D000013B3360BC42E7D020780A28F5D133688F
:10E2E0000D2BF2D00D20FEF71DFA2078EDE74FF050
:10E2F000FF30704705F0AAF809230360DCE7002D22
:10E30000B2DD2A462146304601AB04F065F800280C
:10E31000CDD1019B1F44A7E74CA60120ACB701203B
:10E3200048A60120022834DDF0B50338072883B061
:10E330002ADC204B4FF40B7707FB0037D7F8283245
:10E34000DB0721D50C4615460026B5F5007F23DDF9
:10E3500001AB4FF400722146384604F009F950B978
:10E36000019BB3F5007FA5EB03051C441E44ECD2D2
:10E37000304603B0F0BD05F069F84FF4FA6303606E
:10E380004FF0FF3003B0F0BD05F060F809230360E3
:10E39000F6E74FF0FF307047002DE9DD2A462146B1
:10E3A000384601AB04F0E4F80028E4D1019B1E4498
:10E3B000DEE700BF4CA601202DE9F043022883B020
:10E3C00040F39880C41E072C00F394804FF40B7523
:10E3D000794F05FB04F57E19D6F82832D90740F1AC
:10E3E000898001A9304603F01FFF002850D1337CFB
:10E3F0005A0663D51B066DD44FF40B7505FB04F567
:10E4000007EB05080198D8F82010DFF8AC91FDF76C
:10E4100075FF00283CD1D8F82430DA7A42F0200287
:10E42000DA72D8F8082059F805109A76C2F3072056
:10E43000D876097803296AD04FF40B7202FB047274
:10E44000CB21D2681A77100A5877100C120E9877E1
:10E45000DA7799750022B225422050219A74DA7435
:10E46000DD7518765976019B0122DA70019DEB78F3
:10E47000002B46D12B78032B4ED06B78022B15D96D
:10E480004FF40B7303FB04731A7C22F040021A74DE
:10E490004FF40B7000FB04740020D4F8283223F0F2
:10E4A0000103C4F8283203B0BDE8F0834FF40B73C6
:10E4B00003FB04731A7C22F040021A7401A930464F
:10E4C00003F0B2FE0028E3D14FF40B7303FB04F317
:10E4D000F850DDE7019BF269587805F128013944CD
:10E4E0000123FDF711FC0028D2D1337C03F07F0318
:10E4F000337481E704F0AAFF092303604FF0FF3073
:10E50000D1E7284603F064FE0028B9D1B2E7120C27
:10E51000110A1A7559758FE72B79012BADD105F1C9
:10E5200034010B4605F50D70002203F8012B8342E0
:10E530004FF00008F9D12869EB6885F81C024FEA12
:10E54000102E85F81DE24FEA104E000E2A6A85F85B
:10E550001EE285F81F024FEA132E180C85F82032B0
:10E560001B0E85F821E285F822024FF0550EAA20F5
:10E5700085F823325223013285F832E285F83302DE
:10E580004FF0610E412085F8343085F83530722324
:10E5900085F8370085F81A0285F8183285F819329F
:10E5A0002A6385F836E085F81BE201236878FDF7D9
:10E5B000ABFB85F8048060E74CA601200EB42DE982
:10E5C000F04F8EB0179B03F00302012A43D0022ABA
:10E5D00035D032B14FF0FF300EB0BDE8F04F03B090
:10E5E00070470126AB4D074600242B46D3F828225E
:10E5F00012F0010F03F50B730DD00134082CF5D187
:10E6000004F024FF172303604FF0FF300EB0BDE885
:10E61000F04F03B07047324601A968460097FEF7F5
:10E62000B3F900282FD04FF40B7000FB04F4002343
:10E630002B5104F00BFF4FF4FA630360CAE79C050B
:10E640001BD413F4806F0CBF03260B2613F0080FA6
:10E6500018BF3326C6E79D0509D413F4806F0CBF9D
:10E6600002260A2613F0080F18BF3226BAE713F461
:10E67000806F0CBF12260A26F4E713F4806F0CBFDC
:10E6800013260B26E2E79DE80A0002A80293FDF795
:10E690009DFE002871D19DF93330002BC3DB16F0AD
:10E6A0001C0F00F0D7809DF80E3013F0110FBAD177
:10E6B000300700F1F180DDF804E0DEF83010099B4E
:10E6C0004FF40B7202FB0452116253629EF8000079
:10E6D000D97E9A7E032842EA012100F0D3804FF4CC
:10E6E0000B7202FB04F2A81802F128078160597F1F
:10E6F000B3F81EC01B7F45F802E041EA0C2243EA52
:10E700000223C360BEF80630838000222F440674C3
:10E7100007F500713B464274C261426103F8012B68
:10E720008B42FBD1B10640F185804FF40B7909FB98
:10E7300004F905EB0903DE68002E7BD05E61BEF8AC
:10E740000A8099684FEA482846454DD9C8EB060625
:10E7500002E0464548D91E4655F8090003F048FC3A
:10E7600001280146C8EB060301D9421CF1D14FF440
:10E770000B7303FB0453996155E716F01C0F3FF42C
:10E7800052AF04287FF44FAF02A8029F04F0FCFAB6
:10E7900000287FF448AF08993846FDF7AFFD002800
:10E7A0007FF441AF099B1B78E52B03D0012102A820
:10E7B000002B62D108993846FDF7A0FD00287FF4B0
:10E7C00032AF099B024603F1200103F8012B8B4273
:10E7D000FBD10B220AA9099803F01CFD46F008069C
:10E7E0000123F6B2FB7063E74FF40B7000FB04509B
:10E7F000C6F308038161EBB1DDF804E0DEF8183000
:10E800000239023B9942BFF40EAFBEF80A30DEF87F
:10E810002C2001FB0322002A3FF405AF02EB562215
:10E82000C2619EF8010039460123FDF74FFC002824
:10E830007FF4F9AE4FF40B7303FB0453E01CD3F8E1
:10E84000282242F00102C3F828220EB0BDE8F04FA2
:10E8500003B070479DF80E30D9063FF5E4AEB2071D
:10E8600002D5DF073FF5DFAE3007DDF804E07FF5C6
:10E8700024AF46F04006F6B21FE7FDF789FB0028FB
:10E8800089D0D0E6587D1A7D42EA002241EA024151
:10E8900025E700BF4CA601200199099B0A78DF7E7D
:10E8A000987E032A40EA072770D0CB229A73422031
:10E8B00050224FF0B20E5A7483F80FE01874099B7F
:10E8C0002022DA72099B00229A76DA7608780328E9
:10E8D00004BF1A755A75099B002201201A775A77CE
:10E8E0009A77DA77C87017B9DDF804E0C1E7012F2D
:10E8F0007FF699AEDDF80880D8F818309F42BFF453
:10E9000092AE019B4046D3F830B0B9462BE00128C7
:10E910003FF489AEB0F1FF3F3FF485AEB9F1010F8E
:10E920007FF681AED8F818309945BFF47CAE4946E1
:10E930000022404603F0BEFB00287FF474AED8F8F6
:10E940001810D8F810308A1E934208D298F8042084
:10E95000013342F00102C8F8103088F804208A45DB
:10E9600007D20298D146494603F042FB824600286E
:10E97000CDD159460198FDF7C1FCDDF804E0013F17
:10E98000CEF80C7000283FF474AF4CE6587D1A7D29
:10E9900042EA002247EA024787E700BF2DE9F04F2D
:10E9A00085B00C460391017802900093002945D070
:10E9B00002F10803234D019304F10C060198B6F50A
:10E9C000F07FA0F1080730D2B0F5487F2DD21E4B62
:10E9D000DDF80CB00C2202FB013202F1FF3A00F12B
:10E9E000FF394FF0C048494638461AF8014F00F049
:10E9F00087FC5846594600F06FFC2C23A8F80030DD
:10EA0000BDF838C0BDF800E00723012000FA03F28A
:10EA1000224214BFA5F800E0A5F800C013F1FF33AF
:10EA2000F4D20BF1010BB345DDD1029B13F8011FAA
:10EA30000293019B083301930029BFD105B0BDE8C3
:10EA4000F08F00BF00000860006301084369586947
:10EA5000704700BFC36858699B691840704700BF82
:10EA6000C368586900F00100704700BF00EB8101E6
:10EA70004FF00043D1F89020012060F3DC43136194
:10EA8000D1F890201368002043F0004360F39E7398
:10EA90001360704700EB810186B0D1F890201368B5
:10EAA00043F0404359030AD541690969C1F307415D
:10EAB00009B96FF3DF730020136006B07047C168B7
:10EAC000C96AC1F307410029F3D00020136006B0E2
:10EAD000704700BFF0B54C01051987B0D5F8BC33BD
:10EAE0000022D3B1B5F8B263013B3344B3FBF6F374
:10EAF0009BB2B3F5807F64D93602C5F8BC630519B3
:10EB00004FF4807795F8AE633B466EB1B5F8B263CB
:10EB100003FB06F3C5F8BC3308E001273B460519A3
:10EB200095F8AE63002EF1D1D5F8BC3301F115068E
:10EB300000EB461500EB810163F3120295F814E136
:10EB4000D1F8903067F3DC426EF35E721A61C378DD
:10EB5000012B39D0D1F8905042692B68926802F0AD
:10EB6000010282F0010262F35D7343F000436FF330
:10EB70009E732B60C3780BBB021992F8AE33EBB9CE
:10EB8000D2F8BC33D3B192F8B123032A2BD8DFE8F3
:10EB900002F021022102426915690195DA1CADB229
:10EBA000C2F38F0295421ED2C268936943F080631C
:10EBB00093610444C278D4F8BC33A2B1002007B0FA
:10EBC000F0BDC3F30907AAE7D1F89030D5F81821B2
:10EBD0005A61BFE7C768FD6A0395DA1CADB2C2F39C
:10EBE0008F02954211D300EB4610D1F8D040D0F8F7
:10EBF000182198B203308010E0D00023013352F87E
:10EC0000041B21609842F9D1D8E7BB6943F0200387
:10EC1000BB610444C278D4F8BC33002ACED1E2E709
:10EC2000F0B400EB81054FF0FF34D5F890204B0194
:10EC30009460C418C27894F8B163012A14BF002408
:10EC400004240022032E13D8DFE806F002550249FF
:10EC5000C61844F4936496F8AE7344F00104002F90
:10EC600046D196F8B06344F040040EB144F020045D
:10EC7000D5F89060F46047690126BC6906FA01F195
:10EC80002143B961C468A169184441F00073A361CC
:10EC900090F8AC7390F8AF3390F8AD6390F8AE4352
:10ECA00090F8B113B0F8B20367F39C52A3F10203DA
:10ECB00066F3CE22B3FA83F364F3CF325B0963F3D6
:10ECC000514261F3934260F30A02D5F89030032970
:10ECD00008BF42F000521A600020F0BC7047C6180E
:10ECE00044F4D36496F8AE6344F00104002EBFD020
:10ECF00044F48074BCE7C61844F4087496F8AE6314
:10ED000044F00104002EB3D044F4C074B0E700BF57
:10ED10004269136861F301031360704730B4033232
:10ED20009210D0F8D05009D00846002301332C6847
:10ED300040F8044B9A42F9D101EB8201084630BCFD
:10ED4000704700BF30B4C4786CB900EB8200033365
:10ED50009B10D0F8D05006D02246013251F8040B57
:10ED600028609342F9D1002030BC7047094A0A4B11
:10ED700002FB00F0A3FB0023C21A82B003EB520295
:10ED8000002392080193019B01339A420193FAD226
:10ED900002B07047C0D401002549922410B5044642
:10EDA0000A20D4F8CC2013686FF382036FF3410379
:10EDB0006FF3C3036FF3451343F480711160FFF7E2
:10EDC000D5FFD4F8CC306FF3082119601420FFF779
:10EDD000CDFF012010BD00BF2DE9F8430446FEF72A
:10EDE000B7FB1D4B1B78012B10D01C4A11789942A0
:10EDF00018BF13701A4B1A680AB9BDE8F88319498D
:10EE00004020002208831A60BDE8F883144A116884
:10EE1000E1B1154E154D3168DFF85880144FA94601
:10EE20002B688B4203F10102E7D0202A38F8130047
:10EE300008D0C9F800200CB13860F1E700F0E2FD1D
:10EE40003168EDE70023C9F80030F4E705494020B8
:10EE500048831360DDE700BFA8BD0120A4000020A7
:10EE6000B8B7012000000240B8BD0120C8B701209A
:10EE7000BCB701200CBD012010B5044C206818B1AE
:10EE800004F050FB0023236010BD00BFC0B7012079
:10EE900070B54368013B002B04460E46436010DB0F
:10EEA0000268511C01601578013B002B636012DB86
:10EEB00023685A1C2260187845EA00253580012015
:10EEC00070BD0A4B0146186805F05CFA421C054605
:10EED0000AD1002070BD054B2146186805F052FA92
:10EEE000431CE9D1002070BD6368DDE728010020E4
:10EEF00010B54368013B002B0C46436006DB0368FA
:10EF00005A1C026018782070012010BD044B014685
:10EF1000186805F037FA431CF5D1002010BD00BF7A
:10EF20002801002030B5C3B00DF106010446FFF7FB
:10EF3000AFFF10B9002043B030BD0DF103012046F2
:10EF4000FFF7D6FF0028F5D09DF803300025C3B1A8
:10EF50000DF105012046FFF7CBFF013501A900287F
:10EF6000E8D02046FFF7C4FF234601210028E1D066
:10EF70009DF8042002A804F057FD9DF80330AB4231
:10EF8000E6DC0120D7E700BF2DE9F04F85B00F4642
:10EF90000DF10E01904600939DF838600546FFF78D
:10EFA000A7FF00285CD00F9B9DF80EA09C1EBAF115
:10EFB000000F59D1002E40F08E800DF10F067CB36A
:10EFC000B9460197009FD3460DF10F0631462846FA
:10EFD000FFF78EFF0BF1010109F10102002840D07B
:10EFE000D8451FFA81FB12D98FB1B9F5804FC9F30B
:10EFF0008F30C9F30D010AD3B9F5B64FC0F099802F
:10F000006A4B9DF80FE053F8200000F801E09DF8EE
:10F010000F105C451FFA82F98AEA010AD6D8019FCF
:10F020006249B80BC7F30D0251F82000825C002A38
:10F0300000F08580012431462846FFF759FF78B15A
:10F040009DF80F20524572D0594C5A48236823220C
:10F05000DB68012106F000F82368D86804F01CFB87
:10F06000002005B0BDE8F08F002E49D00DF10F064D
:10F07000002CDFD04FF0000B0DF10F064FF001090F
:10F0800031462846FFF734FF0BF101017A1C0028B6
:10F09000E7D0D8451FFA81FB15D9009B9BB1B7F586
:10F0A000804F4FEA9730C7F30D010CD3B7F5B64F39
:10F0B00038BF414B9DF80F7038BF83F800903B4B31
:10F0C00053F8200047549DF80F105C4597B28AEA28
:10F0D000010AD5D8AEE7002C60D057460DF10F06D7
:10F0E00005E09DF80F30BC428AEA030A1DD931467B
:10F0F0002846FFF7FDFE0137BFB20028F1D1AFE788
:10F10000002C48D037460DF10F0605E09DF80F3072
:10F11000BC428AEA030A08D931462846FFF7E8FECE
:10F120000137BFB20028F1D19AE7002483E72046D7
:10F1300097E7214B4FF0010E83F800E060E71F4A8C
:10F1400092F88020002A7FF475AF43F6F27297425E
:10F1500028DD45F6F222974202DC174A01201070A2
:10F1600007F10D029013C2F30D0251F8204045F64D
:10F17000F1204FF0000E874204F802E002DC0E4A54
:10F18000012010700E37BA13C7F30D0751F8222073
:10F190008021D1554EE70DF10F064CE754460DF195
:10F1A0000F0648E77FF446AFE9E700BF44A501201A
:10F1B00028010020006F0108A500002074A501208F
:10F1C0003F49404BD1F888203F4842F47002C1F8D3
:10F1D00088201A68002142F001021A6099601A68BA
:10F1E00022F0847222F480321A6058601A6882B069
:10F1F00022F480221A60D960009101911A6842F4C9
:10F2000080321A6003E0009AB2F5C06F09D01A6824
:10F2100002F400320192009A01320092019A002A0F
:10F22000F1D0284B1B6813F4003318BF012301935E
:10F23000019B012B00D0FEE7224B24491A6C42F0BF
:10F2400080521A640A6842F480420A609A689A609E
:10F250009A6842F400429A609A6842F4A0529A6016
:10F260001A6822F080721A601968164A8801FBD465
:10F27000174B5360136843F0807313601168114B90
:10F280008901FBD5134A40F205711160126802F042
:10F290000702052A00D0FEE79A6822F003029A606E
:10F2A0009A6842F002029A609A6802F00C02082AF8
:10F2B000FAD1034B4FF000629A6002B0704700BF72
:10F2C00000ED00E0003802401030002400700040E3
:10F2D000042A4007003C024070B4084B4FF0C04580
:10F2E000C0F30F242B26C1F30F22C0B2C9B22E8067
:10F2F0001C8018801A80198070BC7047000008605C
:10F3000070B4084B4FF0C045C0F30F242A26C1F358
:10F310000F22C0B2C9B22E801C8018801A801980BA
:10F3200070BC70470000086070B55C1A0D461E4640
:10F330001146131A013403FB0444FFF7E1FF314681
:10F340002846FFF7C9FF4FF0C0432C221A803CB17A
:10F350000449BDF81020002301339C420A80FBD1F0
:10F3600070BD00BF00000860054B1A6812F0C05F56
:10F3700005D0044901204FF0046208609A6070478C
:10F3800000640240B0B7012038B54FF48070FDF73B
:10F390001DFA38BB0220FDF719FAA8B90820FDF7BD
:10F3A00015FA002830D12020FDF710FA28BB1020D4
:10F3B000FDF70CFA00282ED14FF40070FDF706FA85
:10F3C00000282FD11B4904E01B4A1A4902239363EA
:10F3D0000B70194AD36B23F4434323F03A03D363EE
:10F3E0000B7838BD13491448144B00254FF4807432
:10F3F00001220D7084631A60EBE70F4A0D4920204B
:10F40000062390630B70E4E70B4A0A4908200423A3
:10F4100090630B70DDE7084A0649102005239063CE
:10F420000B70D6E7044A03494FF40070072390633A
:10F430000B70CEE7B4B70120002C0140C4B7012007
:10F440000A4A536B13F0450FFBD05A0709D413F047
:10F450000100064B15BF012040F2FF5298639A63EA
:10F460007047024B04229A6303207047002C01402E
:10F4700008B5384A536B13F0450FFBD059070DD42C
:10F4800013F0010306D133490A69D2B290420AD07F
:10F49000102008BD2F4B0120986308BD2D4B04227E
:10F4A0009A63032008BD40F2FF5218468A63FDF7B5
:10F4B00097F9294B03402BB1002805DB420005D505
:10F4C000092008BD184608BD1C2008BD830001D5D1
:10F4D0000A2008BDC10001D50B2008BD020101D5DD
:10F4E0000C2008BD430101D50D2008BDC10101D587
:10F4F0000E2008BD020201D50F2008BD4302C7D46B
:10F50000810201D5112008BDC20201D5122008BD1B
:10F51000030301D5132008BD410301D5142008BD04
:10F52000820301D5152008BDC30301D5162008BDEF
:10F53000010401D5172008BD420401D5182008BDDB
:10F54000830401D5192008BD10F0080F0CBF00205E
:10F550001A2008BD002C014008E0FFFD80B586B0F0
:10F5600000AF786000237B6100233B617868FFF780
:10F570006DFA0346FB6000237B612AE0BB891A46D3
:10F580007B6942FA03F303F00103002B1ED07A6873
:10F590007B6922339B0013449B681B68BB607B7AAA
:10F5A00023F07F03DBB2002B08D07969786801F083
:10F5B0007BF802463B6913433B6107E07969786851
:10F5C00001F04CFB02463B6913433B617B6901330D
:10F5D0007B617B681B781A467B699A42CED83B696F
:10F5E00018461837BD4680BD80B584B000AF78603E
:10F5F0000023FB600023BB607868FFF731FA034605
:10F60000002B71D07868FFF725FA0346BB60BB6812
:10F61000002B01D1002368E03B7A03F00803DBB242
:10F62000002B06D0786802F019F80246FB681343F5
:10F63000FB603B7A03F01003DBB2002B06D0786846
:10F6400000F066FF0246FB681343FB603B7A03F061
:10F650002003DBB2002B06D0786801F021FF0246C0
:10F66000FB681343FB60FB7A03F00403DBB2002B5F
:10F6700006D0786801F050FE0246FB681343FB6039
:10F68000FB7A03F00203DBB2002B06D07868FFF7A9
:10F6900065FF0246FB681343FB60FB7A03F001033E
:10F6A000DBB2002B06D0786801F082FD0246FB68D1
:10F6B0001343FB60FB7A03F02003DBB2002B06D080
:10F6C000786801F0B1FF0246FB681343FB60BB7A28
:10F6D00003F02003DBB2002B06D0786800F0F0FEC8
:10F6E0000246FB681343FB60FB6818461037BD46B3
:10F6F00080BD00BF0148FFF777BF00BFECBD012010
:10F7000010B4A44CFF2323706370C30511D5B0F56A
:10F71000B97F44D024D8B0F58A7F3DD040F26B1336
:10F72000984203D100223423227063705DF8044BA9
:10F7300070477F28FAD8984B1B78EBB9974B03EBAF
:10F74000400213F810305278D9071DD500232370DA
:10F75000FF2A18BF0123E9D0E2545DF8044B70473B
:10F76000B0F5BA7F20D040F275139842DED1002266
:10F77000432322706370D9E7894B03EB400213F8EF
:10F7800010305278D907E1D403F0020303F0FF01EF
:10F790007BB171232370DBE771232370C6E700225E
:10F7A000442322706370C1E70022422322706370F9
:10F7B000BCE7FF2A40F0078169381428B6D801A3B6
:10F7C00053F820F083F800082DF70008A7F8000888
:10F7D00071F800082DF700082DF700082DF7000834
:10F7E00095F800082DF700085FF800085FF800089A
:10F7F0004DF800083BF800082DF700082DF7000829
:10F800002DF700082DF7000829F800082DF700084B
:10F810002DF7000819F80008624B1B78032B85D8D8
:10F82000DFE803F0AEA9A49F5E4B1B78032B3FF6E5
:10F830007DAFDFE803F0918C87825A4B1B78032B56
:10F840003FF674AFDFE803F041535956554B1B7830
:10F85000032B3FF66BAFDFE803F03538476D514BB4
:10F860001B78032B3FF662AFDFE803F0292C6135EC
:10F870004C4B1B78032B3FF659AFDFE803F0504B9E
:10F880004641484B1B78032B3FF650AFDFE803F0AF
:10F8900096918C7D434B1B78032B3FF647AFDFE8F7
:10F8A00003F00B0B17433F4B1B78032B3FF63EAF88
:10F8B000DFE803F00E0517144023237036E74423D6
:10F8C000237033E74223237030E7432323702DE76F
:10F8D000342323702AE78223237027E781232370B0
:10F8E00024E73023237021E7312323701EE74123CF
:10F8F00023701BE78323237018E73323237015E756
:10F90000812283232270637010E730223323227018
:10F9100063700BE7442241232270637006E73422B0
:10F9200043232270637001E784232370FEE63223B1
:10F930002370FBE680232370F8E680228223227066
:10F940006370F3E64322422322706370EEE63122B5
:10F95000322322706370E9E64222442322706370EE
:10F96000E4E68022832322706370DFE631223323B2
:10F9700022706370DAE64322412322706370D5E679
:10F980004222432322706370D0E6812282232270B8
:10F990006370CBE6D8B70120E4B7012024700108DA
:10F9A000246F0108C40000203022322322706370CB
:10F9B000BCE64422422322706370B7E6342244231B
:10F9C00022706370B2E60B46E254C6E64FF0804305
:10F9D0004FF6FE7208481A82084903680A68013324
:10F9E0000132B3F57A7F0A6003D1054A0121002371
:10F9F00011600360704700BFD4B70120540100209C
:10FA00006022002000F4007292B210B5C2B95928E9
:10FA10002AD00D2837D005283BD0062848D0042806
:10FA20002DD0294CFFF76CFE2078FF2812D0FEF76E
:10FA3000CDF96078FF280DD0BDE81040FEF7C6B9BB
:10FA4000C0F30800592813D01F4CFFF759FE207847
:10FA5000FF2800D110BDFEF79BF96078FF28F9D090
:10FA6000BDE81040FEF794B9184B01221A7010BD82
:10FA70000020FEF78DF9154B00221A7010BDBDE86D
:10FA8000104003F017B81249124B012008601A7099
:10FA900010BD114991F8C9300133DBB2042B14BFFA
:10FAA00081F8C93081F8C920BDE81040FEF716B9C9
:10FAB000094991F8C8300133DBB2022B14BF81F839
:10FAC000C83081F8C820EFE7D8B70120E4B701209B
:10FAD00040B801207400002074A501202DE9F041F8
:10FAE000214C236882B01BB1002002B0BDE8F08138
:10FAF0001E4E3368002BF7D11D4A4FF400301370AF
:10FB000003F0F0F807460028EED1DFF88080D8F83F
:10FB10000030012BE8D001251F2301A88DF8043007
:10FB20008DF805708DF806708DF80750FCF704FF0E
:10FB3000104B1149114A12484FF0A40EC3F800E0CF
:10FB4000104BC8F800500D70177006210E4A456022
:10FB5000596013889BB243F4807328461380356044
:10FB6000256002B0BDE8F0813CB80120DCB701207F
:10FB700024200020E8B70120DAB70120DBB70120FC
:10FB8000A06002401060024000540040ECB7012029
:10FB90002DE9F8439D4C2368012B02D00020BDE8DD
:10FBA000F8839B4B1A68012AF8D19A4A1268002AF6
:10FBB000F4D1994D2A68022A00F096819749984A13
:10FBC0004E790F7849785170D1881770B7074CBFBC
:10FBD00021F4807141F4807189B2F607D1804CBF65
:10FBE00021F0800141F08001D1800021196020B90D
:10FBF000002323600120BDE8F8832B68022B1378D3
:10FC000000F0AF80A02B00F2A680602B34BF04254B
:10FC100000255378A02B40F2998045F00105D38848
:10FC20001E0648BF45F01005D80500F196807D4FAF
:10FC30003E68AE42DCD06E4071070DD57A4B6A0744
:10FC40001B7840F10C81032B06D8DFE803F07B6BB7
:10FC500067028120FEF7BAF833070DD5724B2807EB
:10FC60001B7840F1E580032B06D8DFE803F06763DB
:10FC70005F028020FEF7AAF8F1070DD56A4BEA076C
:10FC80001B7840F11A81032B06D8DFE803F03B43D1
:10FC90003F028320FEF79AF8B3070DD5624BA80701
:10FCA0001B7840F1F380032B06D8DFE803F0271F11
:10FCB0001B028220FEF78AF8F1060DD55A4BEA06A0
:10FCC0001B7840F19080032B06D8DFE803F0020296
:10FCD00013074020FEF77AF83D6089E78420FEF79D
:10FCE00075F8F9E73220FEF771F8E5E74220FEF7F4
:10FCF0006DF8E1E73420FEF769F8EDE74420FEF700
:10FD000065F8D9E74320FEF761F8C5E73320FEF731
:10FD10005DF8C1E74120FEF759F8BDE73020FEF756
:10FD200055F899E74420FEF751F895E73120FEF7A2
:10FD30004DF8A1E74320FEF749F89DE74220FEF782
:10FD400045F899E73420FEF741F885E75F2B98BF27
:10FD500045F0020563E708255BE7344B00221A7083
:10FD600065E7282B00F2F380182B34BF04250D46DD
:10FD700053782B49282B32D8172B40F2EA8085BBC9
:10FD80008B78142B00F2EB800B2B8CBF0025042505
:10FD9000D3782349142B22D80B2B40F2DA80CE885B
:10FDA00065B9B70700F1E28016F4004F0CBF0025DB
:10FDB0000825F00740F1D58045F0010542F2FC230B
:10FDC00033400BB145F01005F20400F1C580330556
:10FDD000C3D477057FF52BAF02F078FE27E745F017
:10FDE0000105D688EAE7032B3FF676AFDFE803F09C
:10FDF00002020A064020FDF7CBFF6DE78420FDF7E5
:10FE0000C7FF69E73420FDF7C3FF65E73CB8012071
:10FE1000DCB70120ECB7012044B80120080700201E
:10FE2000CCB70120E0B70120C400002074000020FE
:10FE3000032B3FF621AFDFE803F00E0A0602802015
:10FE4000FDF7A6FF18E73120FDF7A2FF14E74320D6
:10FE5000FDF79EFF10E74220FDF79AFF0CE7032B0A
:10FE60003FF6FAAEDFE803F00E0A06028120FDF746
:10FE70008FFFF1E63020FDF78BFFEDE64420FDF724
:10FE800087FFE9E63420FDF783FFE5E6032B3FF625
:10FE900013AFDFE803F00E0A06028220FDF778FFB9
:10FEA0000AE73220FDF774FF06E74220FDF770FFF6
:10FEB00002E74420FDF76CFFFEE6032B3FF6ECAEB5
:10FEC000DFE803F00E0A06028320FDF761FFE3E698
:10FED0003320FDF75DFFDFE64120FDF759FFDBE64C
:10FEE0004320FDF755FFD7E6214E224A96F800C081
:10FEF00096F801E0B77896F804904FEAEC084FEADC
:10FF00006E1108F0180801F0060148EA01010CF032
:10FF10003F0C96F80380767982F800C04FEAA70C70
:10FF200008F0070846EA09260CF0180C41EAD71138
:10FF30000EF03F0EF64307F01F074CEA080C82F85C
:10FF400001E09170D77082F804C0D6804DE6082594
:10FF50000EE745F0020544E702F0ACFD37E708255F
:10FF600016E7710448BF45F0020527E7042520E79E
:10FF700008070020CCB70120104A1378A02B02D923
:10FF80004FF4BA7070475F2B02D840F26B10704785
:10FF90005378A02B02D940F2751070475F2B02D81E
:10FFA0004FF4B9707047D3881A0601D55A207047AC
:10FFB00013F4807F0CBF002076207047CCB701205F
:10FFC00010B5304A304C13680133022B13601FD92F
:10FFD00023782D4A282B0CD8172B13D8A3782A4A1C
:10FFE000142B40F26B100AD80B2B2CD840F26B105C
:10FFF00010BD4FF4BA70A378234A142BF4D94FF4F0
:020000040801F1
:10000000BA7010BD5378282B17D940F27510F2E75B
:1000100021781E48FCF7ACFB61781D48FCF7A8FB73
:10002000A1781C48FCF7A4FBE1781B48FCF7A0FB77
:10003000E1881A48FCF79CFBCAE7172B8CBF00200D
:100040004FF4B970D7E7D378142B02D940F275106A
:1000500010BD0B2B02D84FF4B97010BDD3889A078E
:10006000C4D41C04CBD4D907F0D45A04F3D442F23C
:10007000FC221A400AB15A2010BD13F4E05F18BFE9
:10008000762010BDF0B70120CCB701202471010803
:100090002C710108347101083C7101084471010898
:1000A000F0B585B002F012FE304D314BAC881E68C1
:1000B0006846FCF7A1FB029A2E482F4BA0FB0210CA
:1000C00024F03F042404800C240C87B23C43AC8011
:1000D000298821F001010904090C9E42298029D8B0
:1000E0007300B2FBF3F39BB2032B07F1010798BF38
:1000F00004232F841D4A938313889BB243F001038A
:100100001380138823F4816323F002031B041B0C68
:1001100043F480634FF480411380118193889BB234
:1001200043F40073938013889BB243F00103138060
:1001300005B0F0BD06EB4603B2FBF3F39BB2C3F38D
:100140000B020AB943F001034FF496710B4C074DB3
:1001500001FB00F284FB0201D217C2EBA1120132B3
:1001600092B243F400432A84C4E700BF0054004025
:100170006422002083DE1B43A0860100D34D621061
:1001800008B50B4A13889BB243F40073138013889D
:100190006FEA43436FEA53439BB213801388C3F360
:1001A0000E03138002F092FDBDE80840FFF778BF10
:1001B00000540040002070470023C0F81033184658
:1001C000704700BF0123C0F810330020704700BF04
:1001D000F8B53E4D95F845300446042B23D8DFE8AA
:1001E00003F03C243C1303000023012221270B26AB
:1001F000CA820F754E750B834B831A4602F0AAFC18
:1002000088B985F84500F8BD00230A2221264A75E1
:100210000E75CB820B834B831A4602F09BFC0028A1
:100220004FD003284DD00120F8BD294B4FF4085082
:1002300000221B89C882812706260A834B830F75FB
:100240004E7504F58872204602F084FC0028EAD13D
:10025000032385F845300120F8BD4FF404500022F7
:10026000812706260923C8820A830F754E754B83A2
:1002700004F58872204602F06DFC0028D3D194F872
:10028000130194F81211124B94F8186194F8172185
:1002900094F810711F7001EB002194F8110194F88B
:1002A0001471598002EB062294F8161194F8156126
:1002B000587001201F715E7199711A8185F845008F
:1002C000F8BD042385F845300120F8BD50BD01205C
:1002D000F4B7012070B51A4C94F840100546E9B9FE
:1002E00094F84110164E19B9164B00221A7070BDC1
:1002F0002846FEF7CFFB96F84130072B07D805EBD1
:100300004305B5F88C35C3F30E03A5F88C350023EF
:1003100084F841300B4B00221A7070BDFEF7BAFB17
:1003200094F84030072B07D805EB4303B3F88C252E
:10033000C2F30E02A3F88C25002384F84030CFE7E7
:1003400050BD0120B4BD012030B400F28A52002318
:1003500032F9024F002CDDB205DA0133082BF7D158
:10036000FF2030BC704700EB43006FEA41416FEA69
:100370005141A0F88C15284630BC7047F8B500EB09
:10038000410500EB4114B5F88C559DF8187084F8C0
:10039000AC2305F07F06C5F3C01584F8AD6384F87F
:1003A000AE53BDF81C6084F8AF33002584F8B173F8
:1003B000A4F8B26384F8C45384F8C55313B9012375
:1003C00084F8B033FEF72CFC0020F8BD2DE9F04393
:1003D00091F84430364D0622012B83B00C4685F847
:1003E000422007D0D1F880301B6C9847012003B021
:1003F000BDE8F08391F84530012B074654D0022B1D
:1004000004BF2C4B2B6594F8561094F85230B4F876
:10041000540085F84830002285F8422085F84520B0
:100420000929234AA5F8460098BF0A21A2F84A10D4
:1004300094F84260022E28BF02267EB3013EF6B237
:100440001A0604EBC606A0464FF0030919463846C3
:100450001CD485F84330FFF777FF014685F841004B
:10046000B5F8460094F8213094F820200190CDF89A
:1004700000903846FFF782FFB0450FD098F85A3009
:100480001A0608F1080819463846E2D585F84430BE
:10049000FFF75AFF014685F84000E1E7064B0020D0
:1004A000187003B0BDE8F083044B2B65ABE700BFC9
:1004B00050BD0120BC000020B4BD0120A8000020D8
:1004C00080B485B000AF78607B68D3F890301B684B
:1004D000BB60FB7A43F08003FB72FB7A43F040037E
:1004E000FB727B68D3F89030BA681A600023FB6017
:1004F000BB7B43F02003BB737B68DB68FA685A61FF
:10050000012318461437BD465DF8047B704700BFD1
:1005100080B588B000AF78600023FB7200237B6158
:100520003B7D43F010033B757B68DB687A68D268DB
:1005300091697A69D2430A409A617B68DB681B6AD9
:10054000BB613B7EC3F30303DBB2FB72FB7ADBB21E
:100550007A6822339B0013449B681B68FB60BB7E58
:10056000C3F34303DBB2022B40F08D803B8BC3F31C
:100570000A139BB2002B40F38580FB7ADBB27A68CA
:1005800015335B01134403F58C731B68002B79D082
:10059000FB7ADBB27A6815335B01134403F58C7385
:1005A00019683B8BC3F30A139BB21A467868FEF7AF
:1005B000B5FB3B7EC3F30303DBB218463B7EC3F3BC
:1005C0000303DBB27A6815335B01134403F58C73C4
:1005D0001B683A8BC2F30A1292B21A44796800F18E
:1005E00015035B010B4403F58C731A603B7EC3F368
:1005F0000303DBB218463B7EC3F30303DBB27A6826
:100600005B01134403F570731B683A8BC2F30A1243
:1006100092B21A44796843010B4403F570731A606F
:10062000FB7ADBB27A685B01134403F570731B68D5
:10063000FB61FB7ADBB21A467B68D432F96943F876
:100640002210FB7ADBB27A6822339B0013449B684A
:100650001B693B617B8AC3F3C9039BB2002B11DD8D
:10066000FB7B43F08003FB73FB7B6FF38613FB7311
:10067000FB7ADBB27A6822339B0013449B68FA68EA
:100680001A6000E000BF3B7D43F010033B757B68C0
:10069000DB687A68D26891697A690A439A610123B2
:1006A00018462037BD4680BD80B59CB000AF78604D
:1006B00039607A683B6822339B0013449B68FB6671
:1006C000FB6E9B68BB66FB6EDB687B66BA6E7B6EFF
:1006D0001340BB667A683B6822339B0013449B68D7
:1006E0001B683B6600237B6697F8683003F00403C1
:1006F000DBB2002B1DD00023FB603B7B43F00403E7
:100700003B73FA68FB6E9A607A683B6822339B0001
:1007100013449B68DB683B613B7C43F002033B7402
:100720007A683B6822339B0013449B683A69DA601D
:1007300093E097F8683003F02003DBB2002B09D078
:1007400000237B613B7D43F020033B757A69FB6EA0
:100750009A6082E097F8683003F00803DBB2002B60
:100760003BD07A683B6822339B0013449B68DB686C
:10077000BB613B7E43F002033B767A683B682233E1
:100780009B0013449B68BA69DA607A683B6813443B
:1007900003F5637305221A700023FB613B7F43F06E
:1007A00010033B77FA69FB6E9A6000233B6297F86F
:1007B000203043F0080387F820303A6AFB6E9A60D5
:1007C00097F868306FF3041387F868303B68DBB242
:1007D00019467868FEF75EF93FE097F8693003F054
:1007E0000403DBB2002B38D07A683B6822339B00CD
:1007F00013449B68DB687B6297F8243043F0020364
:1008000087F824307A683B6822339B0013449B6846
:100810007A6ADA603B68DBB219467868FEF73AF923
:100820000023BB6297F8283043F0100387F8283084
:10083000BA6AFB6E9A607A683B68134403F5637387
:1008400008221A700023FB6297F82D3043F004034E
:1008500087F82D30FA6AFB6E9A6097F8693003F0DA
:100860000203DBB2002B27D07A683B6822339B005F
:1008700013449B68DB683B6397F8303043F0020316
:1008800087F830307A683B6822339B0013449B68BA
:100890003A6BDA603B68DBB219467868FEF7FAF823
:1008A00000237B6397F8353043F0020387F8353037
:1008B0007A6BFB6E9A60CBE197F8683003F0010326
:1008C000DBB2002B00F09B807B68DB78012B17D11B
:1008D0007A683B6822339B0013449B681B69FB6565
:1008E0007A683B685B01134403F56F731B68FA6D0C
:1008F000C2F31202991A7B683A68D43243F8221084
:100900007A683B68134403F5637301221A707A68AE
:100910003B68C4339B00134400225A600023BB632E
:1009200097F8383043F0010387F83830BA6BFB6E24
:100930009A6097F8623003F00C03DBB2002B06D00C
:1009400097F8623003F00C03DBB2082B39D17A68D8
:100950003B6822339B0013449B68DB68FB6397F87A
:100960003C3043F0020387F83C307A683B6822331E
:100970009B0013449B68FA6BDA603B68DBB2194654
:100980007868FEF787F800233B6497F8403043F01F
:10099000100387F840303A6CFB6E9A607A683B68C7
:1009A0001E335B01134404331B7883F00103D9B277
:1009B0007A683B681E335B01134404330A461A709D
:1009C00045E197F8623003F00C03DBB20C2B40F0EA
:1009D0003E8197F8633043F0200387F863307A68EC
:1009E0003B6822339B0013449B683A6E1A607A6816
:1009F0003B68134403F29B3301221A7028E197F8F5
:100A0000683003F00203DBB2002B7DD07A683B68CC
:100A100022339B0013449B68DB687B6497F8443067
:100A20006FF3410387F844307A683B6822339B00B8
:100A300013449B687A6CDA607A683B68134403F568
:100A400063731B78DBB2012B07D17A683B681344D0
:100A500003F29B3301221A704AE07A683B68134420
:100A600003F563731B78DBB2052B07D17A683B680B
:100A7000134403F29B3304221A7039E07A683B680E
:100A8000134403F563731B78DBB2062B08D07A6836
:100A90003B68134403F563731B78DBB2082B0ED15C
:100AA0007A683B68C4339B00134400225A607A681A
:100AB0003B68134403F29B3303221A7018E097F843
:100AC000623003F00C03DBB20C2B11D17A683B6867
:100AD0001E335B01134404331B7883F00103D9B246
:100AE0007A683B681E335B01134404330A461A706C
:100AF0000023BB6497F8483043F0020387F848307E
:100B0000BA6CFB6E9A60A3E097F8683023F07F031D
:100B1000DBB2002B3BD07A683B6822339B00134446
:100B20009B68DB68FB6497F84C3043F0020387F85E
:100B30004C307A683B6822339B0013449B68FA6C04
:100B4000DA607A683B68C4339B0013445B685A1CC4
:100B500079683B68C4339B000B445A607A683B68F1
:100B6000134403F5637306221A703B68DBB219461F
:100B70007868FDF78FFF00233B6597F8503043F00E
:100B8000800387F850303A6DFB6E9A6060E097F80A
:100B9000683003F01003DBB2002B59D097F86230B5
:100BA00003F00C03DBB20C2B1CD17A683B682233B8
:100BB0009B0013449B68DB687B6597F8543043F0D7
:100BC000020387F854307A683B6822339B00134451
:100BD0009B687A6DDA603B68DBB219467868FDF78E
:100BE00059FF21E097F8623003F00C03DBB2002BD1
:100BF00006D097F8623003F00C03DBB2082B13D158
:100C000097F8633043F0800387F8633097F86330D8
:100C10006FF3861387F863307A683B6822339B0052
:100C200013449B683A6E1A607A683B68134403F574
:100C3000637303221A700023BB6597F8583043F0A2
:100C4000100387F85830BA6DFB6E9A6000E000BF61
:100C5000012318467037BD4680BD00BF80B59AB0ED
:100C600000AF786039607A683B6822339B00134498
:100C70009B687B667B6E9B683B667B6EDB68FB6577
:100C80003A6EFB6D13403B667A683B6822339B00EB
:100C900013449B681B68BB6597F8603003F004033E
:100CA000DBB2002B1DD00023BB603B7A43F0040372
:100CB0003B72BA687B6E9A607A683B6822339B000D
:100CC00013449B68DB68FB603B7B43F002033B7390
:100CD0007A683B6822339B0013449B68FA68DA60A9
:100CE00060E297F8603003F02003DBB2002B09D0FC
:100CF00000233B613B7C43F020033B743A697B6EED
:100D00009A604FE297F8613003F00203DBB2002BE8
:100D100023D07A683B6822339B0013449B68DB68CE
:100D20007B613B7D43F002033B757A683B6822336D
:100D30009B0013449B687A69DA603B68DBB2194612
:100D40007868FDF7A7FE0023BB617B7E43F00203BA
:100D50007B76BA697B6E9A6024E297F8603003F084
:100D60000103DBB2002B33D07A683B68C4339B00AD
:100D7000134400225A607A683B6822339B00134474
:100D80009B68DB68FB613B7F43F002033B777A683B
:100D90003B6822339B0013449B68FA69DA603B6826
:100DA000DBB219467868FDF775FE00233B6297F8C1
:100DB000203043F0010387F820303A6A7B6E9A6056
:100DC0007A683B68134403F5637301221A70E9E102
:100DD00097F8603003F00803DBB2002B2ED000231D
:100DE0007B6297F8243043F0080387F824307A6A4E
:100DF0007B6E9A607A683B6822339B0013449B6841
:100E0000DB68BB6297F8283043F0020387F828308C
:100E10007A683B6822339B0013449B68BA6ADA60A5
:100E20003B68DBB219467868FDF734FE7A683B68A8
:100E3000134403F5637305221A70B3E197F8603029
:100E400003F01003DBB2002B35D07A683B68C43363
:100E50009B00134400225A607A683B6822339B004F
:100E600013449B68DB68FB6297F82C3043F0020365
:100E700087F82C307A683B6822339B0013449B68C8
:100E8000FA6ADA603B68DBB219467868FDF702FE61
:100E900000233B6397F8303043F0100387F830307D
:100EA0003A6B7B6E9A607A683B68134403F5637310
:100EB00003221A7076E197F8603023F07F03DBB2EB
:100EC000002B3BD07A683B6822339B0013449B681D
:100ED000DB687B6397F8343043F0020387F83430E3
:100EE0007A683B6822339B0013449B687A6BDA6014
:100EF0003B68DBB219467868FDF7CCFD7A683B6841
:100F0000C4339B0013445B685A1C79683B68C43344
:100F10009B000B445A607A683B68134403F5637383
:100F200006221A700023BB6397F8383043F0800321
:100F300087F83830BA6B7B6E9A6033E197F860308F
:100F400003F04003DBB2002B35D07A683B68C43332
:100F50009B00134400225A607A683B6822339B004E
:100F600013449B68DB68FB6397F83C3043F0020353
:100F700087F83C307A683B6822339B0013449B68B7
:100F8000FA6BDA603B68DBB219467868FDF782FDE0
:100F900000233B6497F8403043F0400387F840302B
:100FA0003A6C7B6E9A607A683B68134403F563730E
:100FB00004221A70F6E097F8613003F00403DBB204
:100FC000002B39D07A683B6822339B0013449B681E
:100FD000DB687B6497F8443043F0020387F84430C1
:100FE0007A683B6822339B0013449B687A6CDA6012
:100FF0003B68DBB219467868FDF74CFD0023BB6403
:1010000097F8483043F0100387F84830BA6C7B6E8D
:101010009A607A683B68134403F5637308221A7078
:101020000023FB6497F84D3043F0040387F84D30FC
:10103000FA6C7B6E9A60B5E097F8603003F00203BB
:10104000DBB2002B00F0AE807A683B6822339B0055
:1010500013449B68DB683B6597F850306FF341039E
:1010600087F850307A683B6822339B0013449B68B2
:101070003A6DDA607A683B68134403F563731B7852
:10108000DBB2012B20D17A683B68134403F29B3317
:1010900001221A7097F85A3003F00C03DBB2082BC8
:1010A00074D17A683B681E335B01134405331B78A7
:1010B00083F00103D9B27A683B681E335B011344A5
:1010C00005330A461A7062E07A683B68134403F5F8
:1010D00063731B78DBB2032B07D17A683B68134438
:1010E00003F29B3302221A7051E07A683B68134482
:1010F00003F563731B78DBB2042B16D17A683B6867
:101100005B01134403F56C731B78012B05D13B681D
:10111000DBB219467868FDF7A9FC7A683B6813448E
:1011200003F29B3302221A7031E07A683B68134461
:1011300003F563731B78DBB2052B07D17A683B6834
:10114000134403F29B3304221A7020E07A683B6850
:10115000134403F563731B78DBB2062B17D17A684F
:101160003B68C4339B0013445B68032B0FD17A6840
:101170003B68134403F29B3303221A707A683B687E
:10118000C4339B00134400225A6000E000BF0023D8
:101190007B6597F8543043F0020387F854307A6D3A
:1011A0007B6E9A60012318466837BD4680BD00BF3C
:1011B00080B588B000AF78600023FB610023BB617D
:1011C0000023FB6000237B6100233B617B68D3F835
:1011D000CC301B687B617B68D3F8CC301B683B61EB
:1011E0003B7C6FF382033B743B7C6FF341033B74A6
:1011F0003B7C6FF3C3033B743B7C6FF345133B7441
:101200003B7D03F00203DBB2002B0CD03B7C43F0B0
:1012100002033B743F4B1B685B6878689847BB6967
:1012200043F00103BB613B7D03F00803DBB2002BFD
:1012300052D03B7C43F008033B743B7D03F0040336
:10124000DBB2002B48D0334B1B685B68786898474B
:10125000BB7D03F00603DBB2042B05D0BB7D03F09E
:101260000603DBB2022B31D17B685B691B68FB6034
:10127000BB7D03F00603DBB2042B15D17B685B69F1
:1012800041F270725A603B7B03F00303DBB2022B26
:101290001FD07B681B7A022B03D102217868FDF7EF
:1012A00037FD0123FB6116E07B685B694BF68032FA
:1012B0005A603B7B03F00303DBB2012B0BD001210F
:1012C0007868FDF725FD0123FB6104E00123FB6144
:1012D00002E000BF00E000BF3B7D03F02003DBB273
:1012E000002B07D03B7C43F020033B74BB6943F0E9
:1012F0000103BB61FB69002B02D07868FDF74EFD4E
:101300007B68D3F8CC303A691A60BB69184620373D
:10131000BD4680BD5071010880B586B000AF7860D1
:101320007B685B691B69BB603B7BC3F3C303DBB2B8
:101330007A685B01134403F56F731B6803339B08E2
:10134000FB8296E03B899B00BB82BA8A3B7BC3F35E
:10135000C303DBB279685B010B4403F56F731B6851
:101360009A4219D93B7BC3F3C303DBB27A685B01B2
:10137000134403F56F731B68BB8200233B61FB7C46
:1013800043F00403FB747B68DB687A68D268916978
:101390003A69D2430A409A613B7BC3F3C303DBB291
:1013A0007A685B01134403F56F731B6803339B0872
:1013B000FB823B7BC3F3C303DBB27A6815335B016B
:1013C000134403F58C7319683B7BC3F3C303DBB28F
:1013D0001A46BB8A7868FDF7B5FC3B7BC3F3C303B1
:1013E000DBB218463B7BC3F3C303DBB27A68153329
:1013F0005B01134403F58C731A68BB8A1A4479683D
:1014000000F115035B010B4403F58C731A603B7B01
:10141000C3F3C303DBB218463B7BC3F3C303DBB2A6
:101420007A685B01134403F56F731A68BB8AD21A9A
:10143000796843010B4403F56F731A603B7BC3F378
:10144000C303DBB218463B7BC3F3C303DBB27A684A
:101450005B01134403F570731A68BB8A1A447968F8
:1014600043010B4403F570731A607B685B691B6969
:10147000BB603B89FA8A9A420CD23B7BC3F3C3031D
:10148000DBB27A685B01134403F56F731B68002BB2
:101490007FF458AF012318461837BD4680BD00BF02
:1014A00080B588B000AF78607B68DB68DB6AFB6082
:1014B0003B7CC3F3C303DBB27A685B01134403F5DF
:1014C0006F731B6803339B08FB8396E0BB899B000B
:1014D000BB83BA8B3B7CC3F3C303DBB279685B018C
:1014E0000B4403F56F731B689A4219D93B7CC3F315
:1014F000C303DBB27A685B01134403F56F731B68A7
:10150000BB830023BB613B7E43F020033B767B68BB
:10151000DB687A68D2689169BA69D2430A409A61F5
:101520003B7CC3F3C303DBB27A685B01134403F56E
:101530006F731B6803339B08FB833B7CC3F3C303BC
:10154000DBB27A6815335B01134403F58C731968B9
:101550003B7CC3F3C303DBB21A46BB8B7868FDF751
:10156000F1FB3B7CC3F3C303DBB218463B7CC3F304
:10157000C303DBB27A6815335B01134403F58C7344
:101580001A68BB8B1A44796800F115035B010B44A0
:1015900003F58C731A603B7CC3F3C303DBB21846BC
:1015A0003B7CC3F3C303DBB27A685B01134403F5EE
:1015B0006F731A68BB8BD21A796843010B4403F529
:1015C0006F731A603B7CC3F3C303DBB218463B7CEA
:1015D000C3F3C303DBB27A685B01134403F5707392
:1015E0001A68BB8B1A44796843010B4403F5707386
:1015F0001A607B68DB68DB6AFB60BB89FA8B9A4206
:101600000CD23B7CC3F3C303DBB27A685B011344A7
:1016100003F56F731B68002B7FF458AF0123184646
:101620002037BD4680BD00BF80B584B000AF786074
:101630000023FB60084B1B689B6878689847FB7B1E
:1016400043F02003FB737B68DB68FA685A6101236F
:1016500018461037BD4680BD5071010880B584B072
:1016600000AF78600023FB60084B1B681B6878683C
:1016700098473B7B43F008033B737B68DB68FA6861
:101680005A61012318461037BD4680BD50710108CC
:101690002DE9F043DFF84C80D8F80030984283B051
:1016A0001AD20F4E05460F1A06EB001600244FF013
:1016B0001409002331462046CDF800903A4601F047
:1016C00015FED8F800300135AB4204F1010406F1F3
:1016D000100601D9142CECD103B0BDE8F08300BF93
:1016E0004CB801200CB8012004F08EB810B5094B9D
:1016F000402000220C244FF4806198605C601961E6
:101700001A60DA6001F00CFB2046BDE81040FDF7DE
:10171000AFBE00BFC0BD012038B50F4A0F4B1268E5
:10172000002012044FF480610D244025D8601A6017
:101730009D6019615C6001F0F3FA2046FDF798FEA8
:1017400008B1022038BDFBF74BF8C0F34320043842
:1017500018BF012038BD00BF00B80120C0BD012066
:1017600038B52A4B19685A69140601D5080600D401
:1017700038BD8021264A596113691906F8D41369C6
:101780005B060ED4234A1378591E072903D8224832
:101790000178490801700133DBB20A2B0DD81370B0
:1017A00038BD1C4A1378591E0729F4D81A48017805
:1017B000490861F07F010170EDE7174C20780023A4
:1017C000F028137013D0E02817D0144D144A2B883A
:1017D00011881843814205D0124B10801B6893B1C9
:1017E000114B186000232B600023237038BD0B4A77
:1017F000136843F400731360F6E7084A136843F470
:1018000080731360F0E7FEF7FDF8EBE7003C014062
:101810000004024048B8012049B8012008B801205E
:101820004CBC012040B80120BCB7012038B5104C99
:10183000104D03E00020FEF7ABF948B92368002BF8
:10184000F8D1FEF74BF90020FEF7A2F90028F5D0F9
:101850002B68022B06D0FEF78FFB0028EED1064B3B
:10186000186038BDFEF7ACFB0028E7D1F7E700BFF2
:101870003CB8012044B8012004B80120F0B5254A45
:10188000254B127883B053F822702025002304469C
:1018900002460E4618463946009501F027FD2246BD
:1018A00000231E490095012001F020FD224600235F
:1018B0001B490095022001F019FD009522460023E6
:1018C0001849032001F012FD0095DEB93346224687
:1018D0001549042001F00AFD202522460095002329
:1018E0001249052001F002FD114A124B92F88020A6
:1018F000009553F8221006202246002301F0F6FC42
:1019000003B0F0BD012322460B49042001F0EEFC98
:10191000E2E700BFC4000020A4710108BC71010807
:10192000C8600108E4600108D0710108D87101089D
:1019300074A50120B4710108C47101082DE9F843B0
:10194000644BD3F8C4305A0711D4634B1C6800228F
:101950001A604CB9614B1B6833B1614B1B68012B9A
:1019600000F08480002B59D02046BDE8F8835D4C00
:10197000DFF888915C4E00274FF0FF054FF001081B
:1019800008FA07F3DB43DBB2A9F81A500F20A9F8D5
:101990001830FAF73FFE3369DB4303F01F03474477
:1019A000042004F8013FFAF727FE082FE6D14F483C
:1019B0000778FB0711D54E4D02792B795340DF068E
:1019C00035D512F0100F444B40F2723418BF4FF46B
:1019D000B97403C885E80300B9E7C37903F00203CB
:1019E00003F0FF017BBB424DDFF814C10A46864677
:1019F00077B1AE5C00237E4008FA03F4344212D083
:101A000002EB82010B443CF8131009B127424BD082
:101A10000132082A25D01EF8017FE9E7FEF75EF8BB
:101A20002046BDE8F8830133052BE5D1F0E71E071A
:101A300030D4DC073BD512F0010F40F26624264B70
:101A400018BF6624C5E72A4D8279AB7953401B073E
:101A500009D512F0080F40F24A241F4B18BF4A2440
:101A6000B7E7002933D11C4B1C68B2E72046FEF7CC
:101A70008FF800283FF478AF1E4B1B68022B23D051
:101A8000FEF77AFA1C4B1A6882423FF46DAF186079
:101A9000044669E740F2751312F0080F40F27534FE
:101AA00018BF1C460C4B94E741F40071B0E7C279B3
:101AB000EB795340D907D6D512F0010F40F27624C6
:101AC000054B18BF762484E7FEF77AFADAE7024B73
:101AD0000C467EE774A50120BCB7012018B8012090
:101AE0003CB801200FB801200010024010B80120BE
:101AF0001CB8012044B8012004B8012000080240AD
:101B000054710108F0B583B00024064600942146C4
:101B100040F2DF1340F21F324FF41670FDF704FC61
:101B2000002E63D000944FF6FF734FF416722021FD
:101B30006848FCF733FF684D00232B70FCF766F80C
:101B4000664B1B68002B40F0BD80FFF7F7FE0024BA
:101B5000762827463CD01538512832D8DFE800F0E7
:101B60005C5A3131315856545250313129B0AEACF3
:101B7000AAA8313131A6A4A2A09E31319C9A989690
:101B80009492313131908E8C8A88313131868482C1
:101B9000807E3131317C7A317831313131313131BE
:101BA00031313131316531313131313131313131F1
:101BB000315E6323062C04D82B5501342F55FCF7D6
:101BC00025F80120FDF708F9FFF7B8FE7628C2D105
:101BD00000240021009140F2DF1340F21F324FF445
:101BE0001670FDF7A1FB204603B0F0BD00964FF63E
:101BF000FF734FF4167220213948FCF7CFFE9AE7A5
